:100000000C94E9100C94E2130C940D140C94381415
:100010000C9463140C948E140C94B9140C94E41482
:100020000C940F150C9419110C9419110C941911AE
:100030000C9419110C9419110C9419110C94191198
:100040000C9419110C9462320C9419110C9419111E
:100050000C9419110C9419110C949F260C941B11DB
:100060000C9419110C9432170C94DE170C9419117E
:100070000C9419110C9419110C9419110C94191158
:100080000C9419110C9419110C9419110C94191148
:100090000C9419110C9419110C9419110C94191138
:1000A0000C9419110C9419110C9419110C94191128
:1000B0000C9419110C9419110C9419110C94191118
:1000C0000C9419110C9419110C9419110C94191108
:1000D0000C9419110C9419110C9419110C941911F8
:1000E0000C94191158125D1262126C127612EF12F2
:1000F0008012881290129A12A412AE12BD12C71268
:10010000EF12D112DB12E5121313161305130913A4
:100110000F134D131A131E13241328132C13321309
:1001200036133A134D1340134413481365176B17D6
:100130007C1787178F17A4179317A41797179B1768
:10014000A417A117491F471F701F6D1F6B1FA71F03
:10015000A41FA21F0020CE1FCB1FC91F084AD73BD8
:100160003BCE016E84BCBFFDC12F3D6C74319ABD86
:1001700056833DDA3D00C77F11BED9E4BB4C3E91AA
:100180006BAAAABE000000803F05A84CCDB2D44E99
:10019000B93836A9020C50B9918688083CA6AAAA9B
:1001A0002ABE000000803F004E414E494E4954593E
:1001B000494E46CDCCCC3D0AD7233C17B7D1387732
:1001C000CC2B329595E6241FB14F0A000020410048
:1001D00000C84200401C4620BCBE4CCA1B0E5AAE92
:1001E000C59D7400000A0B02090C0D0E08070304DC
:1001F00001000000000000000000000000000000FE
:1002000000000000000000000000000000000012DC
:1002100011100000000000000000000000000000BD
:10022000000000000000000000010210202008086B
:100230001020401020408002010201080402010148
:100240000204081020408080402010080402018031
:100250000402018040201008040201080402010188
:10026000020408102040800102040810204080058C
:10027000050505070508080808020202020A0A081F
:100280000804040404010101010101010103030345
:100290000303030303040707070C0C0C0C0C0C0CE2
:1002A0000C0202020206060606060606060B0B0BE9
:1002B0000B0B0B0B0B000020002300260029002C49
:1002C000002F0032000001000003010601090100B7
:1002D000002200250028002B002E003100340002EF
:1002E000010000050108010B010000210024002786
:1002F000002A002D00300033000101000004010736
:10030000010A014F4646004F4E006563686F3A0090
:100310004572726F723A004572726F72207772691D
:1003200074696E6720746F20454550524F4D210A05
:100330000063616E63656C00706F7765726F6666EF
:10034000002F2F616374696F6E3A0020573A0020C6
:10035000573A00202F002042403A0020403A0054F3
:100360006865726D616C2052756E617761790045C8
:100370003120544845524D414C2052554E41574131
:10038000590042656400202D20496E76616C6964D5
:10039000206578747275646572206E756D62657221
:1003A00020210A0048656174696E67206661696C86
:1003B0006564004265640048656174696E67206623
:1003C00061696C65640045312048656174696E67D8
:1003D000206661696C6564004D494E54454D50205E
:1003E0007472696767657265640045312045727291
:1003F0003A204D494E54454D5000426564004D41F0
:100400005854454D50207472696767657265640081
:100410004531204572723A204D415854454D5000A7
:1004200042656400626564002C2073797374656DA5
:100430002073746F70706564212048656174657203
:100440005F49443A200023646566696E652044452F
:100450004641554C545F004B6420004B6920004BD3
:100460007020000062656400504944204175746F3B
:1004700074756E652066696E6973686564212050C5
:10048000757420746865206C617374204B702C2027
:100490004B6920616E64204B6420636F6E737461DE
:1004A0006E74732066726F6D2062656C6F77206961
:1004B0006E746F20436F6E66696775726174696FE1
:1004C0006E2E680A00504944204175746F74756E31
:1004D00065206661696C6564212074696D656F755E
:1004E000740A00546865726D616C2052756E617794
:1004F000617900453120544845524D414C205255B8
:100500004E41574159004265640048656174696E07
:1005100067206661696C65640045312048656174D7
:10052000696E67206661696C6564004265640050AD
:100530004944204175746F74756E65206661696CFD
:100540006564212054656D706572617475726520F3
:10055000746F6F20686967680A00204B643A200056
:10056000204B693A2000204B703A20000A20436C4F
:10057000617373696320504944200A002054753A1E
:100580002000204B753A2000206D61783A20002031
:100590006D696E3A200020643A2000206269617320
:1005A0003A2000504944204175746F74756E65207F
:1005B00073746172740A00504944204175746F74F9
:1005C000756E65206661696C6564212054656D7087
:1005D0006572617475726520746F6F2068696768F1
:1005E0000A001000AD0330016A0150022B017003B4
:1005F0000A019004F500B005E500D006D800F00728
:10060000CE001009C500300ABE00500BB700700CB8
:10061000B100900DAB00B00EA600D00FA200F010FC
:100620009D0010129900301395005014920070151F
:100630008E0090168B00B0178700D0188400F01938
:100640008100101B7E00301C7B00501D7900701E45
:100650007600901F7300B0207000D0216E00F02251
:100660006B00102469003025660050266300702757
:10067000610090285E00B0295C00D02A5900F02B60
:100680005600102D5400302E5100502F4E00703067
:100690004B0090314800B0324500D0334200F03476
:1006A0003E0010363B003037370050383300703989
:1006B0002E00903A2900B03B2300D03C1B00F03DB7
:1006C0001100103F0100F03F00001000C9021001AE
:1006D0002C014001220170011801B0010E01F0014E
:1006E00004015002FA00B002F0003003E600D0032B
:1006F000DC009004D2007005C800A006BE0000080F
:10070000B400B009AA00D00BA000600E96006011E2
:100710008C000015820020197800C01D6E00A022F8
:100720006400B0275A00902C500000314600E0349D
:100730003C0010383200903A2800603C1E00A03D7A
:100740001400803E0A00203F00006F70656E005468
:100750005249474745524544003A20007A5F6D614F
:1007600078007A5F6D696E00795F6D617800795FFE
:100770006D696E00785F6D617800785F6D696E00FD
:100780005265706F7274696E6720656E6473746F02
:1007900070207374617475730A00205A3A002059EE
:1007A0003A0020583A00656E6473746F7073206865
:1007B00069743A2000486F6D696E67206661696CE4
:1007C000656400496E76616C696420657874727541
:1007D0006465720A0045303A20005A3A2000593ABE
:1007E00020004D53312C4D53322C4D533320506942
:1007F0006E730A583A20004D6963726F73746570A6
:100800007320756E617661696C61626C650A0020A7
:100810005A3A0020593A0020436F756E7420583AB6
:1008200000C23100001C260000F4190000D80F009F
:1008300000EB080000C00400007502000040010049
:100840000024F4D43050C38E20C2A24017828B7093
:1008500011127A910D816CD90AA861E108C7586616
:1008600007615143061E4B5D05C145A7041A41119E
:1008700004093D9803713931034036DB0265339139
:1008800002D4305402802E1D02632CEE01752AC55D
:1008900001B028A001102781018F2564012B244B72
:1008A00001E0223401AC211F018D200D01801FFCCD
:1008B00000841EED00971DDF00B81CD200E61BC6A9
:1008C00000201BBC00641AB200B219A8000A19A0CB
:1008D000006A189900D117910040178B00B5168453
:1008E0000031167E00B31579003A157300C7146FF6
:1008F0000058146A00EE1366008813630025135E27
:1009000000C7125B006C12570015125400C1115140
:100910000070114F0021114B00D61049008D104777
:10092000004610440002104200C00F4000800F3EFD
:1009300000420F3C00060F3B00CB0E3800930E37F1
:10094000005C0E3500270E3400F30D3200C10D316E
:1009500000900D3000600D2E00320D2D00050D2C85
:1009600000D90C2B00AE0C2900850C29005C0C274B
:1009700000350C27000E0C2600E80B2400C40B24C5
:1009800000A00B23007D0B23005A0B2100390B2103
:1009900000180B2000F80A1F00D90A1E00BB0A1E0F
:1009A000009D0A1D00800A1D00630A1C00470A1BE7
:1009B000002C0A1B00110A1A00F7091A00DD091998
:1009C00000C4091900AB091900920917007B091826
:1009D00000630917004C0916003609160020091695
:1009E000000A091500F5081500E0081400CC0814E9
:1009F00000B8081400A4081400900813007D081221
:100A0000006B081300580812004608120034081141
:100A100000230811001208110001081100F007104E
:100A200000E0071000D0071000C0071000B0070F4B
:100A300000A107100091070E0083070F0074070F35
:100A40000065070E0057070E0049070E003B070D13
:100A5000002E070E0020070D0013070D0006070DDE
:100A600000F9060C00ED060D00E0060C00D4060CA3
:100A700000C8060C00BC060C00B0060C00A4060B57
:100A80000099060C008D060B0082060B0077060B02
:100A9000006C060B0061060A0057060B004C060AA4
:100AA0000042060A0038060A002E060A0024060A3A
:100AB000001A060A001006090007060A00FD0509CB
:100AC00000F4050900EB050900E2050900D9050954
:100AD00000D0050900C7050900BE050900B50508D5
:100AE00000AD050800A50509009C0508009405084F
:100AF000008C050800840508007C050800740508C2
:100B0000006C050700650508005D0507005605082F
:100B1000004E050700470507004005080038050797
:100B200000310507002A050700230507001C0506FC
:100B300000160507000F0507000805060002050757
:100B400000FB040600F5040700EE040600E80406B6
:100B500000E2040700DB040600D5040600CF04060B
:100B600000C9040600C3040600BD040600B704065D
:100B700000B1040500AC040600A6040600A00405AC
:100B8000009B04060095040500900406008A0405F5
:100B90000085040500800406007A0405007504053C
:100BA00000700405006B040500660405006104057F
:100BB000005C04050057040500520405004D0405BF
:100BC0000048040500430405003E0404003A0405FF
:100BD0000035040500300404002C0405002704043B
:100BE00000230405001E0404001A04040016040572
:100BF00000110404000D04040009040500040404A9
:100C00000000040400FC030400F8030400F40304DF
:100C100000F0030400EC030400E8030400E4030410
:100C200000E0030400DC030400D8030400D4030440
:100C300000D0030400CC030400C8030300C5030371
:100C40000024F404D9201BC40C5C0E9804C4095F72
:100C50000265077101F405F900FB04B3004804873D
:100C600000C10369005803550003034500BE023A62
:100C7000008402310053022A0029022500040220C8
:100C800000E4011C00C8011900AF0117009801140D
:100C90000084011300710110006101100051010E68
:100CA0000043010D0036010B002B010B0020010B4E
:100CB00000150109000C01090003010800FB0008F0
:100CC00000F3000800EB000700E4000600DE000669
:100CD00000D8000600D2000600CC000500C70005C1
:100CE00000C2000500BD000400B9000400B5000406
:100CF00000B1000400AD000400A9000400A5000339
:100D000000A20003009F0004009B00030098000362
:100D1000009500020093000300900003008D000284
:100D2000008B00030088000200860002008400039C
:100D300000810002007F0002007D0002007B0002B3
:100D400000790002007700010076000200740002C2
:100D50000072000100710002006F0002006D0001CE
:100D6000006C0002006A00010069000200670001D7
:100D700000660001006500010064000200620001DD
:100D80000061000100600001005F0002005D0001E1
:100D9000005C0001005B0001005A000100590001E5
:100DA00000580001005700010056000100550001E5
:100DB00000540001005300000053000100520001E4
:100DC0000051000100500001004F0001004E0000E2
:100DD000004E0001004D0001004C0001004B0000DE
:100DE000004B0001004A00010049000100480000DA
:100DF00000480001004700010046000000460001D5
:100E000000450000004500010044000100430000CF
:100E100000430001004200000042000100410000C8
:100E20000041000100400001003F0000003F0001C0
:100E3000003E0000003E0001003D0000003D0001BA
:100E4000003C0000003C0000003C0001003B0000B2
:100E5000003B0001003A0000003A000100390000A8
:100E6000003900010038000000380000003800019F
:100E70000037000000370001003600000036000097
:100E8000003600010035000000350000003500018B
:100E90000034000000340000003400010033000082
:100EA0000033000000330001003200000032000077
:100EB000003200010031000000310000003100016B
:100EC000003000000030000000300001002F000062
:100ED000002F0000002F0000002F0001002E000056
:100EE000002E0000002E0001002D0000002D00004B
:100EF000002D0000002D0001002C0000002C00003F
:100F0000002C0000002C0001002B0000002B000032
:100F1000002B0000002B0001002A0000002A000026
:100F2000002A0000002A000100290000002900001A
:100F3000002900000029000000290001002800000D
:100F40000028000000280000002800000028000100
:100F500000270000002700000027000000270000F5
:100F600000270001002600000026000000260000E7
:100F700000260000002600010025000000250000DA
:100F800000250000002500000025000000250001CC
:100F900000240000002400000024000000240000C1
:100FA00000240001002300000023000000230000B3
:100FB00000230000002300000023000000230001A4
:100FC0000022000000220000002200000022000099
:100FD000002200000022000100210000002100008A
:100FE000002100000021000000210000002100007D
:100FF000002100010020000000200000002000006F
:101000000020000000200000002000000020000060
:1010100000200001001F0000001F0000001F000052
:10102000001F0000001F0000001F0000001F000143
:10103000001E0000001E0000001E0000001E000038
:10104000003A0A0020286D6D2900204500205A0032
:1010500020204D3930372058005374657070657208
:10106000206D6F746F722063757272656E74733A5F
:101070000A0020204D393030204B004C696E6561EC
:101080007220416476616E63653A0A0020204D3813
:101090003531205A005A2D50726F6265204F6666B6
:1010A0007365740020440020490020204D33303403
:1010B00020500020440020490020204D33303120B2
:1010C00050005049442073657474696E67733A0A1E
:1010D0000020204D3432302053004175746F20427F
:1010E0006564204C6576656C696E673A0A00204538
:1010F00000205A002059002058002054002053009E
:1011000020204D32303520420020453C6D61785F13
:10111000655F6A65726B3E0020583C6D61785F7850
:101120005F6A65726B3E20593C6D61785F795F6ADA
:1011300065726B3E205A3C6D61785F7A5F6A6572BA
:101140006B3E00416476616E6365643A20423C6D9B
:10115000696E5F7365676D656E745F74696D655FF9
:1011600075733E20533C6D696E5F666565647261A0
:1011700074653E20543C6D696E5F74726176656C77
:101180005F66656564726174653E0020540020529C
:101190000020204D323034205000416363656C657F
:1011A000726174696F6E2028756E6974732F733263
:1011B000293A20503C7072696E745F616363656C9C
:1011C0003E20523C726574726163745F6163636553
:1011D0006C3E20543C74726176656C5F616363653C
:1011E0006C3E0A00204500205A0020590020204D66
:1011F0003230312058004D6178696D756D20416342
:1012000063656C65726174696F6E2028756E6974B0
:10121000732F7332293A0A00204500205A002059C2
:101220000020204D3230332058004D6178696D75B3
:101230006D206665656472617465732028756E69DA
:1012400074732F73293A0A005374657073207065A4
:101250007220756E69743A0A0020204732312020CE
:1012600020203B20556E69747320696E206D6D00DF
:1012700048617264636F6465642044656661756C7F
:10128000742053657474696E6773204C6F61646574
:10129000640A00282300002823000064000000E8FE
:1012A0000300000000964300009643000000410048
:1012B0000020420000C9420000C9420000C84400AA
:1012C00000D243290A002062797465733B2063725F
:1012D0006320002073746F72656420736574746991
:1012E0006E67732072657472696576656420280084
:1012F000202863616C63756C6174656429210A0040
:1013000020213D2000454550524F4D20435243205F
:101310006D69736D61746368202D202873746F721A
:1013200065642920002053697A653A2000496E647B
:1013300065783A2000204D61726C696E3D563634F6
:10134000290A00454550524F4D2076657273696FEA
:101350006E206D69736D6174636820284545505235
:101360004F4D3D00290A002062797465733B20636C
:101370007263200053657474696E67732053746FD1
:10138000726564202800454550524F4D20646174B9
:101390006173697A65206572726F722E0A005072ED
:1013A0006F62696E67206661696C65640A005761E7
:1013B000726E696E673A20486F6D696E672042757C
:1013C0006D702044697669736F72203C20310A0089
:1013D0000202042066697273740A00486F6D65200A
:1013E0000020746F6F206C6F6E6720657874727563
:1013F00073696F6E2070726576656E7465640A003D
:1014000020636F6C6420657874727573696F6E20E9
:1014100070726576656E7465640A0020453A002036
:101420005A3A0020593A00583A000000F0410000B2
:10143000F04100000041FF01010000A0400000A0B9
:10144000400000004000002543000045430000210B
:1014500043000040C000003E4300001F4300002244
:101460004300003E4300001F43000040C00000E076
:10147000C0000000C020746F6F206C6F6E67206525
:101480007874727573696F6E2070726576656E74AC
:1014900065640A0020636F6C6420657874727573EC
:1014A000696F6E2070726576656E7465640A00629D
:1014B0007573793A2070617573656420666F722068
:1014C000696E7075740A00627573793A207061757F
:1014D00073656420666F7220757365720A006275A9
:1014E00073793A2070726F63657373696E670A006F
:1014F0004D3131372050726F6265207375636365BB
:10150000737366756C0A0020496E76616C6964209D
:1015100065787472756465722000205A3A20002044
:10152000593A200042656420583A200050726F6298
:1015300065205A204F66667365743A20003F5A2032
:101540006F7574206F662072616E676520282D327A
:1015500020746F2035290A00220A00556E6B6E6FC9
:10156000776E20636F6D6D616E643A202200454591
:1015700050524F4D204F4B0A004543484F00494EB3
:10158000464F004552524F52530044525952554E05
:1015900000434F4D4D554E49434154494F4E006F06
:1015A00066660079157E1583158A159115444542A6
:1015B00055473A00205A00205900580020204D611C
:1015C000783A2000205A00205900580020204D6908
:1015D0006E3A2000536F667420656E6473746F708A
:1015E000733A20002569730025696D202569730011
:1015F0002569682025696D202569730025696420A7
:101600002569682025696D20256973002569792081
:10161000256964202569682025696D202569730086
:101620005072696E742074696D653A20004D3131D5
:10163000332053002F2F20004361703A004D4F5448
:10164000494F4E5F4D4F44455300544845524D411C
:101650004C5F50524F54454354494F4E00415554EE
:101660004F5245504F52545F53445F535441545569
:10167000530050524F4D50545F535550504F525499
:1016800000454D455247454E43595F5041525345E1
:101690005200434153455F4C494748545F425249C9
:1016A0004748544E45535300544F47474C455F4CB1
:1016B000494748545300534F4654574152455F5091
:1016C0004F574552004255494C445F50455243459F
:1016D0004E54004C4556454C494E475F4441544199
:1016E000005A5F50524F4245004155544F4C4556A9
:1016F000454C005052494E545F4A4F420050524FA1
:101700004752455353004155544F5245504F525440
:101710005F54454D5000564F4C554D45545249432A
:1017200000454550524F4D0042494E4152595F4687
:10173000494C455F5452414E534645520053455221
:1017400049414C5F584F4E5F584F464600464952FC
:101750004D574152455F4E414D453A4D61726C695E
:101760006E20204649524D574152455F56455253CF
:10177000494F4E3A322E302E302E313031204558DE
:101780005452554445525F545950453A536D616C1B
:101790006C4C6179657220534F555243455F434FFE
:1017A00044455F55524C3A68747470733A2F2F63F6
:1017B0006F64652E616C6570686F626A65637473CF
:1017C0002E636F6D2F646966667573696F6E2F4D3A
:1017D00041524C494E2050524F544F434F4C5F564C
:1017E000455253494F4E3A312E30204D41434849DE
:1017F0004E455F545950453A4C756C7A426F74208F
:101800004D696E692045585452554445525F434FC7
:10181000554E543A3120555549443A3335313438D0
:101820003762362D636139612D346331612D38376C
:1018300036352D6436363862316461363538350ACE
:101840000020284E6F7420796574206D6561737572
:101850007265642900202041766572616765206D9C
:1018600065617375726564206261636B6C61736836
:1018700020286D6D293A002020536D6F6F746869C0
:101880006E6720286D6D293A2020202020202020FE
:10189000202020202020202020530020204261638F
:1018A0006B6C6173682044697374616E6365202892
:1018B0006D6D293A2020202020202020002020208B
:1018C00020202846312E30203D2066756C6C2C205F
:1018D00046302E30203D206E6F6E65290A00202094
:1018E000436F7272656374696F6E20416D6F756EC0
:1018F000742F466164652D6F75743A202020202076
:1019000046006163746976653A0A00696E00426157
:10191000636B6C61736820636F7272656374696F67
:101920006E2069732000205A0020506F736974691B
:101930006F6E616C204572726F723A0A004E6F7A58
:101940007A6C6520546970204F7574657220446903
:101950006D656E73696F6E733A0A002020546F7064
:101960003A2000202046726F6E743A200020204CEE
:101970006566743A20004261636B6C6173683A0A71
:1019800000205A0043656E7465723A0A00202046B2
:10199000726F6E743A200020204C6566743A200005
:1019A0002020546F703A200053696465733A0A002E
:1019B000426564204C6576656C696E6720004661FF
:1019C000696C656420746F20656E61626C6520428D
:1019D0006564204C6576656C696E670A00426564D3
:1019E000204C6576656C20436F7272656374696F15
:1019F0006E204D61747269783A000A0A426564206B
:101A00004C6576656C20436F7272656374696F6EA6
:101A1000204D61747269783A00202B000A436F727E
:101A2000726563746564204265642048656967680F
:101A3000742076732E2042656420546F706F6C6F33
:101A400067793A0A00202B000A42656420486569DC
:101A500067687420546F706F6772617068793A0AB2
:101A60002020202B2D2D2D204241434B202D2D2B8E
:101A70000A2020207C202020202020202020202020
:101A80007C0A204C207C20202020282B292020206C
:101A9000207C20520A2045207C202020202020204D
:101AA000202020207C20490A2046207C20282D2927
:101AB000204E20282B29207C20470A2054207C20DF
:101AC000202020202020202020207C20480A2020A8
:101AD000207C20202020282D29202020207C2054FC
:101AE0000A2020207C2020202020202020202020B0
:101AF0007C0A2020204F2D2D2046524F4E54202D61
:101B00002D2B0A2028302C30290A003474682070CC
:101B1000726F626520706F696E742C2064697374D3
:101B2000616E63652066726F6D20706C616E653AE0
:101B30002000202844525952554E2900473239205E
:101B40004175746F20426564204C6576656C696EE2
:101B500067003F20284C2C522C462C4229206F75C0
:101B600074206F6620626F756E64732E0A003F509A
:101B7000726F626520706F696E7473202859292016
:101B8000697320696D706C61757369626C6520287A
:101B9000322D32292E0A003F50726F626520706F1D
:101BA000696E74732028582920697320696D706CE0
:101BB00061757369626C652028322D32292E0A0006
:101BC0003F2856296572626F7365206C6576656C77
:101BD00020697320696D706C61757369626C652032
:101BE00028302D34292E0A00416476616E63652009
:101BF0004B3D003F4B2076616C7565206F757420FE
:101C00006F662072616E67652028302D3130292E75
:101C10000A004D31313720486F7420456E642048EA
:101C2000656174696E672E2E2E0A4D313034205353
:101C30003137302054300A473238204F310A47318B
:101C400020593235205A31302046353030300A4D57
:101C500031303920523137302054300A4D3131374C
:101C6000205265776970696E67206E6F7A7A6C654D
:101C70000A54300A47312058343520593137322040
:101C800046353030300A4731205A310A4D3130392B
:101C900020523137300A47312058343520593137F6
:101CA000322046343030300A4731205834352059FC
:101CB0003137322046343030300A473120583435FD
:101CC00020593137322046343030300A47312058DD
:101CD000343520593137322046343030300A4731DC
:101CE0002058343520593137322046343030300ACC
:101CF000473120583435205931373220463430307E
:101D0000300A473120583435205931373220463493
:101D10003030300A4731205834352059313732209D
:101D200046343030300A4731205834352059313765
:101D3000322046343030300A47312058343520596B
:101D40003137322046343030300A4731205834356C
:101D500020593137322046343030300A473120584C
:101D6000343520593137322046343030300A47314B
:101D7000205A31350A4D3130362053323535200A5C
:101D800047302058302059300A4D313039205231F7
:101D900036302054300A4D3130370A0020466C6FFF
:101DA000773A200020643A0020693A0020703A0017
:101DB000204500205A00205900204D39322058007B
:101DC00043290A0061626C656420286D696E207485
:101DD000656D70200064697300656E00436F6C640C
:101DE00020657874727564657320617265200020C7
:101DF0005400205200416363656C65726174696FC1
:101E00006E3A205000496E76616C69642065787482
:101E100072756465720A0020643A0020693A0020F5
:101E2000703A0047322F473320626164207061723C
:101E3000616D65746572730A005072696E746572C3
:101E40002073746F707065642064756520746F20F2
:101E50006572726F72732E204669782074686520EF
:101E60006572726F7220616E6420757365204D39E2
:101E7000393920746F20726573746172742E202852
:101E800054656D7065726174757265206973207236
:101E9000657365742E2053657420697420616674BF
:101EA00065722072657374617274696E67290A00C5
:101EB0004E6F20436865636B73756D207769746836
:101EC000206C696E65206E756D6265722C204C61A8
:101ED0007374204C696E653A2000636865636B73A8
:101EE000756D206D69736D617463682C204C61732E
:101EF00074204C696E653A20004C696E65204E7501
:101F00006D626572206973206E6F74204C6173740A
:101F1000204C696E65204E756D6265722B312C20E8
:101F20004C617374204C696E653A20004D3131303C
:101F300000526573656E643A200020420020500014
:101F40006F6B00220A00656E7175657565696E6755
:101F5000202200504944204175746F74756E6520CD
:101F60006661696C656421204261642065787472E1
:101F700075646572206E756D6265720A006F6B0024
:101F80002020506C616E6E657242756666657242A5
:101F9000797465733A20002046726565204D656D41
:101FA0006F72793A2000436F6D70696C65643A20F6
:101FB0004D617220313820323031390A00207C20C6
:101FC000417574686F723A2028416C657068204FC3
:101FD000626A6563747320496E632E2C204C756CA5
:101FE0007A426F7420476974205265706F73697408
:101FF0006F7279290A0000204C6173742055706457
:10200000617465643A2000322E302E302E3130312A
:102010000A004D61726C696E0020536F66747761BF
:1020200072652052657365740A0020576174636895
:10203000646F672052657365740A002042726F777F
:102040006E206F75742052657365740A00204578A0
:102050007465726E616C2052657365740A00506F0E
:1020600077657255700A0073746172740A00507259
:10207000696E7465722068616C7465642E206B698A
:102080006C6C28292063616C6C6564210A004B49E3
:102090004C4C2063617573656420627920746F6FA6
:1020A000206D75636820696E61637469766520745C
:1020B000696D65202D2063757272656E7420636F83
:1020C0006D6D616E643A20004D3132310A47302027
:1020D0005A31300A4732382058302059300A4731B7
:1020E000320A4D31303920523136300A4D313137D4
:1020F0002050726F62696E67206265640070726F53
:1021000062655F7265776970650050726F62696EB3
:1021100067206661696C6564004D31313720426526
:1021200064206C6576656C696E67206661696C65B4
:10213000642E0A4730205A31300A47302045300A91
:102140004D3330302050323520533838300A4D333B
:102150003030205035302053300A4D33303020504D
:10216000323520533838300A4D3330302050353036
:102170002053300A4D333030205032352053383818
:10218000300A47342053310070726F62655F6661B8
:10219000696C65640050726F746563746564205087
:1021A000696E0A0025301D0C1E282924311C0B18CD
:1021B0004527232F1B0A174443222B1A4142043878
:1021C00003FF3604080606000100621A1730886B08
:1021D000C59111241FBECFEFD1E2DEBFCDBF00E01D
:1021E0000CBF13E0A0E0B2E0E2E8FEE601E00BBFC6
:1021F00002C007900D92A03AB107D9F72EE0A0EAED
:10220000B3E001C01D92AD3EB207E1F710E1C9EEA7
:10221000D0E100E006C021970109802FFE010E9455
:10222000D6AFC53ED10780E00807A9F766D40C9465
:102230003FB70C9400001F920F920FB60F9211241B
:102240002F933F938F939F93AF93BF938091A1035D
:102250009091A203A091A303B091A4033091A00395
:1022600023E0230F2D3720F40196A11DB11D05C0D9
:1022700026E8230F0296A11DB11D2093A003809391
:10228000A1039093A203A093A303B093A40380910E
:10229000A5039091A603A091A703B091A80301966E
:1022A000A11DB11D8093A5039093A603A093A7033E
:1022B000B093A803BF91AF919F918F913F912F91C0
:1022C0000F900FBE0F901F9018952FB7F894609144
:1022D000A1037091A2038091A3039091A4032FBF47
:1022E00008953FB7F8948091A5039091A603A0911B
:1022F000A703B091A80326B5A89B05C02F3F19F0EE
:102300000196A11DB11D3FBFBA2FA92F982F882775
:10231000820F911DA11DB11DBC01CD0142E0660FD0
:10232000771F881F991F4A95D1F708958F929F9222
:10233000AF92BF92CF92DF92EF92FF926B017C013E
:10234000D0DF4B015C01C114D104E104F104F1F0D0
:1023500091D3C7DFDC01CB0188199909AA09BB0910
:10236000883E9340A105B10570F321E0C21AD1085F
:10237000E108F10888EE880E83E0981EA11CB11CCC
:10238000C114D104E104F10421F7DDCFFF90EF90F7
:10239000DF90CF90BF90AF909F908F9008957894EA
:1023A00084B5826084BD84B5816084BD85B582605A
:1023B00085BD85B5816085BDEEE6F0E080818160F8
:1023C0008083E1E8F0E010828081826080838081F8
:1023D00081608083E0E8F0E0808181608083E1EBD0
:1023E000F0E0808184608083E0EBF0E080818160B8
:1023F0008083E1E9F0E08081826080838081816078
:102400008083E0E9F0E0808181608083E1EAF0E0B0
:10241000808182608083808181608083E0EAF0E057
:10242000808181608083E1E2F1E08081826080834D
:10243000808181608083E0E2F1E08081816080833F
:10244000EAE7F0E08081846080838081826080831D
:102450008081816080838081806880831092C10048
:1024600008951F93CF93DF93182FEB0161E016D1EE
:10247000209711F460E004C0CF3FD10531F461E052
:10248000812FDF91CF911F9145C1E12FF0E0ED51F8
:10249000FE4FE4914E2F50E0FA013197E231F10501
:1024A00008F09DC08827EE58FF4F8F4F0C94D6AF91
:1024B00084B5806884BDC7BD97C084B5806284BD83
:1024C000C8BD92C080918000806880938000D093C6
:1024D0008900C093880088C08091800080628093CA
:1024E0008000D0938B00C0938A007EC080918000D2
:1024F000886080938000D0938D00C0938C0074C05E
:102500008091B00080688093B000C093B3006CC02D
:102510008091B00080628093B000C093B40064C02A
:1025200080919000806880939000D0939900C09330
:1025300098005AC080919000806280939000D09360
:102540009B00C0939A0050C0809190008860809357
:102550009000D0939D00C0939C0046C08091A00045
:1025600080688093A0008091A0008F7B8093A00062
:10257000D093A900C093A80037C08091A0008062CA
:102580008093A000D093AB00C093AA002DC080918F
:10259000A00088608093A000D093AD00C093AC00F1
:1025A00023C080912001806880932001D09329016D
:1025B000C093280119C0809120018062809320017E
:1025C000D0932B01C0932A010FC080912001886015
:1025D00080932001D0932D01C0932C0105C0C038F9
:1025E000D1050CF04CCF46CFDF91CF911F910895CC
:1025F00090E0FC013197E231F10508F04EC08827E8
:10260000EC57FF4F8F4F0C94D6AF809180008F779F
:1026100003C0809180008F7D809380000895809119
:102620008000877FF9CF84B58F7702C084B58F7D16
:1026300084BD08958091B0008F7703C08091B00071
:102640008F7D8093B0000895809190008F7707C0B0
:10265000809190008F7D03C080919000877F809350
:10266000900008958091A0008F7707C08091A0000E
:102670008F7D03C08091A000877F8093A000089584
:10268000809120018F7707C0809120018F7D03C04A
:1026900080912001877F809320010895CF93DF935D
:1026A00090E0FC01E75DFD4F2491FC01E159FD4FF5
:1026B0008491882361F190E0880F991FFC01E75114
:1026C000FD4FC591D491FC01E153FD4FA591B4910B
:1026D000611109C09FB7F89488812095822388836F
:1026E000EC912E230BC0623061F49FB7F8943881CF
:1026F000822F809583238883EC912E2B2C939FBF70
:1027000006C08FB7F894E8812E2B28838FBFDF9106
:10271000CF9108951F93CF93DF93282F30E0F901D5
:10272000ED51FE4F8491F901E75DFD4FD491F90120
:10273000E159FD4FC491CC23C1F0162F811158DF10
:10274000EC2FF0E0EE0FFF1FE153FD4FA591B49188
:102750008FB7F894111105C09C91ED2FE095E923F6
:1027600002C0EC91ED2BEC938FBFDF91CF911F91C5
:102770000895CF93DF93282F30E0F901ED51FE4FFC
:102780008491F901E75DFD4FD491F901E159FD4FC5
:10279000C491CC2389F081112BDFEC2FF0E0EE0FF8
:1027A000FF1FEB54FD4FA591B491EC91ED2381E017
:1027B00090E021F480E002C080E090E0DF91CF91D2
:1027C000089508951F920F920FB60F9211240BB621
:1027D0000F922F933F934F935F936F937F938F93BA
:1027E0009F93AF93BF93EF93FF93E0910402F09117
:1027F00005021995FF91EF91BF91AF919F918F9134
:102800007F916F915F914F913F912F910F900BBEF0
:102810000F900FBE0F901F9018951F920F920FB63A
:102820000F9211240BB60F922F933F934F935F9308
:102830006F937F938F939F93AF93BF93EF93FF9388
:10284000E0910602F09107021995FF91EF91BF9177
:10285000AF919F918F917F916F915F914F913F9138
:102860002F910F900BBE0F900FBE0F901F901895D9
:102870001F920F920FB60F9211240BB60F922F9347
:102880003F934F935F936F937F938F939F93AF93F8
:10289000BF93EF93FF93E0910802F091090219951D
:1028A000FF91EF91BF91AF919F918F917F916F9128
:1028B0005F914F913F912F910F900BBE0F900FBEE4
:1028C0000F901F9018951F920F920FB60F92112420
:1028D0000BB60F922F933F934F935F936F937F931A
:1028E0008F939F93AF93BF93EF93FF93E0910A026F
:1028F000F0910B021995FF91EF91BF91AF919F91CC
:102900008F917F916F915F914F913F912F910F9098
:102910000BBE0F900FBE0F901F9018951F920F9235
:102920000FB60F9211240BB60F922F933F934F9334
:102930005F936F937F938F939F93AF93BF93EF9327
:10294000FF93E0910002F09101021995FF91EF9140
:10295000BF91AF919F918F917F916F915F914F91B7
:102960003F912F910F900BBE0F900FBE0F901F90B5
:1029700018951F920F920FB60F9211240BB60F925B
:102980002F933F934F935F936F937F938F939F9377
:10299000AF93BF93EF93FF93E0910202F091030294
:1029A0001995FF91EF91BF91AF919F918F917F9179
:1029B0006F915F914F913F912F910F900BBE0F90B0
:1029C0000FBE0F901F9018951F920F920FB60F9287
:1029D00011240BB60F922F933F934F935F936F93F6
:1029E0007F938F939F93AF93BF93EF93FF93E09168
:1029F0000C02F0910D021995FF91EF91BF91AF91EB
:102A00009F918F917F916F915F914F913F912F9106
:102A10000F900BBE0F900FBE0F901F9018951F9236
:102A20000F920FB60F9211240BB60F922F933F9374
:102A30004F935F936F937F938F939F93AF93BF93C6
:102A4000EF93FF93E0910E02F0910F021995FF9121
:102A5000EF91BF91AF919F918F917F916F915F9116
:102A60004F913F912F910F900BBE0F900FBE0F9083
:102A70001F90189508954F925F926F927F92AF9238
:102A8000BF92CF92DF92EF92FF920F931F93CF935B
:102A9000DF93CDB7DEB729013A019B01AC012419C0
:102AA0003509460957098A899B89AC89BD89BC01CA
:102AB000CD016A197B098C099D090E9475AFA80197
:102AC000970124193509460957090E94BAAFCA016E
:102AD000B9016A0D7B1D8C1D9D1DDF91CF911F914A
:102AE0000F91FF90EF90DF90CF90BF90AF907F90CD
:102AF0006F905F904F900895089551DCFDDF0E9424
:102B000008ABC0E0D0E00E9487AB2097E1F30E94C1
:102B10000000F9CFCF93C82F0E947930CC2349F021
:102B200024982C9A65E070E080E090E0FFDB149A36
:102B300003C0249A2C981498CF91089580E0EACF8E
:102B4000CF92DF92EF92FF926B017C0183E3C81674
:102B5000D104E104F10468F082E3C81AD108E10865
:102B6000F10862E370E080E090E0E0DB0E94C424C2
:102B7000EDCFC701B601DADBFF90EF90DF90CF9089
:102B80000C94C424DC01FB01460F571FE417F50722
:102B9000C1F081912D913C911197382798E0B901AE
:102BA000660F771F37FF06C09B0181E2282780E16F
:102BB000382701C09B01915091F711963C932E93B9
:102BC000E5CF0895CF93DF93FC018491EF01219627
:102BD000882319F087D2FE01F8CFDF91CF910895B5
:102BE0008AE093E0EFCF80E193E0ECCF0F931F9367
:102BF000CF93DF931F921F92CDB7DEB769837A839D
:102C0000E1DF6981062F7A81172FF80181918F0109
:102C1000882311F067D2F9CF0F900F90DF91CF91F9
:102C20001F910F910895CF93DF93EB01CBDF6AE003
:102C300070E0CE01DF91CF9148C3CF92DF92EF9247
:102C4000FF926A017B01BEDF4AE050E0C701B60196
:102C5000FF90EF90DF90CF9027C3CF92DF92EF925B
:102C6000FF926A017B01AEDF42E050E0C701B6018E
:102C7000FF90EF90DF90CF90B3C3CF92DF92EF92AF
:102C8000FF926A017B019EDF42E050E0C701B6017E
:102C9000FF90EF90DF90CF90A3C3CF93DF93EB0132
:102CA00091DF6AE070E0CE01DF91CF9123C3CF9234
:102CB000DF92EF92FF926A017B0184DF4AE050E0ED
:102CC000C701B601FF90EF90DF90CF900DC3811147
:102CD00003C083E093E002C087E093E073CFF7DFA7
:102CE0008AE000C2CF93DF931F921F92CDB7DEB769
:102CF0002091E70E3091E80ECE01019621153105A5
:102D000019F48D5E9E4002C0821B930B9A838983C7
:102D100089819A810F900F90DF91CF91089581E082
:102D2000089581E008958F929F92AF92BF92CF92C3
:102D3000DF92EF92FF920F931F93CF93DF931F9237
:102D40001F92CDB7DEB76C0159018B017B01E40EF8
:102D5000F51E0E151F0561F1F60180809180F801C6
:102D600061918F016983C4016A830E9429B76A81D6
:102D7000681779F0C4010E9431B7C4010E9429B7D5
:102D80009981891731F02CDF87E193E01BDF81E027
:102D900010C041E050E0BE016F5F7F4FC501F2DE21
:102DA000F601408151814F5F5F4F51834083D1CF06
:102DB00080E00F900F90DF91CF911F910F91FF90C6
:102DC000EF90DF90CF90BF90AF909F908F9008953D
:102DD0008F929F92AF92BF92CF92DF92EF92FF922B
:102DE0000F93CF93DF931F92CDB7DEB75C016B01DA
:102DF0007A014901F501808191810E9429B7898377
:102E0000002311F0F601808341E050E0BE016F5FC6
:102E10007F4FC401B7DEF501408151814F5F5F4FA5
:102E200051834083FFEFCF1ADF0A81E0E81AF108EF
:102E300009F780E00F90DF91CF910F91FF90EF9015
:102E4000DF90CF90BF90AF909F908F90089598E2C1
:102E500088E10FB6F894A895809360000FBE909318
:102E6000600008951F920F920FB60F9211240BB6B7
:102E70000F920F931F932F933F934F935F936F93F3
:102E80007F938F939F93AF93BF93CF93DF93EF93F2
:102E9000FF930091CF03D091CE0311E01D0F1F7758
:102EA000C091C6009091AA03492F092E000C550B22
:102EB000660B770B4C30510508F046C0FA018827A5
:102EC000EA56FF4F8F4F0C94D6AFCD3441F0CE343D
:102ED000B9F481E005C0CA3330F0CD3471F582E039
:102EE0008093AA034AC0C03308F047C0C03209F437
:102EF00044C0CD3211F541C0C13329F0C43329F0AB
:102F0000C032D9F43AC083E0EBCF88E0E9CFC033D8
:102F100021F0C13391F486E0E3CF84E0E1CFC83300
:102F200061F485E0DDCFC23341F487E0D9CFC1330E
:102F300021F489E0D5CFC03311F08BE0D1CF8AE006
:102F4000CFCFCA30D1F417C0CA30B9F48091590438
:102F5000882389F0973049F09A3059F0953059F428
:102F600010926F021092E60E06C081E080935A0420
:102F700002C00E94C2A91092AA03101731F0ED2FCF
:102F8000F0E0E253FC4FC283D12FD093CE03FF91E8
:102F9000EF91DF91CF91BF91AF919F918F917F91F1
:102FA0006F915F914F913F912F911F910F910F90D2
:102FB0000BBE0F900FBE0F901F9018951F920F928F
:102FC0000FB60F9211240BB60F922F938F939F93EE
:102FD000EF93FF938091AD032091AC03281791F0FC
:102FE000E82FF0E0E455FC4F92818F5F8F71909352
:102FF000C6008093AD039091C00090649093C00090
:10300000281305C08091C1008F7D8093C100FF917E
:10301000EF919F918F912F910F900BBE0F900FBE4C
:103020000F901F9018959B01AC011092C0002115C4
:1030300081EE380741055105C1F08091C0008260E2
:103040008093C00060E079E08DE390E00E94BAAF29
:10305000CA01B901615071098109910922E030E08A
:1030600040E050E00E94BAAF02C020E130E030936F
:10307000C5002093C4008091C10080618093C1008D
:103080008091C10088608093C1008091C1008068F8
:103090008093C1008091C1008F7D8093C100109208
:1030A000AB0308958091CE039091CF03891759F017
:1030B000E92FF0E0E253FC4F82819F5F9F7790936E
:1030C000CF0390E008958FEF9FEF0895EEECF3E0CB
:1030D000808181830895EEECF3E080819181891BEA
:1030E0008F77089591E09093AB039091C10095FD87
:1030F00004C09091C00095FD40C02091AC032F5FAB
:103100002F710FB607FC34C09091AD03291322C074
:103110009091C00095FF1DC09091AD034091AC030C
:10312000491791F0E92FF0E0E455FC4F32819F5FA1
:103130009F713093C6009093AD033091C00030640E
:103140003093C000491305C09091C1009F7D9093BA
:10315000C100DACFE091AC03F0E0E455FC4F82838C
:103160002093AC038091C10080628093C1000895D8
:103170009091AD032913EECFFBCF8093C6008091D1
:10318000C00080648093C00008958DE0ABDF8AE0CA
:10319000A9CFCF93DF93EC018991882311F0A2DFAF
:1031A000FBCFDF91CF91F1CF8F929F92AF92BF92E1
:1031B000EF92FF921F93CF93DF93CDB7DEB7A09727
:1031C0000FB6F894DEBF0FBECDBF61157105810546
:1031D000910579F110E0842E912CA12CB12CEE24D4
:1031E000E394F12CEC0EFD1EE10EF11C17FDFA9498
:1031F000A50194010E9498AFF7016083B901CA014B
:103200001F5F611571058105910549F7115010F196
:10321000E1E0F0E0EC0FFD1FE10FF11D17FDFA9565
:1032200080818A3010F097E301C090E3890F5ADF64
:10323000EDCF80E3A0960FB6F894DEBF0FBECDBFF2
:10324000DF91CF911F91FF90EF90BF90AF909F9033
:103250008F9048CFA0960FB6F894DEBF0FBECDBFBB
:10326000DF91CF911F91FF90EF90BF90AF909F9013
:103270008F900895CF92DF92EF92FF926B017C01C5
:1032800097FF0AC08DE22EDFF094E094D094C094B2
:10329000C11CD11CE11CF11C4AE0C701B601FF9022
:1032A000EF90DF90CF9080CF4115510511F4862F1C
:1032B00019CF4A30510509F4DDCF76CFAB01682F25
:1032C000880F770B880B990BEFCFAB01BC01990FDF
:1032D000880B990BE9CFAB01BC01990F880B990BB7
:1032E000E3DF53CFE1DF51CF4115510511F4862FB4
:1032F000F9CE5ACFAB01BC0180E090E0F5CF8F92C0
:103300009F92AF92BF92CF92DF92EF92FF92CF93B4
:103310006B017C01B42E20E030E0A9010E946DAC6D
:1033200087FF06C08DE2DEDEF7FAF094F7F8F0943E
:10333000C0E060E070E080E09FE3CB1541F02DEC51
:103340003CEC4CEC5DE30E94ABAECF5FF6CF9B0153
:10335000AC01C701B6010E9494AB6B017C010E94D5
:10336000E1AC4B015C014AE01FDFCC2379F1C501E0
:10337000B4010E940DAD9B01AC01C701B6010E94D2
:1033800093AB6B017C018EE2ADDE20E030E040E2E9
:1033900051E4C701B6010E94ABAE4B015C010E9433
:1033A000DCAC6B01770FEE08FF08C701B60162DFE6
:1033B000C701B6010E940FAD9B01AC01C501B4016C
:1033C0000E9493AB6B017C01C150F9F6CF91FF9045
:1033D000EF90DF90CF90BF90AF909F908F90089527
:1033E0008ECFCF92DF92EF92FF920F931F930E94A6
:1033F00065110091540410915504209156043091A8
:1034000057046B017C01C01AD10AE20AF30AF7FCE7
:1034100052C08B019C010C53164F2F4F3F4F00930E
:103420005404109355042093560430935704079B7B
:1034300039C0069B37C0059B35C02091B4042111CB
:1034400031C0049B2FC00091500410915104209171
:10345000520430915304011511052105310571F015
:10346000DC01CB01801B910BA20BB30B80569A4E53
:10347000A109B109B7FF02C068E701C060E060932D
:103480005804809102016111809588708093000139
:1034900070E086E01F910F91FF90EF90DF90CF904A
:1034A0000C94311260935004709351048093520431
:1034B00090935304C8CF1F910F91FF90EF90DF902E
:1034C000CF90089581E08093590408959091150656
:1034D0008917D1F00E949C5A80911506882359F0D3
:1034E00048E552E064E572E080E592E00E945F59B1
:1034F0001092150607C081E08093150680E592E0E2
:103500000E94CD590C94BE4E089580E0DFDF81EF1C
:1035100095E00C942DA50F931F93CF93DF931F92EB
:10352000CDB7DEB78C0181E493E069834BDBC80142
:1035300049DB6981662339F08AE00F90DF91CF91F2
:103540001F910F91CFCD0F90DF91CF911F910F91D0
:10355000089561E088E393E0DECF61E081E393E0EA
:10356000DACFEF92FF920F931F93CF93DF931F92C7
:10357000CDB7DEB78C017B0180E24983B3DD4981A1
:103580004F3F11F084E501C082E4ACDD8AE3AADD9F
:10359000F801608171818281938142E050E020DFF7
:1035A000F701408151816281738183E593E055DBAE
:1035B00062E070E080E090E00F90DF91CF911F918A
:1035C0000F91FF90EF900C949611FB01DC01129685
:1035D0004D915D916D917C91159741155105610556
:1035E000710599F080819181A281B381841B950B33
:1035F000A60BB70B80959095A095B0958827B7FD41
:1036000083959927AA27BB27089580E00895811103
:1036100009C0CB016F3F710519F010F08FEF90E0FA
:103620008093C704089597FF03C08091B40409C034
:1036300027E1289FF001299FF00D1124E853FB4F4B
:10364000828590E008954F925F926F927F928F9261
:103650009F92AF92BF92CF92DF92EF92FF92CF9361
:10366000DF9300D01F92CDB7DEB7E090D004F0908A
:10367000D1048090CC049090CD04A090CE04B09062
:10368000CF0420ED3CEC4CE45DE36091DB047091F1
:10369000DC048091DD049091DE040E94ABAE2B012E
:1036A0003C0120918C0430918D0440918E04509106
:1036B0008F04C501B4010E9493AB9B01AC01C3010F
:1036C000B2010E94ABAE2B013C0123E333E343E79D
:1036D0005FE3609188047091890480918A049091DD
:1036E0008B040E94ABAE9B01AC01C301B2010E94EE
:1036F00094AB69837A838B839C83609388047093F3
:10370000890480938A0490938B0480928C04909215
:103710008D04A0928E04B0928F04E114F104A1F004
:10372000B701FF0C880B990B0E940FADA501940106
:103730000E9493AB6B017C0120E030E040E251EC51
:103740000E946DAC87FF07C081E080937F04412C0D
:10375000512C3201C1C020E030E040E251E4C70109
:10376000B6010E9470AE181654F481E080937F0475
:10377000412C512C2FE7622E23E4722EADC0809194
:103780007F04882351F010927B0410927C041092E5
:103790007D0410927E0410927F0420917B0430916E
:1037A0007C0440917D0450917E04C701B6010E94C3
:1037B00094AB4B015C0160937B0470937C04809319
:1037C0007D0490937E042091D3043091D4044091E1
:1037D000D5045091D604C701B6010E94ABAE2B01AF
:1037E0003C016093800470938104809382049093E1
:1037F00083042091D7043091D8044091D90450918A
:10380000DA04C501B4010E94ABAE9B01AC01609328
:103810008404709385048093860490938704C30185
:10382000B2010E9494AB29813A814B815C810E9454
:1038300093AB2B013C0120E030E04FE753E40E94C2
:1038400070AE20E030E0A9011816DCF4C701B60123
:103850000E9470AE1816B4F5A7019601C501B40117
:103860000E9493AB60937B0470937C0480937D04EF
:1038700090937E04412C512C9FE7692E93E4792E7E
:103880002BC0C301B2010E946DAC87FF25C020E0B0
:1038900030E0A901C701B6010E946DAC87FF19C0D5
:1038A000A7019601C501B4010E9493AB60937B040C
:1038B00070937C0480937D0490937E04412C512C62
:1038C00032010AC0412C512C8FE7682E83E4782EF8
:1038D00003C0412C512C3201C301B2010F900F9053
:1038E0000F900F90DF91CF91FF90EF90DF90CF90EE
:1038F000BF90AF909F908F907F906F905F904F9010
:1039000008954F925F926F927F928F929F92AF92A3
:10391000BF92CF92DF92EF92FF92CF93DF93CDB71A
:10392000DEB72C970FB6F894DEBF0FBECDBF8091E7
:10393000AE049091AF04A091B004B091B10489831A
:103940009A83AB83BC836091B2047091B304072E59
:10395000000C880B990B0E940FAD29813A814B8195
:103960005C810E9493AB6B017C01209177043091C4
:1039700078044091790450917A040E9494AB4B01F1
:103980005C0160937704709378048093790490933A
:103990007A042091B5043091B6044091B704509157
:1039A000B804C701B6010E94ABAE6D837E838F83DE
:1039B000988760936B0470936C0480936D0490936C
:1039C0006E042091B9043091BA044091BB04509127
:1039D000BC04C501B4010E94ABAE69877A878B87AE
:1039E0009C8760936F04709370048093710490932C
:1039F000720420ED3CEC4CE45DE36091BD047091F9
:103A0000BE048091BF049091C0040E94ABAE2B0114
:103A10003C01209167043091680440916904509101
:103A20006A0469817A818B819C810E9493AB9B019E
:103A3000AC01C301B2010E94ABAE2B013C0123E3F8
:103A400033E343E75FE36091730470917404809102
:103A50007504909176040E94ABAE9B01AC01C3014A
:103A6000B2010E9494AB2B013C01609373047093EC
:103A70007404809375049093760489819A81AB8154
:103A8000BC818093670490936804A0936904B09309
:103A90006A0429853A854B855C856D817E818F819D
:103AA00098850E9494ABA30192010E9493AB2B01D5
:103AB0003C0120E030E04FE753E40E9470AE20E08C
:103AC00030E0A9011816DCF4C701B6010E9470AEFF
:103AD0001816B4F5A7019601C501B4010E9493AB75
:103AE00060937704709378048093790490937A04B8
:103AF000412C512C9FE7692E93E4792E2BC0C301F2
:103B0000B2010E946DAC87FF25C020E030E0A90122
:103B1000C701B6010E946DAC87FF19C0A7019601CD
:103B2000C501B4010E9493AB60937704709378044D
:103B30008093790490937A04412C512C32010AC06D
:103B4000412C512C8FE7682E83E4782E03C0412C42
:103B5000512C3201C301B2012C960FB6F894DEBF8E
:103B60000FBECDBFDF91CF91FF90EF90DF90CF9050
:103B7000BF90AF909F908F907F906F905F904F908D
:103B800008954F925F926F927F928F929F92AF9221
:103B9000BF92CF92DF92EF92FF920F931F93CF933A
:103BA000DF933C01C62F662389F01DD86AE070E0E0
:103BB0008C2F90E08ADB86E893E004D880E090E0E8
:103BC0000E9407AA60E070E0CB017AC0B0E2A0E0FA
:103BD0006A2F70E0AB014B0F511D559547954A1761
:103BE00011F04B130BC0E8E4F7E065917491072ED8
:103BF000000C880B990B0E940FAD62C0CA0101979F
:103C0000880F991F880F991FFC01E653F94F059102
:103C100014919A01220F331F220F331FF901E6532B
:103C2000F94FC591D4916016710614F4B42FD2CF18
:103C3000A42FC615D7050CF4CBCF8453994FFC01A4
:103C4000E590F490F901E453F94FC590D490B70191
:103C50000F2C000C880B990B0E940FAD4B015C01DF
:103C6000B301601B710B072E000C880B990B0E948F
:103C70000FAD2B013C01B6016E197F09072E000C18
:103C8000880B990B0E940FAD9B01AC01C301B201DF
:103C90000E94ABAE6B017C01C01BD10BBE01DD0FDE
:103CA000880B990B0E940FAD9B01AC01C701B601B7
:103CB0000E9474AC9B01AC01C501B4010E9494AB9D
:103CC000DF91CF911F910F91FF90EF90DF90CF90F8
:103CD000BF90AF909F908F907F906F905F904F902C
:103CE00008954F925F926F927F928F929F92AF92C0
:103CF000BF92CF92DF92EF92FF920F931F93CF93D9
:103D0000DF933C01BAE3A0E06A2F70E0AB014B0FF8
:103D1000511D559547954A1711F04B130BC0E8EC10
:103D2000F6E065917491072E000C880B990B0E94A8
:103D30000FAD62C0CA010197880F991F880F991FA4
:103D4000FC01EE51FA4F059114919A01220F331F95
:103D5000220F331FF901EE51FA4FC591D49160162D
:103D6000710614F4B42FD2CFA42FC615D7050CF4C6
:103D7000CBCF8C519A4FFC01E590F490F901EC51B6
:103D8000FA4FC590D490B7010F2C000C880B990BFB
:103D90000E940FAD4B015C01B301601B710B072E3C
:103DA000000C880B990B0E940FAD2B013C01B60152
:103DB0006E197F09072E000C880B990B0E940FAD1E
:103DC0009B01AC01C301B2010E94ABAE6B017C014F
:103DD000C01BD10BBE01DD0F880B990B0E940FADEC
:103DE0009B01AC01C701B6010E9474AC9B01AC0100
:103DF000C501B4010E9494ABDF91CF911F910F9147
:103E0000FF90EF90DF90CF90BF90AF909F908F90FA
:103E10007F906F905F904F900895CF93DF93C8ECA1
:103E2000D4E060E08A819B81ACDE6C837D838E83ED
:103E30009F83CAEAD4E08A819B8153DF6C837D83B0
:103E40008E839F83A8951092A004DF91CF9108954F
:103E5000CF93DF93CDB7DEB760970FB6F894DEBF90
:103E60000FBECDBF9C01E62F660FFF0BED51FE4F3D
:103E7000E4918E2F90E0FC013797EC30F10508F0CB
:103E8000BFC08827EE55FF4F8F4F0C94D6AF91E0FF
:103E900001C090E080E1FE013196DF01482F1D92C4
:103EA0004A95E9F740EB50E05A83498341EB50E0F3
:103EB0005C834B8343EB50E058874F8344EB50E0E7
:103EC0005A87498742E04F87988BD90101900D921C
:103ED0008A95E1F7A2C081E001C080E08F5F01C058
:103EE00080E040E950E0D90111965C934E9341E99E
:103EF00050E013965C934E93129742E950E015966A
:103F00005C934E93149748E950E017965C934E9358
:103F100016974AE950E019965C934E9318974CE92E
:103F200050E01B965C934E931A9746E950E01D961D
:103F30005C934E931C9793E01E969C931E971F963E
:103F40008C936BC081E001C080E08F5F01C080E096
:103F500040EA50E0F9015183408341EA50E0538345
:103F6000428342EA50E05583448348EA50E0578355
:103F700046834AEA50E0518740874CEA50E0538735
:103F8000428746EA50E05587448794E096878787C2
:103F900044C081E001C080E08F5F01C080E040E26A
:103FA00051E0D90111965C934E9341E251E0139692
:103FB0005C934E93129742E251E015965C934E93B8
:103FC000149748E251E017965C934E9316974AE295
:103FD00051E019965C934E9318974CE251E01B9672
:103FE0005C934E931A9746E251E01D965C934E9374
:103FF0001C9795E01E969C931E971F968C930DC060
:1040000080E1FE013196DF01482F1D924A95E9F7C4
:10401000D90101900D928A95E1F7C90160960FB61A
:10402000F894DEBF0FBECDBFDF91CF9108952F92E0
:104030003F924F925F926F927F928F929F92AF9238
:10404000BF92CF92DF92EF92FF920F931F93CF9385
:10405000DF93CDB7DEB7AE970FB6F894DEBF0FBED5
:10406000CDBF7CA36BA3682FCE014196F1DE2B89D7
:104070003C893EA32DA33F8D3AA3332309F429C1E4
:10408000323021F0EE24EA94FE2C03C0EE24EA94B0
:10409000F12C4BA15CA1452B09F4E0C09701322F14
:1040A0002227330F330F330F40E050E060E074E21B
:1040B00084EF90E00E94BAAF59018FEFA81AB80AB6
:1040C00080E1E1E7F2E0DE01119601900D928A9520
:1040D000E1F7FE013196F8A7EFA301E011E019A284
:1040E00088248A94912C412C94E2592E94EF692EC5
:1040F000712CFAA1F23059F1033009F4A4C0053053
:1041000009F4A1C0EFA1F8A5828193812BA13CA164
:10411000289F6001299FD00C389FD00C1124960154
:1041200040E050E0C301B2010E94BAAF190181E042
:10413000281A31089601220F331F40E050E0C301D6
:10414000B2010E94BAAF2114310431F40AC02FEF3A
:1041500030E022242A94312CE214F30428F41701CD
:1041600003C022242394312C2115310531F069013B
:10417000E216F30628F4670103C0CC24C394D12CC3
:10418000EFA1F8A50280F381E02DFEA7EDA7C10104
:1041900001968E9F90018F9F300D9E9F300D1124B0
:1041A00040E050E0C301B2010E94BAAF29A73AA78C
:1041B0004BA75CA78DA59EA5880F991F8C9D90018C
:1041C0008D9D300D9C9D300D112440E050E0C301C9
:1041D000B2010E94BAAF69A57AA58BA19CA1681B08
:1041E000790B77FF03C0719561957109D501EBA13A
:1041F000FCA1AE1BBF0BB7FF03C0B195A195B109E0
:10420000C901EBA1FCA18E1B9F0B6A177B075CF415
:10421000FC0197FF04C0EE27FF27E81BF90BE61708
:10422000F7070CF049C097FF03C09195819591095C
:104230008A179B0744F4FAA1590109A34601F230F9
:1042400009F045C011E00F5F2FA138A52E5F3F4F49
:1042500038A72FA3083009F04CCF05C011E019A2F0
:1042600088248A94912CE989FA898081912F93700E
:104270008C7F892B8083EDA1FEA12081812F90E08E
:10428000959587959595879543E0880F991F4A9551
:10429000E1F7122F177E812B8083808199A197707F
:1042A000887FF92EF82AF082FAA1F23091F0ED8D94
:1042B000FE8D918280820DC02AA1A9A4BAA409A36F
:1042C0004101223011F01EE0BECF13E0BCCF1AE056
:1042D000BACFAE960FB6F894DEBF0FBECDBFDF915A
:1042E000CF911F910F91FF90EF90DF90CF90BF90F3
:1042F000AF909F908F907F906F905F904F903F9086
:104300002F9008956D9A7598809101018061809336
:10431000010180910201807180930001809101016F
:104320008860809301018091020188708093000170
:104330009D9AA598809101018062809301016AE7AE
:1043400070E088E074DE8091010188608093010153
:104350006AE770E086E06BDE87ED80937A0010926A
:104360007E0010927D0080917E00816080937E00AF
:1043700080917E00846080937E0080E888BD80917B
:104380006E00846080936E006AEF70E080E090E0E1
:104390000E94961185E090E090931A028093190292
:1043A00060E08091150290911602EBDB20E030E096
:1043B00040EA50E40E946DAC87FF0AC0809115026C
:1043C0009091160240979093160280931502E8CFC1
:1043D00081E391E090931C0280931B0260E0809146
:1043E000150290911602CDDB20E030E848E953E455
:1043F0000E9470AE181654F4809117029091180222
:1044000040969093180280931702E8CF80911F0284
:104410009091200266DC20E030E040EA50E40E9407
:104420006DAC87FF0AC080911F02909120024097D7
:104430009093200280931F02E9CF8091A80490916D
:10444000A9044FDC20E030E046E153E40E9470AE66
:10445000181654F480911F02909120024096909378
:10446000200280931F02E9CF08954F925F926F92CE
:104470007F92AF92BF92CF92DF92EF92FF920F9313
:104480001F93CF93DF93CDB7DEB760970FB6F89445
:10449000DEBF0FBECDBF6115710511F4622F05C0DF
:1044A00064177507C1F461E0622760960FB6F8944F
:1044B000DEBF0FBECDBFDF91CF911F910F91FF9057
:1044C000EF90DF90CF90BF90AF907F906F905F9014
:1044D0004F900C948A13D22E8A017B01682FCE0153
:1044E0000196B6DC5F85E889552309F44BC0A981A4
:1044F000BA814C91F0E083E090E0BC016E1B7F0B31
:10450000660F771F2D2D30E02E5F3F4F062E01C026
:10451000220F0A94EAF701C0880F6A95EAF780959E
:104520008423282B2C93523029F0AD85BE85CD9065
:10453000DC9003C0CC24CA94D12C3396EE0FFF1F1D
:1045400081E090E08C0F9D1FE80FF91FA080B180E3
:10455000B70180E090E00E940DAD2B013C01C60147
:10456000B8010E9484AF80E090E00E940DAD9B01F5
:10457000AC01C301B2010E94ABAE0E94DCACF501FC
:104580007183608360960FB6F894DEBF0FBECDBF17
:10459000DF91CF911F910F91FF90EF90DF90CF901F
:1045A000BF90AF907F906F905F904F900895CF92A3
:1045B000DF92EF92FF928091D0049091D104009706
:1045C000B9F0C090CC04D090CD04E090CE04F0902F
:1045D000CF040D97BC01990F880B990B0E940FAD6A
:1045E0009B01AC01C701B6010E946DAC87FD09C0FB
:1045F0001092C3041092C4041092C5041092C60411
:104600001EC020E030E040E050E4C701B6010E9447
:1046100094AB0E94E1AC7093C2046093C1040E9409
:104620006511DC01CB01805E914BAF4FBF4F809392
:10463000C3049093C404A093C504B093C604FF9030
:10464000EF90DF90CF900895CF92DF92EF92FF929C
:104650008091B2049091B3040097B9F0C090AE0479
:10466000D090AF04E090B004F090B1040897BC0182
:10467000990F880B990B0E940FAD9B01AC01C701EC
:10468000B6010E946DAC87FD09C01092A40410927F
:10469000A5041092A6041092A7041EC020E030E0EA
:1046A00040E050E4C701B6010E9494AB0E94E1AC27
:1046B0007093A3046093A2040E946511DC01CB01F6
:1046C000805A9541AF4FBF4F8093A4049093A504A7
:1046D000A093A604B093A704FF90EF90DF90CF9033
:1046E000089580911B0290911C020F9718161906CD
:1046F00014F480E090E09093D1048093D00480E0A3
:1047000056DF1092B3041092B2049EDF80911B0218
:1047100090911C020F971816190614F480E090E08F
:104720009093D1048093D00480E041DF1092D204B2
:1047300075981092B3041092B2041092B404A59824
:104740000895EF92FF920F931F93CF93C82F7B0191
:104750008A01809170028823D1F00E94F315C7016D
:104760000E94E21588E294E00E94E215C7FD08C0AD
:104770006AE070E08C2FCC0F990B0E94651904C081
:1047800084E294E00E94E2158AE00E94721880910F
:10479000900481110DC01092700281E0809390040A
:1047A000C801CF911F910F91FF90EF900C9407AA31
:1047B000CF911F910F91FF90EF9093CF8F3F19F002
:1047C00040E154E002C040E254E06EEF73E0B9CF44
:1047D0008F3F19F04AEE53E002C04AEF53E068ED14
:1047E00073E0AFCF2F923F924F925F926F927F9282
:1047F0008F929F92BF92CF92DF92EF92FF920F9390
:104800001F93CF93DF936C014B01B22E180127FD4C
:1048100004C0C22F220FDD0B02C0C1E0D0E0FA01BC
:104820004080518062807380CC0FDD1FCC0FDD1F74
:104830008E01015A1B4FA3019201F8016081718121
:10484000828193810E946DAC882391F0F8014082AF
:1048500051826282738211E020E030E0A901C3013D
:10486000B2010E9470AE18160CF010E0F60114832D
:10487000F60184818230C9F0833009F456C081305A
:1048800009F070C0FE01E15AFB4F20813181428165
:104890005381F40160817181828193810E946DACAA
:1048A00087FD60C082E0F6018483C15ADB4FB70107
:1048B00080E090E00E940DAD9B01AC0168817981A0
:1048C0008A819B810E9493AB9B01AC01F4016081C2
:1048D0007181828193810E9470AE87FD15C00E9414
:1048E00065112B013C019101A8EEB3E00E94DEAFFF
:1048F000DC01CB01840D951DA61DB71DF60180833B
:104900009183A283B3832EC00E946511F6010081BA
:10491000118122813381DC01CB01801B910BA20B21
:10492000B30BB7FD1FC083E08483FFEFBF1619F000
:104930004FE653E002C042E853E06FE573E08B2D91
:10494000DF91CF911F910F91FF90EF90DF90CF906B
:10495000BF909F908F907F906F905F904F903F900F
:104960002F90EFCEDF91CF911F910F91FF90EF909D
:10497000DF90CF90BF909F908F907F906F905F90CF
:104980004F903F902F900895CF92DF92EF92FF9239
:104990000F931F93CF93DF93CDB7DEB728970FB652
:1049A000F894DEBF0FBECDBF80915A04811113C0B1
:1049B0008091A004811114C028960FB6F894DEBF30
:1049C0000FBECDBFDF91CF911F910F91FF90EF9060
:1049D000DF90CF90089580E090E00E9407AAE8CF92
:1049E0001CDA0E9465116D837E838F839887809186
:1049F000130290911402181619060CF0F3C00197D7
:104A000090931402809313026091D0047091D104AA
:104A1000072E000C880B990B0E940FAD69837A83D7
:104A20008B839C833EE1E32EF12C0FE010E020E02D
:104A3000AE014F5F5F4F6CEC74E08BE994E0D2DE27
:104A4000C090CC04D090CD04E090CE04F090CF0480
:104A50008091190290911A02BC01990F880B990B51
:104A60000E940FAD9B01AC01C701B6010E9470AE60
:104A70001816D4F460911B0270911C02072E000CD2
:104A8000880B990B0E940FAD9B01AC01C701B601C9
:104A90000E946DAC87FF08C080E00E94231B0E942B
:104AA000DCAC7595679501C060E06093D20480919D
:104AB000C3049091C404A091C504B091C6040097AA
:104AC000A105B10541F14D815E816F8178858A0133
:104AD0009B01081B190B2A0B3B0B37FD1CC0609177
:104AE000C1047091C20480E090E00E940DAD9B0172
:104AF000AC016091CC047091CD048091CE04909172
:104B0000CF040E946DAC87FF8EC046EC53E067EB8C
:104B100073E080E016DEBE016B5F7F4F82EA94E0B7
:104B20000E94E51A8823D9F06091A2047091A30431
:104B300080E090E00E940DAD2091AE043091AF0472
:104B40004091B0045091B1040E9470AE18160CF060
:104B500068C043EB53E064EA73E08FEFF2DD6091ED
:104B6000B2047091B304072E000C880B990B0E94BD
:104B70000FAD69837A838B839C839AE0E92EF12CB5
:104B80000FE010E02FEFAE014F5F5F4F6EEA74E071
:104B900086E994E027DEC090AE04D090AF04E090A8
:104BA000B004F090B10420E030E040EA50E4C701E6
:104BB000B6010E9470AE87FD0AC020E030E046E1F9
:104BC00053E4C701B6010E946DAC181624F460E0EE
:104BD0006093B404F1CE0E94811C0E94DCAC7595F8
:104BE0006795F6CFC090CC04D090CD04E090CE0471
:104BF000F090CF0420E030E848E953E4C701B60163
:104C00000E9470AE181694F020E030E040EA50E4C4
:104C1000C701B6010E946DAC87FFF6CE80E0D8DDFB
:104C2000F3CE12DD9CCF80E0C2DC75CF80E0C6DD24
:104C3000C090CC04D090CD04E090CE04F090CF048E
:104C4000E3CFE8ECF4E08081918193838283EAEA08
:104C5000F4E0808191819383828381E08093A0043A
:104C600008951F93CF93DF938091A004811101C019
:104C7000E8DF1092C9041092C8041092AB0410929D
:104C8000AA04C091CA04D091CB04D195C195D10991
:104C90008091D0049091D10411E0181619062CF0DF
:104CA0008091D204811101C010E08091170290918F
:104CB00018029195819591098C179D0714F480E055
:104CC0007DDD112361F0809115029091160291957E
:104CD00081959109C817D90714F480E079DD809196
:104CE000B2049091B304C1E0181619062CF080911B
:104CF000B404811101C0C0E02091AC043091AD0436
:104D00008091A8049091A9048217930714F08FEF63
:104D100055DDCC2381F020911F023091200280913B
:104D2000AC049091AD04821793072CF08FEFDF91C4
:104D3000CF911F914DCDDF91CF911F9108950F938A
:104D40000FB70F9300916E000B7F00936E00789465
:104D50000F930BB70F930CB70F921F922F933F93A4
:104D60004F935F936F937F938F939F93AF93BF9373
:104D7000EF93FF931124C7D0FF91EF91BF91AF91B3
:104D80009F918F917F916F915F914F913F912F9163
:104D90001F900F900CBF0F910BBF0F910460F89400
:104DA00000936E000F910FBF0F911895CF938091D4
:104DB00012028F3790F08F579091D20490935E0437
:104DC000992311F0759A01C075989091B40490934D
:104DD0005D04992359F0A59A0AC090915E04891741
:104DE00008F0759890915D04891708F0A598805F88
:104DF0008093120290915C0481E0892780935C0487
:104E00008091110285301CF4C1E0C80F01C0C0E0E0
:104E10008230A1F184F4882329F1813009F062C045
:104E200010927B0080E480937C0080917A00806403
:104E300080937A0057C0843009F43EC094F18530E5
:104E400009F050C090915B04911102C080935B0403
:104E500080915B04815080935B04882309F442C0F5
:104E6000C5E040C0809110028F5F80311CF48093B8
:104E7000100238C010921002F4DE34C080917A0023
:104E800086FD2DC080917800909179002091C80412
:104E90003091C904820F931F9093C9048093C80472
:104EA00021C010927B0082E480937C0080917A0084
:104EB000806480937A0016C080917A0086FD11C0CC
:104EC00080917800909179002091AA043091AB04F0
:104ED000820F931F9093AB048093AA0403C0C2E097
:104EE00001C0C4E0C09311020E94C43180918F06BA
:104EF00090919006009729F00197909390068093E7
:104F00008F06CF91089552CFFF920F931F93CF93A7
:104F1000DF93CDB7DEB728970FB6F894DEBF0FBE8C
:104F2000CDBFF82E08EC14E0F80160857185072EDE
:104F3000000C880B990B0E940FAD69837A838B83D9
:104F40009C83F80184819581A681B7818D839E839E
:104F5000AF83B8874DEFBE016F5F7F4FCE010596DF
:104F60000E94B11A0AEA14E0F80160857185072EE3
:104F7000000C880B990B0E940FAD69837A838B8399
:104F80009C83F80184819581A681B7818D839E835E
:104F9000AF83B8874FEFBE016F5F7F4FCE0105969D
:104FA0000E94B11A8BE593E00E94E2158F2D90E0EC
:104FB0000E94131B6AE070E00E94651986E593E089
:104FC0000E94E215F80182856AE070E090E00E949C
:104FD000651928960FB6F894DEBF0FBECDBFDF91DE
:104FE000CF911F910F91FF9008952F923F924F9272
:104FF0005F926F927F928F929F92AF92BF92CF9269
:10500000DF92EF92FF920F931F93CF93DF93CDB771
:10501000DEB7CD54D1090FB6F894DEBF0FBECDBFB9
:105020002E969FAF8EAF2E97162F742E26962FAFEB
:1050300026970E946511688B798B8A8B9B8B17FD55
:1050400004C0A4E1EA2EF12C03C0FCE3EF2EF12C06
:105050002E96AEADBFAD2E972D913D914D915C91A9
:105060002FA738AB49AB5AAB17FD90C4C12E012E08
:10507000000CDD08F60183E0EE0FFF1F8A95E1F7D3
:10508000EB5EFD4F668177816F507109072E000C32
:10509000880B990B0E940FAD9B01AC016FA578A9FD
:1050A00089A99AA90E9470AE1816ECF487EB95E0D6
:1050B000C35BDF4F0FB6F894DEBF0FBECDBFDF91ED
:1050C000CF911F910F91FF90EF90DF90CF90BF9005
:1050D000AF909F908F907F906F905F904F903F9098
:1050E0002F900C94E21583EA95E00E94E215F9DA1C
:1050F00027E12C9DC0012D9D900D1124FC01E8534A
:10510000FB4F2FE7228780E090E0A0E5B1E42396F3
:105110008CAF9DAFAEAFBFAF23979701A8EEB3E0C2
:105120000E94DEAF6BAF7CAF8DAF9EAF9B01AC0139
:1051300088899989AA89BB89280F391F4A1F5B1F53
:105140002BAB3CAB4DAB5EAB81E080936F028888AC
:105150009988AA88BB888EA29FA2A8A6B9A6188EF5
:10516000198E1A8E1B8E1C8A1D8A1E8A1F8A1A820D
:105170001B821C821D821A8690E49C8FACE1AD8F4D
:10518000B6E4BE8F1F8E18A219A21AA21EA61FAACD
:1051900018AE19AE1AAE2FE730E040E050E02E8393
:1051A0003F8348875987EFE7CE2ED12CE12CF12C95
:1051B0001AA61BA61CA61DA631E03BA31F861E86B1
:1051C000212C312C00E0198247E11402C001112486
:1051D00088539B4FDC011A962596BFAFAEAF25973B
:1051E000FC013496FDA3ECA3272D770C330B2896F6
:1051F0003FAF2EAF289780916F02882309F48FC2AA
:105200000E9465112B013C018091A004882309F4C0
:10521000FAC00E940D1F17FF0AC02090AE04309004
:10522000AF040091B0043091B10439830CC0ACA13B
:10523000BDA12C9011963C90119712960C9112974B
:105240001396BC91B9839101402F59816F8D78A13C
:1052500089A19AA10E946DAC87FF05C02F8E38A24C
:1052600009A3E981EAA39101402F59816A857C8DC8
:105270008D8D9E8D0E9470AE18162CF42A863C8E61
:105280000D8FF981FE8F2BA1222309F463C02E9686
:10529000AEADBFAD2E972D913D914D915C91B10179
:1052A000802F99810E9470AE18160CF0ACC0A3013B
:1052B0009201281939094A095B092C962CAF3DAF98
:1052C0004EAF5FAF2C97DA01C90188589341A1090D
:1052D000B109B7FD98C0D701C6012E813F8148852D
:1052E0005985821B930BA40BB50BB595A795979584
:1052F000879517FF03C08093B40405C02596EEADD3
:10530000FFAD259780832C962CAD3DAD4EAD5FADA6
:105310002C972AA73BA74CA75DA72E96AEADBFAD95
:105320002E97BC91BF8F2E96EEADFFAD2E97F181DB
:10533000F8A32E96AEADBFAD2E971296BC91B9A331
:105340002E96EEADFFAD2E97F381FAA34EA25FA28B
:1053500068A679A62E96AEADBFAD2E972D913D9144
:105360004D915C91B101802F99810E946DAC87FFB6
:105370000BC3D301C2012EA13FA148A559A5821B91
:10538000930BA40BB50BAC01BD0148585341610907
:10539000710977FDF9C24E855F85452B09F0DAC1A9
:1053A0008E819F81A885B9858C0D9D1DAE1DBF1D69
:1053B000B595A7959795879517FFE0C28093B4049C
:1053C0002E853F852F5F3F4F3F872E872E96AEADB0
:1053D000BFAD2E97BC91BA872E96EEADFFAD2E973E
:1053E000F181FC8F2E96AEADBFAD2E971296BC917B
:1053F000BD8F2E96EEADFFAD2E97F381FE8F53013C
:10540000420121E02BA320E030E040EA51E42E9657
:10541000AEADBFAD2E976D917D918D919C910E9407
:1054200094AB9B01AC01B101802F99810E9470AEB9
:1054300018162CF48FE295E00E94E21570C1D3019A
:10544000C201288939894A895B89821B930BA40B85
:10545000B50BB7FD8BC0812F17FD80E055DD8AE0CD
:105460000E947218D301C2018053984FAF4FBF4FB3
:10547000888B998BAA8BBB8B9EA5911155C02FA9A8
:1054800038AD49AD5AADB101802F99810E9470AEFF
:10549000181694F520E030E040E050E4B101802F90
:1054A00099810E9494AB6FAB78AF89AF9AAF2BAD67
:1054B0003CAD4DAD5EAD240D351D461D571D2BABCE
:1054C0003CAB4DAB5EAB23962CAD3DAD4EAD5FAD71
:1054D00023976FA578A989A99AA90E9493AB9B01EC
:1054E000AC0181E08EA7B101802F99810E9470AE3E
:1054F0001816E4F11EA63AC0D301C2012BA93CA99B
:105500004DA95EA9821B930BA40BB50BB7FD2EC052
:105510001F3F19F049E155E002C04BE255E06AE057
:1055200075E0812F0ED922C020E030E040EA51E43E
:105530002E96AEADBFAD2E976D917D918D919C91C4
:105540000E9493AB9B01AC01B101802F99810E9415
:105550006DAC87FF0BC01F3F19F043EF54E002C052
:1055600046E055E063EE74E0812FEBD8D301C20131
:10557000880F991FAA1FBB1F2EA13FA148A559A59F
:10558000821B930BA40BB50B88199909AA09BB09B7
:1055900081389F44A241B10528F085EC94E00E9437
:1055A000E215BDC04E855F8528968EAD9FAD2897CC
:1055B000841795070CF01FCE433051050CF41BCE19
:1055C00088E694E00E94E21517FD05C023E6E22E6E
:1055D00024E0F22E04C094E6E92E94E0F92E86E44D
:1055E00094E00E94E215C7010E94E2154A815B81A6
:1055F0006C817D818FE594E00E942D168AE00E94E7
:10560000721886E494E00E94E215C7010E94E21538
:105610004C895D896E897F898BE594E00E942D1607
:105620008AE00E94721886E494E00E94E215C701A5
:105630000E94E215488D598D6A8D7B8D87E594E037
:105640000E942D168AE00E94721826969FAD26971A
:10565000992309F4BCC117FF31C02A813B814C81D9
:105660005D812093B5043093B6044093B704509302
:10567000B8042CEA35EC47E25EE36C897D898E89BB
:105680009F890E94ABAE6093B9047093BA04809373
:10569000BB049093BC042CEA35EC47E25EE3688DD2
:1056A000798D8A8D9B8D0E9474AC6093BD0470933C
:1056B000BE048093BF049093C00489C147E11402E3
:1056C00090011124890108531B4F8A819B81AC8171
:1056D000BD81F80183879487A587B6872CEA35ECCE
:1056E00047E25EE36C897D898E899F890E94ABAE1B
:1056F000D8011F966D937D938D939C9352972CEABE
:1057000035EC47E25EE3688D798D8A8D9B8D0E9432
:1057100074ACF801638B748B858B968B58C1C35B1B
:10572000DF4F0FB6F894DEBF0FBECDBFDF91CF9134
:105730001F910F91FF90EF90DF90CF90BF90AF90AF
:105740009F908F907F906F905F904F903F902F90A1
:105750000C9471238AA49BA4ACA4BDA4880E991EAA
:10576000AA1EBB1E2AA53BA54CA55DA5281B390B6F
:105770004A0B5B0BCA01B9012E813F8148855985CF
:105780000E9475AFA50194010E94BAAFD701C6016E
:10579000820F931FA41FB51F84319105A105B10588
:1057A000FCF06C017D018C3E9105A105B1052CF04A
:1057B0006BEEC62ED12CE12CF12C40E8C416D1049E
:1057C000E104F104DCF08EEF90E0A0E0B0E08C1991
:1057D0009D09AE09BF098E839F83A887B98712C030
:1057E00054E1C52ED12CE12CF12C24E130E040E035
:1057F00050E02E833F834887598704C0CE82DF82E2
:10580000E886F986B701A6018BE995E00E941D168E
:105810004E815F816885798586E995E00E941D1635
:105820004A855C8D6D8D7E8D8FE895E00E942D16EA
:105830004F8D58A169A17AA188E895E00E942D16A4
:105840004E855F85433051050CF4AACD6E817F8172
:10585000888599850E940FAD20E030E040E850E453
:105860000E94ABAE6A837B838C839D832A853C8DAB
:105870004D8D5E8D6F8D78A189A19AA10E9493AB09
:105880002BED3FE049E450E40E94ABAE20E030E075
:1058900040E05FE30E94ABAE9B01AC016A817B817B
:1058A0008C819D810E9474AC6A877B878C879D87E1
:1058B000C501B4010E940FAD2FE632E143E85AE37F
:1058C0000E94ABAE4B015C012AE939E949E15FE393
:1058D0006A857B858C859D850E94ABAE6A837B83C0
:1058E0008C839D839B01AC010E9494ABA501940124
:1058F0000E9474AC6C8B7D8B8E8B9F8BA501940169
:105900006A817B818C819D810E94ABAE20E030E07A
:1059100040E05EE30E94ABAE688F798F8A8F9B8FE9
:105920004A855B856C857D8582E895E00E942D1611
:10593000B501A4018CE795E00E942D168CE695E058
:105940000E94E2154A815B816C817D8186E695E04B
:105950000E942D164C895D896E897F8980E695E0CD
:105960000E942D16488D598D6A8D7B8D8AE595E0B4
:105970000E942D168AE00E94721812CD2596EEAD77
:10598000FFAD259780831CCD1BA23DCD20E030E0EC
:1059900047E053E46FA578A989A99AA90E9470AE3F
:1059A00018160CF483CB83EA95E00E94E2150E945E
:1059B00071238FE78093B40420E030E040E051E4AD
:1059C00023962CAF3DAF4EAF5FAF2397A6CBC35B03
:1059D000DF4F0FB6F894DEBF0FBECDBFDF91CF9182
:1059E0001F910F91FF90EF90DF90CF90BF90AF90FD
:1059F0009F908F907F906F905F904F903F902F90EF
:105A00000895CF92DF92EF92FF92809195048823C0
:105A1000A1F10E946511C0909104D0909204E09091
:105A20009304F0909404DC01CB018C199D09AE091C
:105A3000BF09B7FD22C00E9465116B017C01209156
:105A4000950430E0A8EEB3E00E94DEAFDC01CB01AC
:105A50008C0D9D1DAE1DBF1D8093910490939204EB
:105A6000A0939304B093940480E04EDA8AE0FF9010
:105A7000EF90DF90CF900C947218FF90EF90DF9032
:105A8000CF9008952F923F924F925F926F927F92A4
:105A90008F929F92AF92BF92CF92DF92EF92FF923E
:105AA0000F931F93CF93DF93CDB7DEB764970FB6F5
:105AB000F894DEBF0FBECDBF898B6A8B81E08093E7
:105AC0006F021A821B821C821D8219861A861B860F
:105AD0001C8621E0288719821D863CE33E874CE125
:105AE0004F8756E4588BC12CD12C80E8E82E9FEBD1
:105AF000F92E812C912C54016091D0047091D10425
:105B0000072E000C880B990B0E940FAD6B8B7C8BC2
:105B1000182F092F9B01482F592FB601C7010E944A
:105B20006DAC882399F12091CC043091CD04409143
:105B3000CE045091CF046B897C89812F902F0E94D5
:105B40006DAC881F8827881F89838A89882311F173
:105B500099819923F9F080916F0264960FB6F894B9
:105B6000DEBF0FBECDBFDF91CF911F910F91FF9090
:105B7000EF90DF90CF90BF90AF909F908F907F90ED
:105B80006F905F904F903F902F900895CB8ADC8A62
:105B90001E2D0F2D0E9465116B017C01DC01CB01D4
:105BA00029853A854B855C85821B930BA40BB50B2D
:105BB000B7FD34C0D701C60188519C4FAF4FBF4FCE
:105BC00089879A87AB87BC8789899ED98FE493E0C0
:105BD0000E94E21581149104A104B104C9F0D50119
:105BE000C40188519C4FAF4FBF4FBC01CD016C1910
:105BF0007D098E099F0928EE33E040E050E00E94C5
:105C000098AFCA01B9014AE050E00E94541903C09C
:105C10008FE30E9472188AE00E9472180E94FBAA09
:105C20000E9465116093FF0B7093000C8093010C30
:105C30009093020C2090CC043090CD049091CE042F
:105C40009E83A091CF04AF839101492F5A2F6B8976
:105C50007C89812F902F0E9493AB2B013C0120E087
:105C600030E0A9010E9470AE87FF04C0C301B201F9
:105C7000905802C0C301B20120E030E040E251E49C
:105C800081149104A104B10481F40E946DAC87FFDA
:105C900012C0B88546015701BB2369F0E8EE8E0EAD
:105CA000E3E09E1EA11CB11C06C00E9470AE181637
:105CB00014F446015701F981FF2391F12A813B81B8
:105CC0004C815D81211531054105510541F0D70118
:105CD000C601821B930BA40BB50BB7FD21C091012C
:105CE0004E815F816D857E858F8598890E9493ABFB
:105CF00020E030E040EC5FE30E946DAC87FD2BCFED
:105D0000D701C601805A9541AF4FBF4F8A839B830D
:105D1000AC83BD832D863E869E819F87AF81A88BF5
:105D200080916F02882309F416CF81149104A10495
:105D3000B10431F41886CB88DC88E12EF02EDCCE5D
:105D4000B8EECB1AB3E0DB0AE108F108C818D908AD
:105D5000EA08FB08F7FCEECFFECE2F923F924F925F
:105D60005F926F927F928F929F92AF92BF92CF92EB
:105D7000DF92EF92FF920F931F93CF93DF93CDB7F4
:105D8000DEB763970FB6F894DEBF0FBECDBF898B29
:105D900081E080936F021A821B821C821D82198609
:105DA0001A861B861C8621E0288719821D863CE303
:105DB0003E874CE14F8756E4588BC12CD12C80E8AC
:105DC000E82E9FEBF92E812C912C54016091B204A6
:105DD0007091B304072E000C880B990B0E940FAD35
:105DE0006A8B7B8B182F092F9B01482F592FB601E7
:105DF000C7010E946DAC882399F12091AE043091C7
:105E0000AF044091B0045091B1046A897B89812F1D
:105E1000902F0E946DAC881F8827881F89838989ED
:105E2000882311F199819923F9F080916F0263968B
:105E30000FB6F894DEBF0FBECDBFDF91CF911F919B
:105E40000F91FF90EF90DF90CF90BF90AF909F9019
:105E50008F907F906F905F904F903F902F9008951C
:105E6000CA8ADB8A1E2D0F2D0E9465116B017C01F1
:105E7000DC01CB0129853A854B855C85821B930B20
:105E8000A40BB50BB7FD34C0D701C60188519C4F98
:105E9000AF4FBF4F89879A87AB87BC8780E034D8E4
:105EA0008BE493E00E94E21581149104A104B104F3
:105EB000C9F0D501C40188519C4FAF4FBF4FBC0101
:105EC000CD016C197D098E099F0928EE33E040E071
:105ED00050E00E9498AFCA01B9014AE050E00E9428
:105EE000541903C08FE30E9472188AE00E9472184E
:105EF0000E94FBAA0E9465116093FF0B7093000C37
:105F00008093010C9093020C9091AE049E83A0911B
:105F1000AF04AF832090B0043090B104292F3A2F02
:105F2000A1016A897B89812F902F0E9493AB2B015D
:105F30003C0120E030E0A9010E9470AE87FF04C060
:105F4000C301B201905802C0C301B20120E030E0A9
:105F500040EA50E481149104A104B10481F40E9448
:105F60006DAC87FF12C0B88546015701BB2369F0AD
:105F7000E8EE8E0EE3E09E1EA11CB11C06C00E943E
:105F800070AE181614F446015701F981FF2391F100
:105F90002A813B814C815D812115310541055105E7
:105FA00041F0D701C601821B930BA40BB50BB7FDC3
:105FB00021C02E813F81A1016D857E858F859889C5
:105FC0000E9493AB20E030E040EC5FE30E946DACB8
:105FD00087FD2BCFD701C601805A9541AF4FBF4FE8
:105FE0008A839B83AC83BD839E819D87AF81AE876F
:105FF0002F86388A80916F02882309F416CF811486
:106000009104A104B10431F41886CA88DB88E12E1A
:10601000F02EDCCEB8EECB1AB3E0DB0AE108F108D3
:10602000C818D908EA08FB08F7FCEECFFECEEBE96A
:10603000F4E0108211821282138214820895CF93A9
:10604000C82F6115710519F0CB010E94E21589E591
:1060500097E00E94E215C11103C08AE497E002C0F4
:106060008FE497E00E94E2158AE0CF910C947218B9
:106070008091E7048093E80408958091E6048823E2
:1060800019F01092E604089585EB97E00C9407AAA6
:106090008091E804811105C08091E204811101C062
:1060A000089562E070E080E090E00E94A015809189
:1060B000E304882339F061E070E080E090E00E9422
:1060C000A015F5CF08958093E8048093E704E0CF0E
:1060D00026982E9A25982D9A24982C9A3F98479A7C
:1060E0000A98129A0998119A81E0EDCF8093E804FA
:1060F000CFCF8093E204CCCF8091E604882339F19E
:106100009091E6048091E104981709F10E94F0153E
:1061100086EA97E00E94E2158091E60480FD1CC0AB
:106120008091E60484FD18C08091E60481FD1EC0C4
:106130008091E60485FD1AC08091E60482FD20C0AE
:106140008091E60486FD1CC08AE00E94721880914E
:10615000E6048093E104089580E00E94635AAB0155
:10616000BC0182EA97E00E942D16DECF81E00E94FA
:10617000635AAB01BC018EE997E00E942D16DCCF7B
:1061800082E00E94635AAB01BC018AE997E00E9459
:106190002D16DACFCF9380E897E00E94E21583B105
:1061A000C1E086FB882780F96AE777E08C2747DF24
:1061B00086B164E777E0881F8827881F40DF83B1B6
:1061C00085FB882780F96EE677E08C2738DF80B181
:1061D00082FB882780F968E677E08C2730DF83B17F
:1061E0008295817062E677E08C2729DF80B1869501
:1061F00081706CE577E08C27CF9121CF8091E50409
:106200001E9904C081608093E50403C08E7F809353
:10621000E5048091E504379B4DC080618093E504DF
:106220008091E5041D9904C082608093E50403C059
:106230008D7F8093E5048091E504029904C080621B
:106240008093E50403C08F7D8093E5048091E5048D
:106250001C9904C084608093E50403C08B7F809305
:10626000E5048091E504019904C080648093E5040D
:1062700003C08F7B8093E5049091E0048091E50456
:10628000981731F092E09093E3048093E00409C002
:106290008091E304882329F081508093E3048823CC
:1062A00069F08091E80481110CC08091E2048111B1
:1062B00008C008958F7E8093E504B2CF9093E404E4
:1062C000F0CF8091570580FF1BC0909158058091B9
:1062D000E40490FF0BC080FF13C08091E60481604E
:1062E0008093E60480E00E94615A0AC084FF08C0DF
:1062F0008091E60480618093E60480E00E94615A08
:106300008091570581FF1BC0909158058091E4044E
:1063100091FF0BC081FF13C08091E60482608093DF
:10632000E60481E00E94615A0AC085FF08C080919E
:10633000E60480628093E60481E00E94615A8091C5
:10634000570582FF20C08091580582FF10C08091C0
:10635000E2048823C1F08091E40482FF14C080919C
:10636000E60484608093E60482E00C94615A809194
:10637000E40486FF08C08091E60480648093E6040C
:1063800082E00C94615A089539CFCF938823A1F00D
:10639000C82F0E94F01584E50E9472186AE070E030
:1063A0008C2F90E00E94651980E20E94721883ECA5
:1063B00097E0CF910C94E215CF91089508958091C4
:1063C000940690919106891B8F7019F480E090E0FB
:1063D000089590918E06992351F0833030F48FEF19
:1063E000890F19F080938E06F1CF10928E06E091FE
:1063F000910686E5E89FF0011124EB56F94F808164
:1064000080FDE4CF809191068F5F8F70809393061B
:106410009091910680919206981306C08091930600
:1064200080939206CF010895CF010895EFE6F0E042
:1064300080818260808308958091580580FF09C023
:1064400080910B018270809309018FEF8093E904A2
:1064500009C080910B01809582708093090181E0D1
:106460008093E9048091580581FF0AC080910B0157
:1064700080958170809309018FEF8093EA0408C0B2
:1064800080910B0181708093090181E08093EA047F
:106490008091580582FF09C080910B018470809320
:1064A00009018FEF8093EB0409C080910B01809567
:1064B00084708093090181E08093EB040000000068
:1064C000000008950F930FB70F9300916E000F9384
:1064D0000B7F00936E0000916F000D7F00936F00A3
:1064E0000F930BB70F930CB70F921F922F933F93FD
:1064F0004F935F936F937F938F939F93AF93BF93CC
:10650000EF93FF9311240E94423BFF91EF91BF91C3
:10651000AF919F918F917F916F915F914F913F913B
:106520002F911F900F900CBF0F910BBF0F91026026
:10653000F89400936F000F9100936E000F910FBFBE
:106540000F911895CF92DF92EF92FF920F931F93C6
:10655000809156058823D1F01092560580915905F7
:1065600090915A05892B91F01092570510925A0577
:10657000109259059091940680919106981731F0E8
:10658000809191068F5F8F7080939106809159055D
:1065900090915A05892B09F4AAC140912505509183
:1065A0002605609127057091280590914D05009171
:1065B000190510911A0520911B0530911C05041B2B
:1065C000150B260B370B892F90E0A0E0B0E00817E1
:1065D00019072A073B0710F4D901C801E82F840FD7
:1065E000951FA61FB71F8093250590932605A0939E
:1065F0002705B09328052091840030918500225E04
:106600003F4F40913D0550913E0560913F0570918F
:10661000400580912D0590912E05A0912F05B091F8
:106620003005840F951FA61FB71F80933D059093DB
:106630003E05A0933F05B0934005B7FD1CC0409AAE
:106640004091ED045091EE046091EF047091F004DC
:106650008091E904082E000C990BAA0BBB0B840F48
:10666000951FA61FB71F8093ED049093EE04A0938F
:10667000EF04B093F00440914105509142056091C0
:106680004305709144058091310590913205A091A8
:106690003305B0913405840F951FA61FB71F809353
:1066A000410590934205A0934305B0934405B7FD7F
:1066B0001CC0419A4091F1045091F2046091F3049E
:1066C0007091F4048091EA04082E000C990BAA0B37
:1066D000BB0B840F951FA61FB71F8093F1049093E7
:1066E000F204A093F304B093F40440914505509153
:1066F0004605609147057091480580913505909158
:106700003605A0913705B0913805840F951FA61F57
:10671000B71F8093450590934605A0934705B09316
:106720004805B7FD1CC0429A4091F5045091F6040B
:106730006091F7047091F8048091EB04082E000C2E
:10674000990BAA0BBB0B840F951FA61FB71F809335
:10675000F5049093F604A093F704B093F8044091E5
:10676000490550914A0560914B0570914C05809107
:10677000390590913A05A0913B05B0913C05840FF5
:10678000951FA61FB71F8093490590934A05A093B4
:106790004B05B0934C05B7FD3CC0C090F904D090B8
:1067A000FA04E090FB04F090FC044091EC04042E09
:1067B000000C550B660B770B4C0D5D1D6E1D7F1D80
:1067C0004093F9045093FA046093FB047093FC0423
:1067D0004091290550912A0560912B0570912C0557
:1067E000841B950BA60BB70B8093490590934A0524
:1067F000A0934B05B0934C059091580580910E05E0
:1068000093FF04C0815080930E0503C08F5F809377
:106810000E05809184009091850082179307C8F33C
:1068200080913D0590913E05A0913F05B0914005B6
:10683000B7FD15C04091290550912A0560912B059F
:1068400070912C05841B950BA60BB70B80933D050F
:1068500090933E05A0933F05B093400540988091EA
:10686000410590914205A0914305B0914405B7FDC3
:1068700015C04091290550912A0560912B05709112
:106880002C05841B950BA60BB70B809341059093A9
:106890004205A0934305B093440541988091450576
:1068A00090914605A0914705B0914805B7FD15C0E8
:1068B0004091290550912A0560912B0570912C0576
:1068C000841B950BA60BB70B80934505909346054B
:1068D000A0934705B09348054298E15041F080915C
:1068E00084009091850082179307C8F388CE1F918A
:1068F0000F91FF90EF90DF90CF900895CF92DF92AD
:10690000EF92FF9280910D05882309F465C0C09035
:106910002505D0902605E0902705F09028054091A8
:106920001D0550911E0560911F05709120058091F5
:106930000E054C155D056E057F05E8F420911305E5
:1069400030911405E0911105F0911205E217F3075B
:1069500090F4815080930E05215031093093140535
:106960002093130540912502509126026091270241
:106970007091280234C0C416D506E606F706E8F47E
:10698000209113053091140540910F055091100589
:106990002417350790F48F5F80930E052F5F3F4FCC
:1069A000309314052093130540912502509126023F
:1069B000609127027091280212C08FEF9FEFDC01D7
:1069C0008093250290932602A0932702B093280279
:1069D0004FEF5FEFBA0103C04FEF5FEFBA01809155
:1069E0000E0587FD06C080910B018074809309011C
:1069F00006C080910B0180958074809309012091DD
:106A0000840030918500225E3F4F80910E058823DF
:106A100011F1439A80918400909185008217930729
:106A2000C8F380910E0587FF04C08F5F80930E0529
:106A300003C0815080930E05439880910E058823F2
:106A400021F3809184009091850082179307C8F309
:106A5000225E3F4FDACFCB01BA01FF90EF90DF907B
:106A6000CF900895BC012091590530915A0540916D
:106A7000590550915A052417350711F09A01F7CF9F
:106A800081E06217730709F080E00895CF93DF93E8
:106A9000EC0188819981AA81BB81EDEEF4E08083CD
:106AA0009183A283B383EB0188819981AA81BB8101
:106AB00084839583A683B783EA0188819981AA811B
:106AC000BB8180879187A287B387E90188819981FB
:106AD000AA81BB8184879587A687B787DF91CF91ED
:106AE00008953F924F925F926F927F928F929F9202
:106AF000AF92BF92CF92DF92EF92FF920F931F93CC
:106B0000CF93DF93CDB7DEB728970FB6F894DEBFEB
:106B10000FBECDBFA0915905B0915A05109739F11C
:106B20008090250590902605A0902705B090280517
:106B30004091190550911A0560911B0570911C0533
:106B400084169506A606B706C8F01092570510924F
:106B50005A051092590590919406809191069817C4
:106B600031F0809191068F5F8F708093910670ED68
:106B7000C72E77E0D72EE12CF12C97C1409121054B
:106B800050912205609123057091240548155905FF
:106B90006A057B0508F46EC00091520510915305FB
:106BA0002091540530915505D1964D915D916D918F
:106BB0007C91D497EE27059FF12D169FC001269F4B
:106BC000900D259F800D911D069FF00D811D9E1F2C
:106BD000159FF00D811D9E1F249FF00D811D9E1F8E
:106BE000149FF10D8E1F9E1FF6958E1F9E1F709F86
:106BF000800D911D719F900D1124FD01EB5BFF4FE6
:106C00004081518162817381480F591F611D711D3F
:106C10004093090550930A0560930B0570930C058A
:106C20003497C080D180E280F380C416D506E60692
:106C3000F70640F4C0920905D0920A05E0920B05D0
:106C4000F0920C054091090550910A0560910B05E1
:106C500070910C0581E298E0BB24B394FC01C590CF
:106C6000D590E590F490C416D506E606F70608F42C
:106C700075C27FC240901D0550901E0560901F0593
:106C800070902005481459046A047B0408F080C001
:106C900020914E0530914F0540915005509151057E
:106CA0002D833E834F835887D1960D911D912D9151
:106CB0003C91D4974D815E816F817885EE27419F0D
:106CC000F12D529FC001629F900D619F800D911D1B
:106CD000429FF00D811D9E1F519FF00D811D9E1F33
:106CE000609FF00D811D9E1F509FF10D8E1F9E1FF6
:106CF000F6958E1F9E1F349F800D911D359F900D20
:106D000011248C0120E030E0C0900905D0900A05E4
:106D1000E0900B05F0900C05CD01875B9F4FFC01C7
:106D20000C151D052E053F05C0F44081518162817F
:106D3000738149835A836B837C83C01AD10AE20A28
:106D4000F30AC416D506E606F70610F46A017B01BD
:106D500081E298E03324339410C0C080D180E28077
:106D6000F380F6CFF694E794D794C794330C049647
:106D700028E08D33920709F480C2FC01059115913A
:106D8000259134910C151D052E053F0558F375C24C
:106D900080910E058823D9F0D7964D915C91D897B4
:106DA00060E070E0009125021091260220912702F8
:106DB00030912802041715072607370741F0109273
:106DC000290210922A0210922B0210922C0240915A
:106DD000210250912202609123027091240277FFD8
:106DE0005CC0AF5BBF4F8D919D910D90BC91A02D6C
:106DF00021E238E041E0F901C590D590E590F490AA
:106E0000C816D906EA06FB0658F4B695A7959795D5
:106E10008795440F2C5F3F4F58E02D33350759F7C6
:106E200040934D0580329105A105B10520F480E223
:106E300090E0A0E0B0E08097A109B109811578E069
:106E40009707A105B10508F4CEC224E0929FF00196
:106E500011249F012F5B334FF90132966591749194
:106E6000EE27879FA001869F410D5E1F06944E1F4F
:106E70005E1F112460E070E0F90185919491A0E01B
:106E8000B0E0841B950BA60BB70B80932102909367
:106E90002202A0932302B0932402C0902102D0903A
:106EA0002202E0902302F0902402809159059091F3
:106EB0005A05892B09F01DC382DA90935A058093F5
:106EC0005905892B09F415C3E0915905F0915A052C
:106ED000808183FF19C09F012F5D3F4FAF01435E4B
:106EE0005F4FBF01675E7F4FCF014596CFDD909129
:106EF0009406809191069817F9F2809191068F5F20
:106F00008F7080939106D8CFC588D688E788F08C9B
:106F100081E0C114D104E104F10409F480E0018DA1
:106F2000128D238D348D011511052105310509F0D0
:106F30008260458D568D678D70A1411551056105A3
:106F4000710509F084608093570510924E051092E8
:106F50004F05109250051092510510925205109253
:106F60005305109254051092550585A196A1A7A12D
:106F7000B0A58093190590931A05A0931B05B093B3
:106F80001C05882499245401881A990AAA0ABB0A64
:106F90008092490590924A05A0924B05B0924C050B
:106FA0008092450590924605A0924705B09248050B
:106FB0008092410590924205A0924305B09244050B
:106FC00080923D0590923E05A0923F05B09240050B
:106FD000CC0CDD1CEE1CFF1CC0922D05D0922E05A2
:106FE000E0922F05F0923005000F111F221F331F72
:106FF0000093310510933205209333053093340507
:10700000440F551F661F771F409335055093360573
:10701000609337057093380541A152A163A174A113
:10702000440F551F661F771F4093390550933A054B
:1070300060933B0570933C05880F991FAA1FBB1FE7
:107040008093290590932A05A0932B05B0932C05D6
:1070500010922505109226051092270510922805FA
:1070600081A592A5A3A5B4A580932105909322059F
:10707000A0932305B093240585A596A5A7A5B0A93F
:1070800080931D0590931E05A0931F05B0932005C6
:1070900086A980930D05882309F183AD94AD909363
:1070A00012058093110581AD92AD909310058093E8
:1070B0000F051092290210922A0210922B021092B0
:1070C0002C0287A990ADA0E0B0E0809325029093B8
:1070D0002602A0932702B09328020BC08FEF9FEFE8
:1070E000DC018093250290932602A0932702B0939F
:1070F000280285A990915805891719F080935805A1
:107100009BD97CD88FEF9FEFDC0180932102909375
:107110002202A0932302B0932402E0915905F0913A
:107120005A05EB5BFF4F80819181A281B3818093EF
:10713000090590930A05A0930B05B0930C0521E275
:1071400038E041E0F901C590D590E590F490C8167B
:10715000D906EA06FB0608F46BC176C176956795F9
:1071600057954795BB0C0496E8E08D339E0709F0D0
:1071700075CDB0924D05403251056105710520F481
:1071800040E250E060E070E040525109610971094D
:10719000411588E058076105710500F194E0599F99
:1071A000F0011124CF018F5B934FFC013296E590E3
:1071B000F490F701DD244F9F50014E9FA10CBD1CA0
:1071C0000694AD1CBD1C1124FC01C590D490E12C8B
:1071D000F12CCA18DB08E108F10824C06A017B0120
:1071E000F694E794D794C794F601EC7FCF018F5BB8
:1071F000974F7C01FC0185919491F7013296E590BF
:10720000F49047704E9DB0014F9D700D1124AB015D
:1072100063E0569547956A95E1F76C01C41AD50A63
:10722000E12CF12C0C0D1D1D2E1D3F1D0093520550
:1072300010935305209354053093550590910D05F7
:1072400080910E05992309F465C0882309F42DCE99
:10725000D7968D919C91D897A0E0B0E040912502FF
:107260005091260260912702709128024817590711
:107270006A077B0709F051C018CE30924D05F0E245
:10728000CF16D104E104F10428F430E2C32ED12C4E
:10729000E12CF12CF0E2CF1AD108E108F108C11479
:1072A00028E0D206E104F10408F440C034E0D39EA3
:1072B000C00111248F5B934FFC013296059114910C
:1072C0006C2D3327619FA001609F410D531F0694D1
:1072D000431F531F1124FC01C590D490E12CF12CC5
:1072E000C41AD50AE108F1084D815E816F81788565
:1072F0004C0D5D1D6E1D7F1D40934E0550934F0537
:10730000609350057093510580910D05811132C035
:1073100080910E05882309F4C8CD1092290210929D
:107320002A0210922B0210922C02BFCD97018601E7
:107330003695279517950795F801EC7FCF018F5B60
:10734000974FFC0105911491FC013296459154919F
:107350003C2D3770349FC001359F900D112423E0E0
:10736000969587952A95E1F76801C81AD90AE12C04
:10737000F12CBACF430C511C611C711C48145904E8
:107380006A047B04C8F480910E05882309F48DCD2E
:10739000D7964D915C91D89760E070E000912502FE
:1073A0001091260220912702309128020417150718
:1073B0002607370709F479CD1092290210922A0284
:1073C00010922B0210922C02D7968D919C91D897F7
:1073D000A0E0B0E08093250290932602A0932702BC
:1073E000B093280262CDAC01BD01769567955795A3
:1073F0004795FA01EC7FAF014F5B574FFA0125919A
:107400003491FA013296659174918770869FA0013C
:10741000879F500D1124CA01F3E096958795FA9540
:10742000E1F7A901481B590BCA01A0E0B0E02DCD3E
:10743000B695A79597958795440F2C5F3F4F68E0C9
:107440002D33360709F07ECE40934D0580329105ED
:10745000A105B10520F480E290E0A0E0B0E08097C3
:10746000A109B109811558E09507A105B105F8F00A
:1074700064E0969FF00111249F012F5B334FF901C7
:10748000329665917491EE27879FA001869F410DEA
:107490005E1F06944E1F5E1F1124F901C590D49003
:1074A000E12CF12CC41AD50AE108F10822C0AC0184
:1074B000BD017695679557954795FA01EC7FAF0129
:1074C0004F5B574FFA01C590D490FA01329645911F
:1074D00054918770849F9001859F300D1124C901BC
:1074E000A3E096958795AA95E1F7C81AD90AE12CE9
:1074F000F12CC701B60128960FB6F894DEBF0FBE77
:10750000CDBFDF91CF911F910F91FF90EF90DF9052
:10751000CF90BF90AF909F908F907F906F905F9033
:107520004F903F900895CF92DF92EF92FF921F937A
:10753000CF93DF938FEF9FEF909389008093880024
:107540001AE0C0E0D0E0789480911505909116057E
:10755000A0911705B0911805892B8A2B8B2B11F45C
:107560000E94A2328091290290912A02A0912B02BE
:10757000B0912C02892B8A2B8B2B49F4BFD96093B5
:10758000290270932A0280932B0290932C028091FF
:10759000150590911605A0911705B0911805892B36
:1075A0008A2B8B2B49F49DDA609315057093160591
:1075B0008093170590931805C0901505D090160577
:1075C000E0901705F09018054091290250912A0289
:1075D00060912B0270912C02FC2DED2D3E2D2F2D54
:1075E0004C155D056E057F0520F4F42FE52F362F31
:1075F000272F8F2F9E2FA32FB22F009721E0A207B6
:10760000B10520F08FEF9FEFA0E0B0E0C81AD90AD3
:10761000EA0AFB0AC0921505D0921605E0921705FA
:10762000F09218054F3F2FEF52076207720761F083
:10763000481B590B6A0B7B0B4093290250932A027B
:1076400060932B0270932C02F89420918400309167
:107650008500205F3F4F115039F0C80FD91FC21766
:10766000D30708F470CF01C0E901D0938900C0931B
:1076700088007894DF91CF911F91FF90EF90DF9079
:10768000CF90089550CF90916F0091FB222720F961
:1076900091FF05C090916F009D7F90936F0094E0E3
:1076A000899FF0011124E351FB4F60817181828138
:1076B0009381222329F020916F00226020936F0094
:1076C000089590916F0091FB222720F991FF05C04A
:1076D00090916F009D7F90936F0034E0839FC00175
:1076E0001124FC01E351FB4F408151816281738180
:1076F000FC01E350FB4F408351836283738381E03D
:1077000080935605222329F080916F008260809338
:107710006F00089590916F0091FB222720F991FF4F
:1077200005C090916F009D7F90936F0094E0899FBA
:10773000F0011124E350FB4F6081718182819381BC
:10774000222329F020916F00226020936F0008957A
:107750004F925F926F927F928F929F92AF92BF9261
:10776000CF92DF92EF92FF9280916F0081FB992779
:1077700090F981FF05C080916F008D7F80936F002D
:107780004090ED045090EE046090EF047090F0048F
:107790008090F1049090F204A090F304B090F4046F
:1077A000C090F504D090F604E090F704F090F8044F
:1077B000992329F080916F00826080936F0087E1A8
:1077C00098E00E94E2154AE050E0C301B2010E9435
:1077D000541983E198E00E94E2154AE050E0C501A7
:1077E000B4010E9454198FE098E00E94E2154AE02B
:1077F00050E0C701B6010E9454198AE0FF90EF9053
:10780000DF90CF90BF90AF909F908F907F906F90C0
:107810005F904F900C947218DB019091670599234B
:1078200009F440C0833070F494E0899FF001112482
:10783000E55AFA4FAB01770F660B770B4083518304
:1078400062837383813091F018F08230E9F00895FB
:107850002FEF30E00E94EDAF20ED37E040E050E048
:107860000E94BAAFB9018EE20C9431122FEF30E0D2
:107870000E94EDAF20ED37E040E050E00E94BAAF4B
:10788000B9018DE20C9431122FEF30E00E94EDAF80
:1078900020ED37E040E050E00E94BAAFB9018CE241
:1078A0000C943112089580916705882391F06091BE
:1078B0005B0570915C0580E0AFDF60915F057091C2
:1078C000600581E0A9DF609163057091640582E045
:1078D000A3CF0895EAE0F1E0808188608083808111
:1078E00080618083808180628083DDDFE1E2F1E07E
:1078F0008081887F81608083089567FD2CC08130FE
:1079000061F028F0823099F08330D9F024C06623EA
:1079100011F0A19A2AC0A19828C080910801611194
:10792000809580788093060147FF27C00895809155
:1079300008016111809580748093060147FF23C080
:1079400008958091080161118095887080930601E7
:1079500047FF21C0089547FD26C0813071F038F0FF
:10796000823089F08330B9F0089547FD1CC044236C
:1079700011F0A09A0895A0980895442311F0A29AB6
:107980000895A29808958091080141118095807210
:1079900080930601089580910801411180958071BE
:1079A0008093060108950895643091F040F46130A9
:1079B00059F06230A9F420E040E061E09ECF6830E9
:1079C00059F0603149F00CC020E040E060E095CF14
:1079D00020E041E060E091CF20E041E061E08DCF28
:1079E0000E94F31587EF97E00C94E2150F931F9315
:1079F000CF93999A989A80910701806880930701A4
:107A00009A9A809107018064809307018091070111
:107A1000806280930701809107018860809307014D
:107A20008091070180618093070101E313E0C0E0CA
:107A3000F80161918F018C2FB7DFCF5FC630C1F79E
:107A4000CF911F910F910895D1DFEAE0F1E080819D
:107A50008260808380818160808380818460808374
:107A60008081806480830F9A179A0E9A169A0D9AD5
:107A7000159A0C9A149A389A4098179A8091910501
:107A80008E7F80939105399A4198169A809191053D
:107A90008D7F809391053A9A4298159A809191052D
:107AA0008B7F809391053B9A4398149AA0E8B0E0AD
:107AB0008C918C7F8C93E1E8F0E08081877E8860F8
:107AC00080838C918F738C938081887F8260808388
:107AD00080E090E490938900809388001092850064
:107AE00010928400EFE6F0E08081826080837894D9
:107AF00082E0809358050E941C3281E080936705E4
:107B0000E9CE82EE97E00E94E215919902C080E3EF
:107B100001C081E30E947218909902C080E301C005
:107B200081E30E9472188EED97E00E94E215809129
:107B30000601881F8827881F805D0E94721892990D
:107B400002C080E301C081E30E9472188AED97E0D1
:107B50000E94E2158091060186FD02C080E301C00B
:107B600081E30E9472188091060185FD02C080E3C6
:107B700001C081E30E94721885ED97E00E94E21532
:107B80008091060183FD02C080E301C081E30E9471
:107B900072188091060184FD02C080E301C081E378
:107BA0000C947218CF93DF93CDB7DEB760970FB602
:107BB000F894DEBF0FBECDBF80915002909151026C
:107BC000A0915202B091530289839A83AB83BC8304
:107BD0008091540290915502A0915602B0915702A3
:107BE0008D839E83AF83B88780915802909159020C
:107BF000A0915A02B0915B0289879A87AB87BC87B4
:107C000080915C0290915D02A0915E02B0915F0252
:107C10008D879E87AF87B88B0E94176B6091640237
:107C200070916502072E000C880B990B0E940FAD16
:107C30002AE037ED43E25CE30E94ABAE6093600262
:107C400070936102809362029093630280E00E94CD
:107C5000CE5081E00E94CE5082E00E94CE5023DEC2
:107C60000E945E6B40E150E060E572E0CE0101965B
:107C70000E9425B4892B51F060960FB6F894DEBFB0
:107C80000FBECDBFDF91CF910C94964E60960FB68C
:107C9000F894DEBF0FBECDBFDF91CF91089587343A
:107CA000924041F00E94F31586E893E10E94E215AC
:107CB00081E0089580E00895EF92FF920F931F9363
:107CC000CF93DF93CDB7DEB7C458D1090FB6F89480
:107CD000DEBF0FBECDBFED961CAE1DAE1EAE1FAEFD
:107CE000ED9785E492E5A2E5B0E0E9968CAF9DAF13
:107CF000AEAFBFAFE997CF57DF4F19821882C15897
:107D0000D04084E690E0C158DF4F99838883CF57F5
:107D1000D0400E948F16109269059E012F573F4F49
:107D200044E050E0BE016B587F4FCE0181589F4F19
:107D30000E949316C158DF4F88819981CF57D04058
:107D40000296C158DF4F99838883CF57D040CF57D1
:107D5000DF4F19821882C158D04081E0CC57DF4FE5
:107D60008883C458D0409E012F573F4F41E050E0D8
:107D7000BE016C577F4FCE0181589F4F0E949316D2
:107D80009E012F573F4F48E450E066E476E0CE0175
:107D900081589F4F0E9493169E012F573F4F40E1FD
:107DA00050E066E176E0CE0181589F4F0E94931625
:107DB0008AE097EDA3EABCE3ED968CAF9DAFAEAF42
:107DC000BFAFED979E012F573F4F44E050E0BE01FB
:107DD00067587F4FCE0181589F4F0E9493168E01A6
:107DE0000F5F1F4F8CE0F80111928A95E9F79E0111
:107DF0002F573F4F4CE050E0B801CE0181589F4FC4
:107E00000E94931680E090E0A0E2B1E489839A8317
:107E1000AB83BC839E012F573F4F44E050E0B80135
:107E2000CE0181589F4F0E949316ED961CAE1DAE59
:107E30001EAE1FAEED9783E0AE968FAFAE978983EF
:107E40009E012F573F4F44E050E0BE0167587F4FDF
:107E5000CE0181589F4F0E9493169E012F573F4F8E
:107E600041E050E0BE0163597F4FCE0181589F4FE2
:107E70000E9493169E012F573F4F41E050E0B801FA
:107E8000CE0181589F4F0E9493162AE0F22EFA9459
:107E90009E012F573F4F44E050E0FF2049F0BE01C4
:107EA00067587F4FCE0181589F4F0E949316EFCFA6
:107EB0006AE675E0CE0181589F4F0E9493169E019D
:107EC0002F573F4F44E250E061EF75E0CE018158FB
:107ED0009F4F0E94931683E0CD57DF4F8883C3588E
:107EE000D040EE968FAFEE97E1961CAE1DAE1EAE63
:107EF0001FAEE19719821A821B821C82ED961CAE7E
:107F00001DAE1EAE1FAEED979E012F573F4F41E0B5
:107F100050E0BE016D577F4FCE0181589F4F0E94A8
:107F200093169E012F573F4F41E050E0BE0163582A
:107F30007F4FCE0181589F4F0E9493169E012F576D
:107F40003F4F44E050E0B801CE0181589F4F0E945E
:107F500093169E012F573F4F44E050E0BE016359F6
:107F60007F4FCE0181589F4F0E9493169AE0E92ED1
:107F7000F12CF1E0EF1AF10871F09E012F573F4FFD
:107F800044E050E0BE0167587F4FCE0181589F4FBB
:107F90000E949316EECFAE961FAEAE978FEF8983F9
:107FA0009E012F573F4F41E050E0BE0163597F4F84
:107FB000CE0181589F4F0E9493169E012F573F4F2D
:107FC00041E050E0B801CE0181589F4F0E949316C6
:107FD00080E1F82EF8018F2D11928A95E9F79E0124
:107FE0002F573F4F40E150E0B801CE0181589F4FDD
:107FF0000E94931688EC90E0AF969FAF8EAFAF973C
:1080000080EF90E0E1969FAF8EAFE19786E490E03D
:108010009A8389838EE690E09C838B83EE961FAED5
:10802000EE97EF961FAEEF979E012F573F4F44E01C
:1080300050E0BE0163597F4FCE0181589F4F0E948F
:1080400093169E012F573F4F44E050E0B801CE01F8
:1080500081589F4F0E9493169E012F573F4F42E039
:1080600050E0BE0163587F4FCE0181589F4F0E9460
:108070009316F8011192FA94E9F780E090E0A0E8F5
:10808000BFE38D879E87AF87B88B8091D304909193
:10809000D404A091D504B091D60489839A83AB838C
:1080A000BC838091D7049091D804A091D904B09159
:1080B000DA048D839E83AF83B8878091DB0490912F
:1080C000DC04A091DD04B091DE0489879A87AB8738
:1080D000BC879E012F573F4F40E150E0B801CE01D1
:1080E00081589F4F0E94931684E190E09A83898380
:1080F0009E012F573F4F42E050E0B801CE0181581A
:108100009F4F0E9493169E012F573F4F4CE050E027
:1081100065EB74E0CE0181589F4F0E94931680E278
:1081200090E09A8389839E012F573F4F42E050E0B1
:10813000B801CE0181589F4F0E94931681E0898338
:108140009E012F573F4F41E050E0B801CE018158CA
:108150009F4F0E94931680E2E1E8F2E0D80101907F
:108160000D928A95E1F79E012F573F4F40E250E074
:10817000B801CE0181589F4F0E949316AE961FAE54
:10818000AE979E012F573F4F41E050E0BE0163592B
:108190007F4FCE0181589F4F0E949316198280E035
:1081A00090E0A0E4B0E4ED968CAF9DAFAEAFBFAF72
:1081B000ED979E012F573F4F41E050E0B801CE01AF
:1081C00081589F4F0E9493169E012F573F4F44E0C6
:1081D00050E0BE0167587F4FCE0181589F4F0E94EB
:1081E00093168AE1F80111928A95E9F79E012F57BB
:1081F0003F4F4AE150E0B801CE0181589F4F0E94A5
:10820000931684E3E1EAF2E0D80101900D928A9599
:10821000E1F79E012F573F4F44E350E0B801CE01F4
:1082200081589F4F0E9493161A8219821C821B82CA
:108230001E821D829E012F573F4F46E050E0B8013D
:10824000CE0181589F4F0E9493168DE0F801119244
:108250008A95E9F79E012F573F4F4DE050E0B80156
:10826000CE0181589F4F0E9493169E012F573F4F7A
:1082700044E050E068EB75E0CE0181589F4F0E94CA
:1082800093169E012F573F4F4CE050E06BE575E091
:10829000CE0181589F4F0E9493168CE6F8011192EF
:1082A0008A95E9F79E012F573F4F4CE650E0B80101
:1082B000CE0181589F4F0E9493169E012F573F4F2A
:1082C0004CE050E065EE75E0CE0181589F4F0E9472
:1082D0009316E1961CAE1DAE1EAE1FAEE197E5965D
:1082E0001CAE1DAE1EAE1FAEE5979E012F573F4F31
:1082F00048E050E0BE0163597F4FCE0181589F4F47
:108300000E9493168091690581114FC0C158DF4FBB
:1083100008811981CF57D04004561109CF57DF4F3C
:1083200088819981C158D040AF969FAF8EAFAF97EB
:1083300084E690E0C158DF4F99838883CF57D040BF
:108340009E012F573F4F44E050E067E373E0CE01BA
:1083500081589F4F0E9493169E012F573F4F42E036
:1083600050E0BE0163597F4FCE0181589F4F0E945C
:1083700093160E94F015B80184E793E10E944D1610
:10838000AF964EAD5FADAF9760E070E087E693E1EA
:108390000E94571684E693E10E94E215C8017FDC33
:1083A00090916905892B809369050E94911690919F
:1083B000690581E08927CC57DF4F0FB6F894DEBFFF
:1083C0000FBECDBFDF91CF911F910F91FF90EF9026
:1083D00008951F93CF93DF93CDB7DEB72C970FB6D9
:1083E000F894DEBF0FBECDBFA6E4B6E020E030E0DB
:1083F000C9012430310510F083E090E0880F991F07
:10840000880F991FFC01ED54FD4E459155916591E2
:10841000749154964D935D936D937C935797FC01A3
:10842000ED55FD4E459155916591749194964D93FE
:108430005D936D937C939797FC01ED56FD4E4591AE
:108440005591659174914D935D936D937D932F5FDD
:108450003F4F2430310509F0CBCF80E29EE4A0E00D
:10846000B0E08093560690935706A0935806B093B9
:10847000590680E090E0AAEFB4E480937A069093E6
:108480007B06A0937C06B0937D0640E050E86BE34A
:1084900075E440937E0650937F0660938006709348
:1084A00081068093820690938306A0938406B093FE
:1084B0008506109286061092870610928806109202
:1084C000890610928A0610928B0610928C061092E2
:1084D0008D0680E090E0A0E4B1E4809316069093CE
:1084E0001706A0931806B093190680931A06909366
:1084F0001B06A0931C06B0931D068DEC9CECACEC07
:10850000BEE380931E0690931F06A0932006B093AF
:10851000210680E090E0A0E2B1E4809322069093EF
:108520002306A0932406B09325060E94851A82E5AF
:1085300098EBAEE9BFEB80936A0590936B05A0932F
:108540006C05B0936D0580E090E0A8EAB1E48093FB
:10855000D3049093D404A093D504B093D60485E3B8
:1085600091E5A5E9BEE38093D7049093D804A09346
:10857000D904B093DA0480ED9EEFACEBB3E48093C2
:10858000DB049093DC04A093DD04B093DE0480E070
:1085900090E0A3E9B3E48093B5049093B604A0936C
:1085A000B704B093B80483EC94E6AAE2B1E48093F4
:1085B000B9049093BA04A093BB04B093BC0480EBBD
:1085C00098EBA1E1B5E48093BD049093BE04A09321
:1085D000BF04B093C00481E00E9463300E94DE318A
:1085E0001092B8051092B9051092BA051092BB0509
:1085F0008CE0E5EDF2E0DE01119601900D928A9596
:10860000E1F713E01150C0F084E0189F90011124AD
:10861000E1E0F0E0EC0FFD1FE20FF31F60817181DC
:1086200082819381F901E55AFA4F608371838283D5
:108630009383812FF1D8E6CFB5DA0E94F01580E759
:1086400092E12C960FB6F894DEBF0FBECDBFDF913E
:10865000CF911F910C94E215CF93C82F811102C0C6
:108660000E94F01589E592E10E94E21584E490E110
:108670000E94E2158AE00E9472188AE00E94721835
:10868000C11106C00E94F01588E492E10E94E21533
:108690006FEF81E08C270E94AD93C11108C00E944A
:1086A000F0158AE292E10E94E2150E94F0154091D5
:1086B0006A0650916B0660916C0670916D0681E2BE
:1086C00092E10E942D1640916E0650916F066091C6
:1086D0007006709171068EE192E10E942D16409114
:1086E00072065091730660917406709175068BE165
:1086F00092E10E942D164091760650917706609186
:1087000078067091790688E192E10E942D168AE040
:108710000E947218C11108C00E94F01586EF91E105
:108720000E94E2150E94F01560914606709147067E
:1087300080914806909149060E940DADAB01BC01A5
:108740008DEE91E10E942D1660914A0670914B06C4
:1087500080914C0690914D060E940DADAB01BC017D
:108760008AEE91E10E942D1660914E0670914F069F
:1087700080915006909151060E940DADAB01BC0155
:1087800087EE91E10E942D1660915206709153067A
:1087900080915406909155060E940DADAB01BC012D
:1087A00084EE91E10E942D168AE00E947218C11198
:1087B00008C00E94F0158AE991E10E94E2150E942A
:1087C000F01540917A0650917B0660917C0670917D
:1087D0007D0681E991E10E942D1640917E0650911F
:1087E0007F0660918006709181068EE891E10E947B
:1087F0002D164091820650918306609184067091F7
:1088000085068BE891E10E942D168AE00E9472187D
:10881000C11113C00E94F01583E491E10E94E2159A
:1088200088E191E10E94E21589E091E10E94E21560
:108830008AE00E9472180E94F015609156067091AD
:10884000570680915806909159060E940DADAB01D4
:10885000BC0180E091E10E942D1640918606509166
:10886000870660918806709189068DEF90E10E94DD
:108870002D1640918A0650918B0660918C0670915E
:108880008D068AEF90E10E942D16409116065091B8
:108890001706609118067091190687EF90E10E9403
:1088A0002D1640911A0650911B0660911C0670917E
:1088B0001D0684EF90E10E942D1640911E065091F6
:1088C0001F06609120067091210681EF90E10E94C1
:1088D0002D16409122065091230660912406709136
:1088E00025068EEE90E10E942D168AE00E947218F5
:1088F000C11108C00E94F0158AED90E10E94E215B6
:108900000E94F0156091150670E081ED90E10E94E3
:1089100013168AE00E947218C11108C00E94F01557
:1089200082EC90E10E94E2150E94F0154091D30480
:108930005091D4046091D5047091D60489EB90E1F4
:108940000E942D162CEA35EC47E25EE36091D704D5
:108950007091D8048091D9049091DA040E9474AC8B
:10896000AB01BC0186EB90E10E943D162CEA35EC90
:1089700047E25EE36091DB047091DC048091DD04EA
:108980009091DE040E94ABAEAB01BC0183EB90E1A1
:108990000E943D168AE00E947218C11102C00E9416
:1089A000F0154091B5045091B6046091B7047091F0
:1089B000B8048AEA90E10E942D162CEA35EC47E2D1
:1089C0005EE36091B9047091BA048091BB04909108
:1089D000BC040E9474ACAB01BC0187EA90E10E9428
:1089E0003D162CEA35EC47E25EE36091BD047091E0
:1089F000BE048091BF049091C0040E94ABAEAB0155
:108A0000BC0184EA90E10E943D168AE00E9472183F
:108A1000C11110C00E94F01585E990E10E94E21595
:108A200084E490E10E94E21581E490E10E94E21565
:108A30000E94F01540916A0550916B0560916C059C
:108A400070916D058CE890E10E942D168AE00E94DD
:108A50007218C11108C00E94F0158BE790E10E94C6
:108A6000E2150E94F0154091B8055091B90560914A
:108A7000BA057091BB0582E790E10E942D168AE04D
:108A80000E947218C11108C00E94F01589E590E19A
:108A90000E94E2150E94F01540915B0550915C0523
:108AA00060915D0570915E0580E590E10E9457162A
:108AB00040915F055091600560916105709162057C
:108AC0008DE490E10E945716409163055091640532
:108AD00060916505709166058AE490E10E945716E1
:108AE0008AE0CF910C9472182F923F924F925F922E
:108AF0006F927F928F929F92AF92BF92CF92DF92AE
:108B0000EF92FF920F931F93CF93DF93CDB7DEB712
:108B1000C45AD1090FB6F894DEBF0FBECDBF2DB732
:108B20003EB7CD55DF4F39832883C35AD040C7564F
:108B3000DF4F19821882C959D04084E690E0C956A7
:108B4000DF4F99838883C759D0400E948F1601E078
:108B50009E0127563F4F44E050E0BE016F567F4FC5
:108B6000CE0189569F4F0E94E8169E0127563F4F1F
:108B700042E050E0BE016B567F4FCE0189569F4FB9
:108B80000E94E81643E050E0BE016F567F4F87E336
:108B900093E00E9444B4892B19F1CC56DF4F8881B1
:108BA000C459D040882359F08FE3CF56DF4F8883D4
:108BB000C159D040CE56DF4F1882C259D0400E94D2
:108BC000F015BE016F567F4F83E493E10E94F615C6
:108BD00085E393E10E94E21581E08093690524C555
:108BE000C357DF4F188219821A821B82CD58D0409A
:108BF000C756DF4F19821882C959D04001E09E0143
:108C000027563F4F41E050E0BE0164567F4FCE01F2
:108C100089569F4F0E94E8168DB79EB7C156DF4F09
:108C200099838883CF59D0406E019DE7C90ED11C2E
:108C300080E1E1EEF2E0D60101900D928A95E1F734
:108C40007E01EDE6EE0EF11C80E1E1EFF2E0D701EE
:108C500001900D928A95E1F780E1E1E0F3E09E0159
:108C60002F5F3F4F5901D90101900D928A95E1F78D
:108C7000C456DF4F4881CC59D04050E04D5F5F4F24
:108C8000440F551F440F551F8DB79EB7841B950B7E
:108C90000FB6F8949EBF0FBE8DBFEDB7FEB73196ED
:108CA0001F010091680511E0012728563F4FBF01C1
:108CB000CE0189569F4F0E94E81600916805012752
:108CC0009E0127563F4F44E050E066E576E0CE0136
:108CD00089569F4F0E94E816C456DF4F8880CC59B2
:108CE000D040912CF3E08F0E911C880C991C880CBD
:108CF000991C2DB73EB7281939090FB6F8943EBF15
:108D00000FBE2DBF8DB79EB701962C01EDB7FEB7F4
:108D1000E819F9090FB6F894FEBF0FBEEDBF2DB7E5
:108D20003EB72F5F3F4F39010091680501279E0133
:108D300027563F4FA401BC01CE0189569F4F0E9488
:108D4000E8160091680501279E0127563F4FA401B0
:108D5000B301CE0189569F4F0E94E81630916805F5
:108D6000C256DF4F3883CE59D040332309F4CBC0ED
:108D700011E0C256DF4F0881CE59D04001279E0135
:108D800027563F4F44E050E06AE776E0CE0189562F
:108D90009F4F0E94E8160091680501279E01275603
:108DA0003F4F44E050E06EE776E0CE0189569F4F9A
:108DB0000E94E8160091680501279E0127563F4F43
:108DC00044E050E062E876E0CE0189569F4F0E9471
:108DD000E8160091680501279E0127563F4F44E0A1
:108DE00050E066E876E0CE0189569F4F0E94E81673
:108DF0000091680501279E0127563F4F44E050E04F
:108E00006AE876E0CE0189569F4F0E94E8160091ED
:108E1000680501279E0127563F4F40E150E066E17B
:108E200076E0CE0189569F4F0E94E81600916805B2
:108E300001279E0127563F4F44E050E0BE01635793
:108E40007F4FCE0189569F4F0E94E816C156DF4FD3
:108E500088819981CF59D0400FB6F8949EBF0FBE3C
:108E60008DBF0091680501279E0127563F4F4CE0BA
:108E700050E0BE016F5F7F4FCE0189569F4F0E9429
:108E8000E8160091680501279E0127563F4F44E0F0
:108E900050E0BE0163577F4FCE0189569F4F0E941D
:108EA000E8160091680501279E0127563F4F44E0D0
:108EB00050E0BE0163577F4FCE0189569F4F0E94FD
:108EC000E81601E09E0127563F4F41E050E0B70110
:108ED000CE0189569F4F0E94E8169E0127563F4FAC
:108EE00041E050E0BE016F5F7F4FCE0189569F4F3A
:108EF0000E94E816F701A0808981A89E50011124E4
:108F0000812C912C9DC0C456DF4F8881CC59D04014
:108F100090E09C012E5F3F4FCF55DF4F3983288370
:108F2000C15AD040A6E4B6E040E050E080E090E0D6
:108F30004601B70131E0C356DF4F3883CD59D040E9
:108F4000CF55DF4FE881F981C15AD040E817F907C2
:108F500064F4C356DF4F1882CD59D0409C01843051
:108F6000910558F023E030E008C0F101E40FF51F4F
:108F700000811181228133810BC0220F331F220F08
:108F8000331FF401E20FF31F00811181228133812D
:108F90000D931D932D933D93C356DF4FF881CD590B
:108FA000D040FF2341F0F201E40FF51F0081118151
:108FB0002281338111C09C018430910510F023E09F
:108FC00030E0220F331F220F331FFB01E20FF31F8C
:108FD000008111812281338150960D931D932D9331
:108FE0003C935397C356DF4F2881CD59D04022235D
:108FF00041F0F301E40FF51F0081118122813381DB
:1090000011C09C018430910510F023E030E0220F64
:10901000331F220F331FF501E20FF31F008111816F
:109020002281338190960D931D932D933C939397BA
:1090300001964C5F5F4F8430910509F07BCF98CE4D
:10904000009168058A149B0491F001279E01275620
:109050003F4F44E050E0BE0163577F4FCE01895639
:109060009F4F0E94E8163FEF831A930AE9CF11E061
:1090700001279E0127563F4F44E050E06AE675E025
:10908000CE0189569F4F0E94E8160091680501277E
:109090009E0127563F4F44E250E061EF75E0CE015C
:1090A00089569F4F0E94E81601E09E0127563F4FC8
:1090B00041E050E0BE0165567F4FCE0189569F4F7B
:1090C0000E94E8169E0127563F4F41E050E0B6014E
:1090D000CE0189569F4F0E94E8160091680501272E
:1090E0009E0127563F4F44E050E0B701CE0189561C
:1090F0009F4F0E94E8160091680501279E012756A0
:109100003F4F44E050E0BE016F5F7F4FCE01895674
:109110009F4F0E94E816C556DF4FA880CB59D0401C
:10912000F6018081A89E50011124812C912C009180
:1091300068058A149B0491F001279E0127563F4F32
:1091400044E050E0BE0163577F4FCE0189569F4FE8
:109150000E94E816FFEF8F1A9F0AE9CF11E001275E
:109160009E0127563F4F41E050E0B701CE0189569E
:109170009F4F0E94E8160091680501279E0127561F
:109180003F4F41E050E0BE016F5F7F4FCE018956F7
:109190009F4F0E94E8160091680501279E012756FF
:1091A0003F4F40E150E0BE016F5F7F4FCE018956D7
:1091B0009F4F0E94E8160091680501279E012756DF
:1091C0003F4F44E050E0B701CE0189569F4F0E94C7
:1091D000E8160091680501279E0127563F4F44E09D
:1091E00050E0BE016F5F7F4FCE0189569F4F0E94B6
:1091F000E8160091680501279E0127563F4F42E07F
:1092000050E0B601CE0189569F4F0E94E8160091AA
:10921000680501279E0127563F4F40E150E0BE01FF
:109220006F5F7F4FCE0189569F4F0E94E8160091D5
:10923000680501112EC089809A80AB80BC8020E037
:1092400030E84BE355E4C501B4010E946DAC8823BE
:1092500001F18092D3049092D404A092D504B092EC
:10926000D6048D819E81AF81B8858093D704909379
:10927000D804A093D904B093DA0489859A85AB8584
:10928000BC858093DB049093DC04A093DD04B09351
:10929000DE0411E001279E0127563F4F42E050E0D7
:1092A000BE016F5F7F4FCE0189569F4F0E94E81627
:1092B0000091680501279E0127563F4F4CE050E082
:1092C000BE016F5F7F4FCE0189569F4F0E94E81607
:1092D00000916805011115C020E030E84BE355E42A
:1092E00069817A818B819C810E946DAC882349F0D1
:1092F0008CE0FE013196A5EBB4E001900D928A95C9
:10930000E1F711E001279E0127563F4F42E050E070
:10931000BE016F5F7F4FCE0189569F4F0E94E816B6
:109320000091680501279E0127563F4F41E050E01C
:10933000BE016F5F7F4FCE0189569F4F0E94E81696
:109340000091680501279E0127563F4F40E250E0FB
:10935000BE016F5F7F4FCE0189569F4F0E94E81676
:109360000091680501279E0127563F4F41E050E0DC
:10937000B701CE0189569F4F0E94E81600916805FB
:1093800001279E0127563F4F45E050E0BE016F5F29
:109390007F4FCE0189569F4F0E94E8168091680545
:1093A000811102C00E94DE310091680511E00127A1
:1093B0009E0127563F4F4AE150E0BE016F5F7F4F4D
:1093C000CE0189569F4F0E94E8160091680501273B
:1093D0009E0127563F4F44E350E0BE016F5F7F4F31
:1093E000CE0189569F4F0E94E8160091680501271B
:1093F0009E0127563F4F46E050E0BE016F5F7F4F12
:10940000CE0189569F4F0E94E816009168050127FA
:109410009E0127563F4F4DE050E0BE016F5F7F4FEA
:10942000CE0189569F4F0E94E816009168050127DA
:109430009E0127563F4F44E050E0BE016F5F7F4FD3
:10944000CE0189569F4F0E94E816009168050111D0
:109450000CC089819A81AB81BC818093B8059093BF
:10946000B905A093BA05B093BB0581E008279E011A
:1094700027563F4F4CE050E0BE016F5F7F4FCE015B
:1094800089569F4F0E94E81600916805011109C096
:109490008CE0FE013196ABE5B5E001900D928A9526
:1094A000E1F711E001279E0127563F4F4CE650E0BF
:1094B000BE016F5F7F4FCE0189569F4F0E94E81615
:1094C00019821A821B821C821D821E821F821886AC
:1094D00019861A861B861C860091680501279E0145
:1094E00027563F4F4CE050E0BE016F5F7F4FCE01EB
:1094F00089569F4F0E94E8160091680501279E013A
:1095000027563F4F48E050E0BE016F5F7F4FCE01CE
:1095100089569F4F0E94E816C956DF4F888199816E
:10952000C759D040845691090E944F3E80936905E7
:109530008823C1F00E94F015C956DF4F68817981F8
:10954000C759D040645671098DE293E10E94131609
:1095500067E472E085E293E10E944D168AE00E9482
:10956000721858C0C756DF4F28813981C959D04079
:10957000CB56DF4F88819981C559D04028173907CC
:10958000E9F0109369050E94F315CB56DF4F68810F
:109590007981C559D04085E093E10E944D16C756A8
:1095A000DF4F68817981C959D04080E093E10E9402
:1095B0004D1680EF92E10E94E2152CC08091680563
:1095C000811128C00E94F01507E313E0F801819192
:1095D0008F01882319F00E947218F8CFC956DF4F07
:1095E00068817981C759D0406456710983ED92E151
:1095F0000E941316C756DF4F48815981C959D04080
:1096000060E070E086EC92E10E94571683EC92E1F4
:109610000E94E21580916805811106C0809169055C
:10962000811102C00E94D23D80916805811101C064
:1096300013D80E9491169091690581E08927CD5534
:10964000DF4F28813981C35AD0400FB6F8943EBF0E
:109650000FBE2DBFCC55DF4F0FB6F894DEBF0FBE47
:10966000CDBFDF91CF911F910F91FF90EF90DF90D1
:10967000CF90BF90AF909F908F907F906F905F90B2
:109680004F903F902F90089581E0809368052CDAE9
:10969000109268050895F8DF811126CA0E94E941F9
:1096A00081E00895BF92CF92DF92EF92FF920F93E5
:1096B0001F93CF93DF93CDB7DEB728970FB6F894FB
:1096C000DEBF0FBECDBF9091E204981709F47AC0B7
:1096D000B82E882309F453C080E090E0A0EAB0E4FB
:1096E0008D839E83AF83B887C0906A05D0906B0549
:1096F000E0906C05F0906D0520E030E0A901C70115
:10970000B6010E946DAC87FF0CC0A701960160E016
:1097100070E080EA90E40E9493AB6D837E838F8338
:10972000988720E030E04FE153E46D817E818F81A6
:1097300098850E9470AE181644F480E090E0AFE186
:10974000B3E48D839E83AF83B88720915802309114
:10975000590240915A0250915B026D817E818F8146
:1097600098850E9470AE181654F419821A821B82D2
:109770001C82BE016F5F7F4FCE01059698D4609129
:1097800050027091510280915202909153022091A7
:10979000540230915502409156025091570219825D
:1097A0001A821B821C82E0905802F09059020091AC
:1097B0005A0210915B02FE0131966F01C4D38B2DCA
:1097C0000E94793080E028960FB6F894DEBF0FBE75
:1097D000CDBFDF91CF911F910F91FF90EF90DF9060
:1097E000CF90BF9008952F923F924F925F926F92C9
:1097F0007F928F929F92AF92BF92CF92DF92EF9221
:10980000FF920F931F93CF93DF93CDB7DEB7A0974F
:109810000FB6F894DEBF0FBECDBF1C017F8F6E8FD9
:10982000498F28A3DC018D909D90AD90BC90FB01E9
:10983000408051806280738022ED30E040EE50EC39
:10984000C301B201002309F43BC00E9470AE87FD42
:1098500035C227E030E04EE353E4C301B2010E9479
:109860006DAC18160CF42AC223EA31E040E450EC47
:10987000C501B4010E9470AE87FD20C227E030E030
:1098800042E253E4C501B4010E946DAC18160CF419
:1098900015C227E030E041E253E4C501B4010E9463
:1098A0006DAC18160CF40AC227E030E041E253E434
:1098B000C301B2010E946DAC18160CF4FFC124C0A4
:1098C0000E9470AE87FDFAC127E030E04EE353E41A
:1098D000C301B2010E946DAC18160CF4EFC123EA6B
:1098E00031E040E450ECC501B4010E9470AE87FD48
:1098F000E5C127E030E042E253E4C501B4010E9433
:109900006DAC18160CF4DAC1E0905802F0905902D0
:1099100000915A0210915B0280914C0290914D028D
:10992000A0914E02B0914F028A8F9B8FAC8FBD8F5A
:109930008091460290914702A0914802B09149025D
:1099400080934C0290934D02A0934E02B0934F022D
:1099500019821A821B821C82DE0111966D01A301FD
:109960009201C501B401EFD281E09CDE81113EC1BC
:109970008091910582FF11C020916A0530916B059D
:1099800040916C0550916D0560E070E080E890ECCE
:109990000E9493AB6B017C0106C0C12CD12C40E22C
:1099A000E42E41ECF42ECD8ADE8AEF8AF88E812CEB
:1099B000912CA12C31E4B32E898A9A8AAB8ABC8A75
:1099C000BE016F5E7F4FCE01459671D31091E604C4
:1099D0001092E60482E0FCD1D1D112FD05C060E016
:1099E00070E080EC9FE7BDC0409058025090590253
:1099F00060905A0270905B0289829A82AB82BC822C
:109A000020E030E040EA50E4C301B2010E9494AB90
:109A10006D837E838F8398878E010B5F1F4FBE01FE
:109A20006F5F7F4FC80143D3CD86DE86EF86F88A0D
:109A300080E090E0A0E8BFE389879A87AB87BC8786
:109A4000BE01675F7F4FCE010D9631D3F090E604E3
:109A50001092E60482E0BCD191D1F2FEC0CF809199
:109A60002D0C8F3F09F45BC0C0905802D090590272
:109A7000E0905A02F0905B02809058029090590258
:109A8000A0905A02B0905B0220E030E040E05FE33B
:109A9000C701B6010E9494AB9B01AC01C501B401A2
:109AA0000E946DAC87FF1CC01C991AC080E090E03A
:109AB000A0E8BFE389839A83AB83BC832AE037EDB8
:109AC00043EA5BE3C501B4010E9494AB6D837E83DE
:109AD0008F839887BE016F5F7F4FC801E8D2CCCFDC
:109AE000A7019601C501B4010E9493AB9B01AC0193
:109AF0006091360C7091370C8091380C9091390C34
:109B00000E9494AB6093360C7093370C8093380CA2
:109B10009093390C80912D0C8F5F80932D0C20E059
:109B200030E040E450E46091580270915902809115
:109B30005A0290915B020E94ABAE6B017C01A301C3
:109B40009201C301B2010E9494AB9B01AC01C70119
:109B5000B6010E9494AB2DEC3CEC4CE45EE30E9419
:109B6000ABAE20916A0530916B0540916C05509128
:109B70006D050E9494AB7B018C01898D82508230EF
:109B800048F580E090E0A0E0B1E489839A83AB835C
:109B9000BC83609158027091590280915A02909151
:109BA0005B02A98DA33029F020E030E040EA50E4C8
:109BB00004C020E030E048EC51E40E9494AB6D8397
:109BC0007E838F839887BE016F5F7F4FCE0105969E
:109BD0006ED207C0B98DB13021F480E063DD811110
:109BE00005C0E8A1E33008F449C008C098A193304B
:109BF00008F46DC0E12CF12C00EC1FE72BE3C22E22
:109C000023E0D22ED6018D916D01882319F00E9498
:109C10007218F8CFF101608171818281938143E0F4
:109C200050E00E94F01993E4C92E93E0D92ED6019A
:109C30008D916D01882319F00E947218F8CFEE8D76
:109C4000FF8D608171818281938143E050E00E94A9
:109C5000F01988E4C82E83E0D82ED6018D916D01CD
:109C6000882319F00E947218F8CF43E050E0B70142
:109C7000C8010E94F0198AE00E9472188A8D9B8D9B
:109C8000AC8DBD8D80934C0290934D02A0934E02FB
:109C9000B0934F029701A801B701C8010E9459AFC4
:109CA000882389F080E0FEDC0E94F3158EE993E1C1
:109CB0000E94E2152E2D7F2DC8011AC020E070E011
:109CC00080EC9FE715C02E2D7F2DC80111C08A8D15
:109CD0009B8DAC8DBD8D80934C0290934D02A093D3
:109CE0004E02B0934F02E12CF12C00EC1FE7DACFCB
:109CF000C22ED72E7C01C701B601A0960FB6F894EC
:109D0000DEBF0FBECDBFDF91CF911F910F91FF90AE
:109D1000EF90DF90CF90BF90AF909F908F907F900B
:109D20006F905F904F903F902F900895CF93DF9367
:109D3000C0E5D2E0488159816A817B8187E294E164
:109D40000E942D164C815D816E817F8183E294E1BA
:109D50000E942D16488559856A857B858FE194E19F
:109D60000E942D164C855D856E857F858BE194E183
:109D70000E942D16DF91CF910C94A83B2CE532E088
:109D800048E552E064E572E080E592E00C946E6A8A
:109D90008CE592E00C94BB6ACF93DF9380E00E9445
:109DA000885AC4E7D5E0688379838A839B8381E0FE
:109DB0000E94885A6C837D838E839F8382E00E94F9
:109DC000885A688779878A879B87DF91CF91089522
:109DD0001F93CF93DF93CDB7DEB760970FB6F8949C
:109DE000DEBF0FBECDBF182FD7DF809174059091D5
:109DF0007505A0917605B091770589839A83AB8329
:109E0000BC838091780590917905A0917A05B091F5
:109E10007B058D839E83AF83B88780917C0590916D
:109E20007D05A0917E05B0917F0589879A87AB87D4
:109E3000BC8780915C0290915D02A0915E02B0911E
:109E40005F028D879E87AF87B88BCE0101960E94F7
:109E5000CD591E3F51F480E1FE013196A0E5B2E0FC
:109E600001900D928A95E1F716C024E0129FC0017F
:109E70001124FC01E05BFD4FA1E0B0E0AC0FBD1F81
:109E8000A80FB91F8D919D910D90BC91A02D80833D
:109E90009183A283B38360960FB6F894DEBF0FBEA2
:109EA000CDBFDF91CF911F910895AF92BF92CF9216
:109EB000DF92EF920F931F93A12CB12C6501E12C3F
:109EC0008C012CE532E048E552E064E572E080E583
:109ED00092E00E9432691F910F91EF90DF90CF9036
:109EE000BF90AF900895AF92BF92CF92DF92EF9262
:109EF0000F931F93CF93DF9300D01F92CDB7DEB7A0
:109F000069837A838B839C83A12CB12C6501E12C1E
:109F10008E010F5F1F4F2CE835E048E855E064E8FC
:109F200075E080E895E00E9432690F900F900F90E5
:109F30000F90DF91CF911F910F91EF90DF90CF9015
:109F4000BF90AF9008954F925F926F927F928F92E1
:109F50009F92AF92BF92CF92DF92EF92FF920F93B8
:109F60001F93CF93DF93CDB7DEB72C970FB6F8943E
:109F7000DEBF0FBECDBF2B013C0129873A874B873F
:109F80005C8747015801F601E080F180028113816E
:109F900020E030E0A901B701C8010E946DAC811139
:109FA00007C0E2E3F4E185919591A591B49102C0D7
:109FB000C701D8018D839E83AF83B88720E030E04E
:109FC000A901B701C8010E946DAC811108C0E090E1
:109FD0004602F09047020091480210914902C701E1
:109FE000D80189839A83AB83BC83A50194016091D6
:109FF00058027091590280915A0290915B020E941E
:10A000006DAC87FF0BC08092580290925902A092CB
:10A010005A02B0925B02CE01059647DF4092500291
:10A0200050925102609252027092530289859A8531
:10A03000AB85BC858093540290935502A093560241
:10A04000B0935702CE01019630DFA50194016091D3
:10A0500058027091590280915A0290915B020E94BD
:10A0600070AE18165CF48092580290925902A09239
:10A070005A02B0925B02CE01059617DF0E949C5AED
:10A080002C960FB6F894DEBF0FBECDBFDF91CF91F7
:10A090001F910F91FF90EF90DF90CF90BF90AF9006
:10A0A0009F908F907F906F905F904F900895CF9288
:10A0B000DF92EF92FF920F931F936B01FC01E08000
:10A0C000F18002811381E0E5F2E02481358146814F
:10A0D0005781608171818281938135DF1F910F915A
:10A0E000FF90EF90DF90CF900895CF92DF92EF92A4
:10A0F000FF920F931F936A01E0905802F09059026B
:10A1000000915A0210915B02FB0120813181428152
:10A110005381FC01608171818281938114DF1F91E1
:10A120000F91FF90EF90DF90CF90089580914C02B7
:10A1300090914D02A0914E02B0914F028093700514
:10A1400090937105A0937205B093730580914A02B4
:10A1500090914B0290936F0580936E0584E690E09A
:10A1600090934B0280934A020895809170059091DC
:10A170007105A0917205B091730580934C02909384
:10A180004D02A0934E02B0934F0280916E059091C4
:10A190006F0590934B0280934A02089524E0829FBA
:10A1A000C0011124FC01E759FB4E45915591659181
:10A1B0007491FC01E75CFD4F40835183628373839C
:10A1C000FC01E35AFB4E4591559165917491FC0158
:10A1D000E35DFD4F40835183628373830895CF9283
:10A1E000DF92EF92FF92CF93DF93209145022223DB
:10A1F00009F443C0EC01C0902D02D0902E02E090F3
:10A200002F02F0903002A7019601688179818A813E
:10A210009B810E9470AE181624F4C882D982EA820B
:10A22000FB82C0903102D0903202E0903302F09075
:10A230003402A70196016C817D818E819F810E94ED
:10A2400070AE181624F4CC82DD82EE82FF82C090BC
:10A250003502D0903602E0903702F0903802A70124
:10A260009601688579858A859B850E9470AE18164F
:10A2700024F4C886D986EA86FB86DF91CF91FF90C9
:10A28000EF90DF90CF9008958F929F92AF92BF9200
:10A29000CF92DF92EF92FF9280E895E0A0DF80916D
:10A2A000A90383FD7DC0C0908C05D0908D05E09002
:10A2B0008E05F0908F0520915C0230915D024091F7
:10A2C0005E0250915F02C701B6010E946DAC882307
:10A2D00009F466C06091CC047091CD048091CE04E5
:10A2E0009091CF042091A104211117C00E94DCACF1
:10A2F00020911D0230911E026217730774F4C09200
:10A300005C02D0925D02E0925E02F0925F020E94D7
:10A31000F01580E094E10E94E21580908C05909009
:10A320008D05A0908E05B0908F0520915C02309134
:10A330005D0240915E0250915F02C501B4010E942E
:10A3400093AB6B017C0120E030E0A9010E9470AE6C
:10A3500087FF04C0C701B601905802C0C701B6010B
:10A36000209160023091610240916202509163023B
:10A370000E94ABAE20E030E048E453E40E9470AEAF
:10A38000181674F480925C0290925D02A0925E02B4
:10A39000B0925F020E94F01581EE93E10E94E215F7
:10A3A00060914A0270914B02072E000C880B990BAA
:10A3B0000E940FAD20914C0230914D0240914E020F
:10A3C00050914F020E94ABAE2AE037ED43E25CE3CE
:10A3D0000E94ABAE88DD80E1E0E8F5E0A0E5B2E008
:10A3E00001900D928A95E1F7FF90EF90DF90CF906A
:10A3F000BF90AF909F908F9008951F93CF93DF935E
:10A40000882329F0D0919205D095D17001C0D0E079
:10A41000662339F0109192051695117081E0182786
:10A4200001C010E0442341F0C0919205C2FBCC274B
:10A43000C0F981E0C82701C0C0E0D11104C01111EA
:10A4400002C0CC23D1F00E94F0158BED93E10E9465
:10A45000E215DD2319F088E50E947218112319F026
:10A4600089E50E947218CC2319F08AE50E947218BF
:10A4700083ED93E10E94E215C1E08C2FDF91CF9133
:10A480001F910895CF92DF92EF92FF92CF93DF93C7
:10A49000C82FD0E0FE01E053FC4E8491811107C02B
:10A4A0000E94F0158EEA93E10E94E2158AE0FE0117
:10A4B000EE0FFF1FEE0FFF1FE65DFB4EC590D59020
:10A4C000E590F490682F70E080E090E00E940FAD7E
:10A4D0009B01AC01C701B6010E9474ACDF91CF9122
:10A4E000FF90EF90DF90CF9008954F925F926F9220
:10A4F0007F928F929F92AF92BF92CF92DF92EF9214
:10A50000FF920F931F93CF93DF93CDB7DEB768977A
:10A510000FB6F894DEBF0FBECDBF2A013B01690123
:10A52000E82EF12CF701EA5CFB4EE491AA24A394F7
:10A530001E160CF4A12CBB24B39420E030E0A9013A
:10A54000C301B2010E9470AE18160CF0B12C80E06D
:10A55000DFD769837A838B839C8381E0D9D76D832E
:10A560007E838F83988782E0D3D769877A878B87AA
:10A570009C8783E0CDD76D877E878F87988BEE0C85
:10A58000FF1CEE0CFF1C88248394912C8C0E9D1EC6
:10A590008E0C9F1CF40110821182128213829E0184
:10A5A000235F3F4FAE01475F5F4FBE016B5F7F4F41
:10A5B000CE0101960E949369F40140825182628229
:10A5C0007382198A1A8A1B8A1C8A20E030E0A9014A
:10A5D000B801C6010E946DAC811108C0F701E65DAB
:10A5E000FB4E85919591A591B49102C0C801D60109
:10A5F0008D8B9E8BAF8BB88FCE0141966C01E12C79
:10A600008E010B5E1F4F9E01235F3F4FAE01475FE0
:10A610005F4FBE016B5F7F4F40970E944F688CD7A2
:10A62000AB100E943D3068960FB6F894DEBF0FBEA7
:10A63000CDBFDF91CF911F910F91FF90EF90DF90F1
:10A64000CF90BF90AF909F908F907F906F905F90D2
:10A650004F90089521E030E0082E01C0220F0A94A7
:10A66000EAF790919105922B909391059091920524
:10A67000292B2093920524E0829FC0011124FC0124
:10A68000EF5AFB4E4591559165917491FC01E05B49
:10A69000FD4F408351836283738308954F925F928D
:10A6A0006F927F928F929F92AF92BF92FF920F9381
:10A6B0001F93CF93DF93833008F06AC0F82EC82F22
:10A6C000D0E0FE01EA5CFB4E8491CC0FDD1FCC0F85
:10A6D000DD1FFE01EB5BFB4E45905590659074903D
:10A6E000682F880F770B880B990B0E940FAD4B01D9
:10A6F0005C0120E030E040EC5FE3C301B2010E9466
:10A70000ABAEA50194010E94ABAEAB01BC0100E071
:10A7100010E098018F2DE9DEFE01E75CFB4E2591EC
:10A72000359145915491C501B4010E94ABAE4B01E6
:10A730005C0120E030E0A9010E946DAC8823C1F0EB
:10A74000B501A401705800E010E098018F2DCDDE16
:10A750008F2D98DE2B013C01A5019401C501B401A8
:10A760000E9494ABAB01BC01930182018F2DBDDE31
:10A770008F2D70DF03DBFE01E058FA4FC05BDD4F29
:10A7800088819981AA81BB8180839183A283B383CD
:10A79000DF91CF911F910F91FF90BF90AF909F904D
:10A7A0008F907F906F905F904F90089580E1E5EDDE
:10A7B000F5E0DF01982F1D929A95E9F7E8EAF5E0B8
:10A7C000DF01982F1D929A95E9F7E1ECF5E0DF01A2
:10A7D0001D928A95E9F71092BD051092BE05109260
:10A7E000BF051092C00581EF95E00E942DA5109243
:10A7F000910610929406109292061092930610926F
:10A800008E0608954F925F926F927F928F929F92E1
:10A81000AF92BF92CF92DF92EF92FF920F931F936E
:10A82000CF93DF93CDB7DEB768970FB6F894DEBF4E
:10A830000FBECDBF8C015B014A01FC01EF5BFF4FF6
:10A8400060817181828193810E940DAD6B017C01D9
:10A85000D5012D913D914D915C910E94ABAE0E942E
:10A860005AAC0E94E1AC69877A878B879C87F40198
:10A870002081318142815381C701B6010E94ABAE74
:10A880000E945AAC0E94E1AC6D877E878F87988BBF
:10A8900029853A854B855C85283731054105510569
:10A8A00040F488E790E0A0E0B0E089879A87AB8722
:10A8B000BC872D853E854F85588928373105410550
:10A8C000510540F488E790E0A0E0B0E08D879E87D6
:10A8D000AF87B88B9801235B3F4FD9018D919D9134
:10A8E0000D90BC91A02D89839A83AB83BC83BC015E
:10A8F000CD010E940FAD2B013C0169857A858B85C6
:10A900009C850E940DAD698B7A8B8B8B9C8B20E094
:10A9100030E0A901C301B2010E946DAC882329F186
:10A92000A7019601C701B6010E94ABAE4B015C01C5
:10A9300029893A894B895C89CA01B9010E94ABAE69
:10A940009B01AC01C501B4010E9493AB4B015C01BA
:10A95000A3019201C301B2010E9494AB9B01AC011F
:10A96000C501B4010E9474AC03C060E070E0CB018B
:10A970000E945AAC0E94E1AC6D837E838F839887DE
:10A9800069817A818B819C81909580957095619584
:10A990007F4F8F4F9F4F0E940FAD4B015C016D8524
:10A9A0007E858F8598890E940DAD69837A838B831C
:10A9B0009C8320E030E0A901C501B4010E946DAC88
:10A9C000882349F129813A814B815C81CA01B9010F
:10A9D0000E94ABAE6D8B7E8B8F8B988FA7019601FB
:10A9E000C701B6010E94ABAE9B01AC016D897E89A7
:10A9F0008F89988D0E9493AB6B017C01A501940116
:10AA0000C501B4010E9494AB9B01AC01C701B60122
:10AA10000E9474AC03C060E070E0CB010E944AADBC
:10AA2000F80185A096A0A7A0B0A4750164012D81AE
:10AA30003E814F815885C21AD30AE40AF50A0E9462
:10AA4000E1ACC61AD70AE80AF90AF7FE73C020E09B
:10AA500030E0A901C301B2010E946DAC882309F462
:10AA600043C0A3019201C301B2010E9494AB6B01E8
:10AA70007C01C501B4010E940DAD9B01AC01C70171
:10AA8000B6010E94ABAE6B017C0129893A894B89E2
:10AA90005C89CA01B9010E94ABAE9B01AC01C70140
:10AAA000B6010E9493AB6B017C0129813A814B81F5
:10AAB0005C81CA01B9010E94ABAE9B01AC01C70128
:10AAC000B6010E9494AB6B017C0120E030E040E8CD
:10AAD00050E4C301B2010E94ABAE9B01AC01C701BF
:10AAE000B6010E9474AC03C060E070E0CB010E942C
:10AAF0005AAC7B016C0120E030E0A9010E9470AEED
:10AB0000181624F0E12CF12CC12CD12CB701C60170
:10AB10000E94E1AC6D837E838F83988786169706AB
:10AB2000A806B90620F48D829E82AF82B886C12C19
:10AB3000D12C76018D819E81AF81B885F80181A7E6
:10AB400092A7A3A7B4A7C80ED91EEA1EFB1EC5A6CE
:10AB5000D6A6E7A6F0AAEB5BFF4F29853A854B8581
:10AB60005C85208331834283538334968D859E8513
:10AB7000AF85B88980839183A283B38368960FB62B
:10AB8000F894DEBF0FBECDBFDF91CF911F910F9123
:10AB9000FF90EF90DF90CF90BF90AF909F908F90FD
:10ABA0007F906F905F904F9008952F923F924F92B9
:10ABB0005F926F927F928F929F92AF92BF92CF924D
:10ABC000DF92EF92FF920F931F93CF93DF93009743
:10ABD00009F471C08B01EC01D984CA847B846C8434
:10ABE0008D809E80AF80B8842D2D3C2D472D562D15
:10ABF000C501B4010E946DAC811108C00115110599
:10AC000009F459C0F801808180FF55C0888181FD19
:10AC100034C00115110531F0F801258036804780D8
:10AC2000508408C08BE0282E87ED382E83E2482E12
:10AC30008BE3582E89899A89AB89BC89BC01CD01E7
:10AC400090589B01AC010E9494AB2D853E854F85A9
:10AC500058890E94ABAE9B01AC01C201B1010E94B8
:10AC600093AB7B018C019B01AC016D2D7C2D872D5D
:10AC7000962D0E946DAC87FF04C0ED2CFC2C072D97
:10AC8000162D9701A801C501B4010E946DAC88235F
:10AC900091F0888181608883CE010E9432358823BB
:10ACA00021F088818E7F888306C0A701B8014D837B
:10ACB0005E836F837887DF91CF911F910F91FF9013
:10ACC000EF90DF90CF90BF90AF909F908F907F904C
:10ACD0006F905F904F903F902F900895FF920F9349
:10ACE0001F93CF93DF93C0919406C150CF70D09142
:10ACF000920680919406D817E9F060E070E086E54E
:10AD0000F82ECD17B9F0FC9E800111240B56194F77
:10AD1000F801808183FD03C0C80147DFB801C1503D
:10AD2000CF7080919206D81761F3CD1719F0DF5FCD
:10AD3000DF70F7CFDF91CF911F910F91FF900895B2
:10AD40004F925F926F927F928F929F92AF92BF923B
:10AD5000FF920F931F93CF93DF93009709F459C08D
:10AD6000F42EEB018C01FC01808181FD3CC045800B
:10AD70005680678070848D809E80AF80B884A501E6
:10AD80009401C301B2010E946DAC87FF2CC0F80191
:10AD900081899289A389B489BC01CD0190589B0116
:10ADA000AC010E9494ABF801258536854785508912
:10ADB0000E94ABAE9B01AC01C301B2010E9493ABF8
:10ADC0002B013C01A50194010E946DAC87FF0BC0D3
:10ADD000888181608883CE010E943235882391F07A
:10ADE00088818E7F888329853A854B855C856D8136
:10ADF0007E818F8198850E946DAC81110AC0F0928E
:10AE0000920607C04D825E826F827886F09292062B
:10AE1000EACFDF91CF911F910F91FF90BF90AF903C
:10AE20009F908F907F906F905F904F900895CF92FA
:10AE3000DF92EF92FF920F931F93CF93DF931091C6
:10AE40009206C0E0D0E086E5C82E809194061817DF
:10AE500009F1C19EB0011124CB018B56994F7C01A1
:10AE6000FC01808183FD0AC00E2DDF2C209769F044
:10AE7000CE010E943235882341F002C00C2FDD2E16
:10AE80001F5F1F70C02FDD2DE0CF412FB701CE0116
:10AE900057DFF6CFDF91CF911F910F91FF90EF9089
:10AEA000DF90CF9008952F923F924F925F926F92D2
:10AEB0007F928F929F92AF92BF92CF92DF92EF924A
:10AEC000FF920F931F93CF93DF93CDB7DEB72E97EB
:10AED0000FB6F894DEBF0FBECDBF20919106298733
:10AEE000309194063B8796E58B85E9858E1759F05E
:10AEF0008B8581508F70989FF0011124EB56F94F8C
:10AF0000208123FD0DC0812C912CA12CB12C1A86FF
:10AF10001C861D861E86212C312C00E010E01AC0F4
:10AF20008B87E2CFF6E52985F29FC0011124FC0151
:10AF3000EB56F94F1F01808183FF11C0FA84EC8426
:10AF4000DD84CE8489858F5F8F708987FA86EC8651
:10AF5000DD86CE86F9852B85F213E4CF93C065811B
:10AF60007681878190850E9418AFF62EE72ED82E25
:10AF7000C92E0115110509F47FC0F801808180FDFB
:10AF800004C0F101808180FF77C0F8018081816079
:10AF90008083C8010E94323581116AC0F801618145
:10AFA0007281838194810E9418AF2B013C019B0127
:10AFB000AC0160E070E080E89FE30E9474AC4B015C
:10AFC0005C019B01AC016F2D7E2D8D2D9C2D0E946F
:10AFD000ABAE69837A838B839C83A50194016A85D8
:10AFE0007C858D859E850E94ABAE6D837E838F832D
:10AFF0009887AE014F5F5F4FBE016B5F7F4FC80107
:10B0000001DCF80186A9882399F12091B8053091D7
:10B01000B9054091BA055091BB05FD9660817181DB
:10B02000828193810E94ABAE2091660630916706C3
:10B0300040916806509169060E94ABAE4B015C01DD
:10B040009B01AC01C301B2010E94ABAE0E94E1AC16
:10B05000F80172AF61AFA50194016F2D7E2D8D2D8A
:10B060009C2D0E94ABAE0E94E1ACF80174AF63AFBF
:10B07000F80180818E7F80838F2C9E2CAD2CBC2C80
:10B08000810160CF2114310409F473C0F101808182
:10B0900081608083C8010E943235811166C0F10150
:10B0A00061817281838194810E9418AF6B017C0160
:10B0B0009B01AC0160E070E080E89FE30E9474AC0B
:10B0C0002B013C012DEC3CEC4CE45DE30E94ABAE6B
:10B0D00069837A838B839C83A3019201B401C501A8
:10B0E0000E94ABAE6D837E838F839887AE014F5FE6
:10B0F0005F4FBE016B5F7F4FC10184DBF10186A909
:10B10000882399F12091B8053091B9054091BA058D
:10B110005091BB05FD9660817181828193810E946F
:10B12000ABAE20916606309167064091680650915B
:10B1300069060E94ABAE4B015C019B01AC01C701EB
:10B14000B6010E94ABAE0E94E1ACF10172AF61AFFB
:10B150002DEC3CEC4CE45DE3C501B4010E94ABAEC8
:10B160000E94E1ACF10174AF63AFF10180818E7F89
:10B1700080832E960FB6F894DEBF0FBECDBFDF9151
:10B18000CF911F910F91FF90EF90DF90CF90BF90E4
:10B19000AF909F908F907F906F905F904F903F9077
:10B1A0002F900895809194069091920681508F700F
:10B1B000891711F093DD3BDE76CEAF92BF92CF922E
:10B1C000DF92EF92FF920F931F93CF93909194068B
:10B1D00080919106981791F0E091910686E5E89F9D
:10B1E000F0011124EA51F94FC081809191069091AC
:10B1F0009406891729F08F5F8F70F9CFC091C7042B
:10B20000CC2339F10E9465110091A4051091A50588
:10B210002091A6053091A705DC01CB010115110590
:10B220002105310571F48C599F4FAF4FBF4F80936B
:10B23000A4059093A505A093A605B093A705CFEF0D
:10B2400021C0801B910BA20BB30BB7FF1BC0CFEF2C
:10B2500019C01092A4051092A5051092A60510928F
:10B26000A70560E070E020E04FEF50E088E0CF916C
:10B270001F910F91FF90EF90DF90CF90BF90AF9014
:10B280000C9435226C2F70E080E090E01F921F92AA
:10B290001F922FEF2F9326E4A22EB12CC12CD12C7C
:10B2A000E12CF12C8701EA9421E030E040E050E00D
:10B2B0000E943B150F900F900F900F90D4CFCF921C
:10B2C000DF92EF92FF920F931F93CF93DF93CDB74F
:10B2D000DEB728970FB6F894DEBF0FBECDBF209122
:10B2E0001506222309F44AC06A018B017C0120E083
:10B2F00030E040E450E4FC016081718182819381FF
:10B300000E9494AB6D837E838F83988720E030E02A
:10B310004EE353E4F80160817181828193810E9440
:10B3200093AB69837A838B839C839601AE014F5FD5
:10B330005F4FBE016B5F7F4F81EF95E00E9465A478
:10B3400020E030E040E450E46D817E818F8198857B
:10B350000E9493ABF701608371838283938320E023
:10B3600030E04EE353E469817A818B819C810E94B5
:10B3700094ABF801608371838283938328960FB620
:10B38000F894DEBF0FBECDBFDF91CF911F910F911B
:10B39000FF90EF90DF90CF9008950F931F93CF937E
:10B3A000DF93CDB7DEB7AC970FB6F894DEBF0FBE14
:10B3B000CDBF20911506222309F450C08C0161EF06
:10B3C00075E0CE0101960E94E8A520E030E040E45F
:10B3D00050E4F80160817181828193810E9494AB75
:10B3E00069A77AA78BA79CA720E030E04EE353E43F
:10B3F000F80164817581868197810E9493AB6DA36A
:10B400007EA38FA398A79801285F3F4FAE014B5DA5
:10B410005F4FBE01675D7F4FCE0101960E9465A41C
:10B4200020E030E040E450E469A57AA58BA59CA516
:10B430000E9493ABF801608371838283938320E041
:10B4400030E04EE353E46DA17EA18FA198A50E9448
:10B4500094ABF8016483758386839783AC960FB6AB
:10B46000F894DEBF0FBECDBFDF91CF911F910F913A
:10B47000089580916F0081FB992790F981FF05C0A5
:10B4800080916F008D7F80936F00809191068093F3
:10B490009406809392068093930684E680938E06AA
:10B4A00028EE33E03093900620938F06992329F0FD
:10B4B00080916F00826080936F0081E080935605D9
:10B4C00008950C94613BCF93C82F0E948A3B0E9441
:10B4D0000FAD24E0C29FF0011124EA5DF94F2081F5
:10B4E0003181428153810E94ABAECF9108959091FA
:10B4F000940680919106981719F00E94FBAAF7CF45
:10B5000080918F0690919006892BB9F70C94D2A95F
:10B51000CF93C82F0E94433B0E940FAD24E0C29FEF
:10B52000F0011124EA5DF94F20813181428153817C
:10B530000E94ABAECF9108959091940680919106B0
:10B54000981719F00E94FBAAF7CF80918F0690916F
:10B550009006892BB9F708952F923F924F925F92F0
:10B560006F927F928F929F92AF92BF92CF92DF9213
:10B57000EF92FF920F931F93CF93DF93CDB7DEB778
:10B5800066970FB6F894DEBF0FBECDBFB88AAF8600
:10B59000E091A305DC2CDE26672B682B692B19F4C0
:10B5A0008D2D8E7FD82E232B242B252B19F49D2D0A
:10B5B0009D7FD92EEF28E02AE12A19F4AD2DAB7F2B
:10B5C000DA2E8D2D8E278093A30580913A0C9091D1
:10B5D0003B0CA0913C0CB0913D0C8D839E83AF83BE
:10B5E000B88720E030E0A901BC01CD010E946DAC1C
:10B5F000882309F424C18091670290916802A09188
:10B600006902B0916A0289879A87AB87BC87AEE3EB
:10B61000BCE0BE87AD87EF85F889FA83E98387E9C7
:10B6200095E09E8B8D8BA6E4B6E0BC83AB83212C8A
:10B63000312C812C912C5401EC2DF0E0FA8BE98B0C
:10B640008D2D90E09C8B8B8BAD85BE85CD90DD9054
:10B65000ED90FD90BE87AD8720E030E0A901C701E5
:10B66000B6010E946DAC882309F4D2C009891A89F9
:10B67000022C02C0159507950A94E2F70170112774
:10B680008B899C89022C02C0959587950A94E2F7D4
:10B6900080FF38C0ED89FE8960817181828193814C
:10B6A0000E940FAD2B013C010115110529F420E08A
:10B6B00030E040E85FE304C020E030E040E85FEBCA
:10B6C0006D817E818F8198850E94ABAEA701960126
:10B6D0000E94ABAEAB81BC8154962D913D914D91B2
:10B6E0005C9157970E94ABAE9B01AC01C301B201C4
:10B6F0000E9494AB0E94DCACED89FE89608371836B
:10B7000082839383AD89BE89CD90DD90ED90FC90CE
:10B71000C114D104E104F10409F47AC020E030E05E
:10B72000A90169857A858B859C850E946DAC8823EB
:10B7300009F445C0D701C6018827B7FD839599272D
:10B74000AA27BB270817190709F062C020E030E0DC
:10B75000A901C501B4010E946DAC81111CC02985ED
:10B760003A854B855C85EF85F88965857685878583
:10B7700090890E9474AC4B015C0120E030E040E80D
:10B780005FE30E9470AE181634F4812C912C80E88F
:10B79000A82E8FE3B82EC701B6010E940FAD9B0102
:10B7A000AC01C501B4010E94ABAE0E945AAC0E942C
:10B7B000DCAC611571058105910519F429C0C7013B
:10B7C000B6018B019C0197FF07C000271127980144
:10B7D000061B170B280B390BA981BA8155964D9082
:10B7E0005D906D907C905897040D151D261D371D9A
:10B7F000FD01058B168B278B308FC61AD70AE80AF6
:10B80000F90AAD89BE89CD92DD92ED92FC92139733
:10B81000BFEF2B1A3B0AE981FA813496FA83E98358
:10B820008D899E8904969E8B8D8BAB81BC811496ED
:10B83000BC83AB83B3E02B16310409F005CF6696C9
:10B840000FB6F894DEBF0FBECDBFDF91CF911F9131
:10B850000F91FF90EF90DF90CF90BF90AF909F90AF
:10B860008F907F906F905F904F903F902F900895B2
:10B870002F923F924F925F926F927F928F929F9200
:10B88000AF92BF92CF92DF92EF92FF920F931F93EE
:10B89000CF93DF93CDB7DEB7C756D1090FB6F89473
:10B8A000DEBF0FBECDBF1C01A4966FAFA4976F96ED
:10B8B0005FAF4EAF6F9769963FAF2EAF69972896EF
:10B8C000EFAE2897FFAE60960FAF609764961FAFFC
:10B8D0006497CFAAA196BFAEAEAEA197DA014D9103
:10B8E0005D916D917C918091D5059091D605A09147
:10B8F000D705B091D8058A019B01081B190B2A0BAB
:10B900003B0B0BA31CA32DA33EA36F96AEADBFAD07
:10B910006F9714964D915D916D917C9117978091E1
:10B92000D9059091DA05A091DB05B091DC058A017B
:10B930009B01081B190B2A0B3B0B0FA318A729A768
:10B940003AA76F96AEADBFAD6F9718964D915D91CA
:10B950006D917C911B978091DD059091DE05A09102
:10B96000DF05B091E0058A019B01081B190B2A0B2A
:10B970003B0B0FA718AB29AB3AAB6F96AEADBFAD83
:10B980006F971C96CD90DD90ED90FC901F97809165
:10B99000E1059091E205A091E305B091E40526014F
:10B9A0003701481A590A6A0A7B0A09F497C060915C
:10B9B000CC047091CD048091CE049091CF0420915D
:10B9C000A10421112AC00E94DCAC20911D023091FB
:10B9D0001E02621773070CF5C092E105D092E205D2
:10B9E000E092E305F092E4056996EEADFFAD69974C
:10B9F00084859585A685B7858093B4059093B50514
:10BA0000A093B605B093B7050E94F01584E994E1C0
:10BA10000E94E215412C512C3201C301B2010E9457
:10BA20000FAD1FA904E0109FF0011124E05AFD4F53
:10BA300020813181428153810E94ABAE6B017C0138
:10BA400020E030E0A9010E9470AE87FF04C0F7FA41
:10BA5000F094F7F8F0946091660670916706809113
:10BA60006806909169060E94DCAC9B01AC01A8ECD1
:10BA7000B0E00E94F3AF0E940FAD9B01AC01C70183
:10BA8000B6010E9470AE18164CF56F96EEADFFAD84
:10BA90006F9784859585A685B7858093E1059093FA
:10BAA000E205A093E305B093E4056996EEADFFAD22
:10BAB000699784859585A685B7858093B40590930D
:10BAC000B505A093B605B093B7050E94F01585E7BC
:10BAD00094E10E94E215412C512C32018BA19CA1D2
:10BAE000ADA1BEA18827B7FD83959927AA27BB27BB
:10BAF000182F2FA138A549A55AA557FD12608FA56B
:10BB000098A9A9A9BAA9B7FD146077FC1860C30168
:10BB1000B2010E940FADBFA9A4E0BA9FF0011124A9
:10BB2000E05AFD4F20813181428153810E94ABAEAA
:10BB30004B015C0120E030E0A9010E9470AE87FF5C
:10BB400004C0C501B401905802C0C501B40120E091
:10BB500030E040E05FE30E9494AB0E94E1AC6BAF49
:10BB60007CAF8DAF9EAFF101108215AB2BA13CA134
:10BB70004DA15EA12BA73CA74DA75EA757FF0BC009
:10BB800050954095309521953F4F4F4F5F4F2BA7D4
:10BB90003CA74DA75EA78BA59CA5ADA5BEA5F101B1
:10BBA000858B968BA78BB08F2FA138A549A55AA559
:10BBB0002BAB3CAB4DAB5EAB57FF0BC050954095EC
:10BBC000309521953F4F4F4F5F4F2BAB3CAB4DAB6B
:10BBD0005EAB8BA99CA9ADA9BEA9F101818F928F03
:10BBE000A38FB48F2FA538A949A95AA92F962CAF96
:10BBF0003DAF4EAF5FAF2F9757FF0DC050954095AB
:10BC0000309521953F4F4F4F5F4F2F962CAF3DAF53
:10BC10004EAF5FAF2F972F968CAD9DADAEADBFAD44
:10BC20002F97F101858F968FA78FB0A36BA17CA171
:10BC30008DA19EA10E940FAD20912606309127066E
:10BC400040912806509129060E94ABAE27966CAF12
:10BC50007DAF8EAF9FAF2797698B7A8B8B8B9C8B39
:10BC60006FA178A589A59AA50E940FAD20912A06FB
:10BC700030912B0640912C0650912D060E94ABAEC0
:10BC80006B017C016D8B7E8B8F8B988F6FA578A954
:10BC900089A99AA90E940FAD20912E0630912F06F6
:10BCA00040913006509131060E94ABAE6D966CAF5C
:10BCB0007DAF8EAF9FAF6D97698F7A8F8B8F9C8F83
:10BCC000209132063091330640913406509135066A
:10BCD000C501B4010E94ABAE4B015C016D8F7E8F3C
:10BCE0008F8F98A32BA53CA54DA55EA526303105C9
:10BCF0004105510544F58BA99CA9ADA9BEA906979C
:10BD0000A105B10504F52F962CAD3DAD4EAD5FAD4F
:10BD10002F972630310541055105ACF420E030E085
:10BD2000A901C501B4010E9470AE87FF04C0B7FA33
:10BD3000B094B7F8B094D1011D968D929D92AD92BA
:10BD4000BC92509759C0A196EEADFFADA1978080EF
:10BD50009180A280B38020E030E0A901C501B40148
:10BD60000E946DAC882341F0D1011D968D929D9269
:10BD7000AD92BC92509731C027962CAD3DAD4EADE3
:10BD80005FAD2797CA01B9010E94ABAE4B015C01C0
:10BD9000A7019601C701B6010E94ABAE9B01AC01A1
:10BDA000C501B4010E9494AB4B015C016D962CADB2
:10BDB0003DAD4EAD5FAD6D97CA01B9010E94ABAE0E
:10BDC0009B01AC01C501B4010E9494AB0E9418AF65
:10BDD000F101658776878787908B5101C12EEFA48B
:10BDE000F8A809A91AA92FA138A549A55AA56BA198
:10BDF0007CA18DA19EA1B0DB0BAD1CAD2DAD3EADE8
:10BE0000D10191960D931D932D933C939497559644
:10BE10004D915D916D917C9158975D960D911D911D
:10BE20002D913C91909759968D919D910D90BC913B
:10BE3000A02D80179107A207B30710F4D901C801FC
:10BE400084179507A607B70710F4DB01CA010BADED
:10BE50001CAD2DAD3EAD80179107A207B30710F4BE
:10BE6000D901C801F10185A396A3A7A3B0A706979E
:10BE7000A105B105A8F18091C704EF5AFF4F808357
:10BE8000452B462B472B09F01798F101818D928D98
:10BE9000A38DB48D892B8A2B8B2B09F01698F10179
:10BEA000858D968DA78DB0A1892B8A2B8B2B09F0C0
:10BEB00015980BAD1CAD2DAD3EAD012B022B032B08
:10BEC000D1F08091BC05882319F081508093BC0586
:10BED0001FA9111107C0149880E28093BC0502C00D
:10BEE00080E0FEC7E0908606F09087060091880605
:10BEF0001091890608C0E0908A06F0908B060091A8
:10BF00008C0610918D069701A80128966FAD289791
:10BF10007FAD60968FAD609764969FAD64970E94E9
:10BF20006DAC87FFD2C7D1011D962D913D914D91EA
:10BF30005C9150976D962CAF3DAF4EAF5FAF6D9754
:10BF400060E070E080E89FE30E9474AC2B966CAFD9
:10BF50007DAF8EAF9FAF2B979B01AC01B701C8019E
:10BF60000E94ABAE4B015C018091940690919306C8
:10BF7000891B8F7024968FAF2497A501940160E0F0
:10BF800074E284E799E40E9474AC0E947BAE6B017A
:10BF90007C0124968FAD249782508630C0F5809125
:10BFA000560690915706A0915806B0915906C816AA
:10BFB000D906EA06FB0658F58C199D09AE09BF099A
:10BFC000BC01CD01660F771F881F991F2496BFAD56
:10BFD00024970B2F10E020E030E0A90198010E9487
:10BFE00098AFCA01B9010E940DAD0E947BAE6C0DE5
:10BFF0007D1D8E1D9F1D0E940DAD9B01AC0160E05B
:10C0000074E284E799E40E9474AC4B015C01A501E1
:10C0100094016D966CAD7DAD8EAD9FAD6D970E9418
:10C02000ABAE9B01AC010E94ABAE23966CAF7DAF73
:10C030008EAF9FAF2397F1016183728383839483D3
:10C0400005A116A127A130A50FA718AB29AB3AABC4
:10C05000C901B8010E940DAD6FAB78AF89AF9AAF3F
:10C06000A50194010E94ABAE0E945AAC0E94E1ACC3
:10C0700063966CAF7DAF8EAF9FAF6397F101EF5BBF
:10C08000FF4F60837183828393838E010F5E1F4F06
:10C090001CA70BA7005111092D961FAF0EAF2D97AE
:10C0A0000AE616E0A1961FAF0EAFA1978E010F5DB5
:10C0B0001F4F1AA309A32D960EAD1FAD2D971CABD4
:10C0C0000BAB1BA21FA200E81FE3ABA5BCA56D91A3
:10C0D0007D918D919D91BCA7ABA7A50194010E9474
:10C0E000ABAE6B017C01EBA9FCA9619371938193C9
:10C0F0009193FCABEBAB20E030E0A9010E9470AE65
:10C1000087FF04C0F7FAF094F7F8F094A196AEAD6B
:10C11000BFADA1972D913D914D915D91A196BFAF7E
:10C12000AEAFA19767962CAF3DAF4EAF5FAF6797AD
:10C13000C701B6010E9470AE1816C4F4A70196019B
:10C1400067966CAD7DAD8EAD9FAD67970E9474AC68
:10C150006B017C019B01AC016BA17FA1C8010E9416
:10C1600070AE18161CF4CBA2DFA28701EBA5FCA5CC
:10C1700029A13AA1E217F30709F0A7CF20E030E0A8
:10C1800040E85FE36BA17FA1C8010E946DAC87FF0F
:10C190004BC06E0131E1C30ED11C2D96EEACFFAC4D
:10C1A0002D972BA13FA1A801D7016D917D918D9174
:10C1B0009C910E94ABAEF70161937193819391932F
:10C1C0007F01EC15FD0569F77101F1E4EF0EF11C3B
:10C1D00063966CAD7DAD8EAD9FAD63970E940DAD46
:10C1E0002BA13FA1A8010E94ABAE0E94E1ACD701F8
:10C1F0006D937D938D939C9313972BA13FA1A801E1
:10C200006BA17FA1C8010E94ABAE9B01AC0123963C
:10C210006CAD7DAD8EAD9FAD23970E94ABAEF101AD
:10C2200061837283838394832B962CAD3DAD4EAD99
:10C230005FAD2B976FA978AD89AD9AAD0E94ABAE7B
:10C240006BAB7CAB8DAB9EABD10155960D911D9127
:10C250002D913C9158970BA31CA32DA33EA35D9653
:10C260000D911D912D913C9190970FA318A729A78F
:10C270003AA759960D911D912D913C915C970BA772
:10C280001CA72DA73EA70BA11CA12DA13EA1012BF0
:10C29000022B032B41F52BA53CA54DA55EA5232B19
:10C2A000242B252B01F58FA198A5A9A5BAA5892B2B
:10C2B0008A2B8B2BC1F420917E0630917F06409112
:10C2C0008006509181066BA97CA98DA99EA90E9428
:10C2D000ABAE0E945AAC0E94E1AC4B015C01D101B3
:10C2E000D6961C92F0C20BAD1CAD2DAD3EAD012B10
:10C2F000022B032B49F060917A0670917B068091A6
:10C300007C0690917D0608C060918206709183063C
:10C3100080918406909185062BA93CA94DA95EA920
:10C320000E94ABAE0E945AAC0E94E1AC4B015C0192
:10C330002BAD3CAD4DAD5EAD232B242B252BA9F0B1
:10C3400020E030E0A9016091B8057091B9058091B5
:10C35000BA059091BB050E946DAC882331F081E055
:10C3600014141504160417040CF080E0D101D696BD
:10C370008C93882309F4BAC02091A8053091A905AF
:10C380004091AA055091AB056996EEADFFAD699756
:10C3900060817181828193810E9493AB2B013C016A
:10C3A0002091AC053091AD054091AE055091AF059F
:10C3B0006996AEADBFAD699714966D917D918D91E3
:10C3C0009C9117970E9493AB6BAF7CAF8DAF9EAFE4
:10C3D0002091B0053091B1054091B2055091B3055F
:10C3E0006996EEADFFAD699760857185828593850D
:10C3F0000E9493AB6B017C01A3019201C301B201C6
:10C400000E94ABAE2B013C012BAD3CAD4DAD5EAD02
:10C41000CA01B9010E94ABAE9B01AC01C301B201DC
:10C420000E9494AB2B013C01A7019601C701B60104
:10C430000E94ABAE9B01AC01C301B2010E9494AB60
:10C440000E9418AF6B017C012091B4053091B505B5
:10C450004091B6055091B7056996AEADBFAD6997ED
:10C460001C966D917D918D919C911F970E9493AB2D
:10C47000A70196010E9474AC6B017C01F101FD964D
:10C48000608371838283938320E030E040E450E452
:10C490000E9470AE18161CF4F10116AA27C0209154
:10C4A000B8053091B9054091BA055091BB05C70157
:10C4B000B6010E94ABAE9B01AC0160912206709167
:10C4C000230680912406909125060E9474AC2BA926
:10C4D0003CA94DA95EA90E94ABAE0E94E1AC6815D3
:10C4E00079058A059B0510F44B015C018091D1050B
:10C4F0009091D205A091D305B091D405F10141A04E
:10C5000052A063A074A00FA518A929A93AA9801761
:10C510009107A207B30708F4CDC02BA13CA14DA100
:10C520005EA1232B242B252B61F12091360630911F
:10C5300037064091380650913906281539054A05C5
:10C540005B05F8F46FA578A989A99AA90E9475AF2F
:10C550006B017C01A50194016BA17CA18DA19EA121
:10C560000E9475AFC616D706E806F90650F4C70153
:10C57000B6012BA13CA14DA15EA10E9498AF49013B
:10C580005A018BA59CA5ADA5BEA5892B8A2B8B2B0B
:10C5900061F120913A0630913B0640913C06509162
:10C5A0003D06281539054A055B05F8F46FA578A9FD
:10C5B00089A99AA90E9475AF6B017C01A50194011C
:10C5C0006BA57CA58DA59EA50E9475AFC616D70646
:10C5D000E806F90650F4C701B6012BA53CA54DA508
:10C5E0005EA50E9498AF49015A010FA118A529A57F
:10C5F0003AA5012B022B032B61F120913E063091CD
:10C600003F064091400650914106281539054A05DC
:10C610005B05F8F46FA578A989A99AA90E9475AF5E
:10C620006B017C01A50194016FA178A589A59AA54C
:10C630000E9475AFC616D706E806F90650F4C70182
:10C64000B6012FA138A549A55AA50E9498AF490166
:10C650005A01411451046104710409F434C1209158
:10C6600042063091430640914406509145062815F4
:10C6700039054A055B0508F026C16FA578A989A987
:10C680009AA90E9475AF6B017C01A5019401C301B9
:10C69000B2010E9475AFC616D706E806F90608F083
:10C6A00012C1C701B601A30192010E9498AF4901CE
:10C6B0005A0109C12BA13CA14DA15EA1232B242B22
:10C6C000252BE9F160913606709137068091380686
:10C6D00090913906681579058A059B0580F50E94B9
:10C6E0000DAD2FA938AD49AD5AAD0E94ABAE6B016F
:10C6F0007C016BA17CA18DA19EA10E940DAD6BA3BD
:10C700007CA38DA39EA3C501B4010E940DAD2BA1F6
:10C710003CA14DA15EA10E94ABAEA70196010E9473
:10C7200070AE181664F42BA13CA14DA15EA1C70107
:10C73000B6010E9474AC0E94E1AC4B015C018BA578
:10C740009CA5ADA5BEA5892B8A2B8B2BE9F1609109
:10C750003A0670913B0680913C0690913D06681523
:10C7600079058A059B0580F50E940DAD2FA938AD8E
:10C7700049AD5AAD0E94ABAE6B017C016BA57CA5A7
:10C780008DA59EA50E940DAD6BA37CA38DA39EA33A
:10C79000C501B4010E940DAD2BA13CA14DA15EA12C
:10C7A0000E94ABAEA70196010E9470AE181664F409
:10C7B0002BA13CA14DA15EA1C701B6010E9474ACA2
:10C7C0000E94E1AC4B015C010FA118A529A53AA577
:10C7D000012B022B032BE9F160913E0670913F067D
:10C7E0008091400690914106681579058A059B0560
:10C7F00080F50E940DAD2FA938AD49AD5AAD0E940C
:10C80000ABAE6B017C016FA178A589A59AA50E94AA
:10C810000DAD6BA37CA38DA39EA3C501B4010E94A3
:10C820000DAD2BA13CA14DA15EA10E94ABAEA70115
:10C8300096010E9470AE181664F42BA13CA14DA184
:10C840005EA1C701B6010E9474AC0E94E1AC4B012D
:10C850005C014114510461047104A9F16091420624
:10C8600070914306809144069091450668157905BC
:10C870008A059B0540F50E940DAD2FA938AD49AD45
:10C880005AAD0E94ABAE6B017C01C301B2010E94A4
:10C890000DAD2B013C01C501B4010E940DADA301FA
:10C8A00092010E94ABAEA70196010E9470AE1816CD
:10C8B00054F4A3019201C701B6010E9474AC0E9416
:10C8C000E1AC4B015C01F101E35BFF4F808291829F
:10C8D000A282B382C501B4010E940DAD6B017C013F
:10C8E0002BA93CA94DA95EA90E9474AC2B966CAFF4
:10C8F0007DAF8EAF9FAF2B97D10151966D937D93F6
:10C900008D939C9354972DEB37E346E051E4C70198
:10C91000B6010E94ABAE0E94E1ACF10161AB72AB1B
:10C9200083AB94AB86A9882381F1FD962081318168
:10C93000428153816091B8057091B9058091BA0523
:10C940009091BB050E94ABAE2B962CAD3DAD4EAD8C
:10C950005FAD2B970E94ABAE2091660630916706C3
:10C9600040916806509169060E94ABAE9B01AC01F4
:10C9700060E074E284EF99E40E9474AC0E94E1AC40
:10C98000D101D8967C936E93D797D10111960D91D2
:10C990001D912D913C91149763960CAF1DAF2EAF56
:10C9A0003FAF6397C901B8010E9418AF6FA77BAF73
:10C9B0008FAB9BA706E116E065961FAF0EAF65979C
:10C9C0003E0111E1610E711C06E116E021961FAFD8
:10C9D0000EAF21972D964EAC5FAC2D976BA37FA326
:10C9E000182F092F1BAAD201CD90DD90ED90FD905C
:10C9F0002D0120E030E0A901C701B6010E9470AE10
:10CA000087FF04C0F7FAF094F7F8F0942196EEADA2
:10CA1000FFAD219781909190A190B1902196FFAFA9
:10CA2000EEAF2197A5019401C701B6010E9470AE37
:10CA300018160CF03FC0FBA9FF2329F1A5019401B2
:10CA40006FA57BAD8FA99BA50E94ABAE4B015C018E
:10CA50002BA13FA1412F502FC701B6010E94ABAEC1
:10CA6000A50194010E9470AE181614F5A701960155
:10CA7000C501B4010E9474AC6BA37FA3182F092FCA
:10CA800021E02BAB17C0A7019601C501B4010E949C
:10CA900074AC9B01AC016BA17FA1812F902F0E94F0
:10CAA000ABAE6BA37FA3182F092F31E03BAB02C0C5
:10CAB00041E04BAB4614570409F095CF5BA1A59616
:10CAC0005FAFA5978FA1A6968FAFA697A7961FAF2A
:10CAD000A797A8960FAFA89724969FAD2497992360
:10CAE00009F44CC1C090BD05D090BE05E090BF05D3
:10CAF000F090C0052DEB37E346E855E3C701B601DA
:10CB00000E946DAC87FD3AC1C701B6010E9418AF03
:10CB10006B017C019B01AC016FA57BAD8FA99BA52F
:10CB20000E946DAC87FD04C0CFA6DBAEEFAAFBA6CA
:10CB30009601A7016FA57BAD8FA99BA50E9474AC40
:10CB4000A3966CAF7DAF8EAF9FAFA397A1ECB5E07E
:10CB50002196BFAFAEAF219720E030E040E85FE321
:10CB60002BAB3CAB4DAB5EAB24961FAE249721960E
:10CB7000AEADBFAD21976D917D918D919D91219627
:10CB8000BFAFAEAF2197A3962CAD3DAD4EAD5FAD1F
:10CB9000A3970E94ABAE6B017C012D96EEADFFAD6D
:10CBA0002D9781909190A190B1902D96FFAFEEAF0F
:10CBB0002D972496FFAD2497FF2391F02BA93CA934
:10CBC0004DA95EA90E94ABAE6B017C012BA93CA9CB
:10CBD0004DA95EA9C501B4010E94ABAE4B015C0139
:10CBE000A5019401C701B6010E9470AE20E030E0BB
:10CBF000A90118164CF5C501B4010E9470AE1816B3
:10CC00004CF020E030E0A901C701B6010E946DACF4
:10CC100087FF09C0A5019401C701B6010E9493AB2B
:10CC20002B013C0139C02401350177FA709477F863
:10CC30007094A3019201C701B6010E9470AE18164C
:10CC40005CF52601370128C0C501B4010E946DAC16
:10CC500087FD09C020E030E0A901C701B6010E94AC
:10CC600070AE18164CF4A7019601C501B4010E94DC
:10CC700093AB2B013C0110C02601370177FA709469
:10CC800077F87094A5019401C301B2010E9470AEBF
:10CC9000181614F0240135016596AEADBFAD659749
:10CCA000CD90DD90ED90FD906596BFAFAEAF6597EE
:10CCB000A7019601C301B2010E9470AE1816CCF410
:10CCC000A3019201C701B6010E9474AC9B01AC01A3
:10CCD0006BA97CA98DA99EA90E94ABAE6BAB7CAB66
:10CCE0008DAB9EAB2496BFAD2497BF5F2496BFAF9C
:10CCF00024972196EEADFFAD2197E15DF54009F057
:10CD000036CF24963FAD2497332371F02BA93CA94D
:10CD10004DA95EA96FA57BAD8FA99BA50E94ABAE67
:10CD20006FA77BAF8FAB9BA724EA30E74DE75FE3AC
:10CD30006FA57BAD8FA99BA50E94ABAE6B017C015B
:10CD40009B01AC01609193057091940580919505CC
:10CD5000909196050E9470AE181654F4A7019601A2
:10CD60006BA17FA1812F902F0E9470AE181634F016
:10CD70000FA50BA31BAD1FA31FA90BA5A5968FADD8
:10CD8000A597A6969FADA697A796AFADA797A8968D
:10CD9000BFADA8978093930590939405A0939505B4
:10CDA000B09396052BA13FA1412F502F6BA17FA1DE
:10CDB000812F902F0E94ABAE7B018C01CB01D8015B
:10CDC000F10181879287A387B4872B966CAD7DADE7
:10CDD0008EAD9FAD2B9790589B01AC010E9494ABF8
:10CDE0006D962CAD3DAD4EAD5FAD6D970E94ABAE77
:10CDF0009B01AC016BE077ED83E29BE30E9493AB78
:10CE00005B016C01A496FFADA497FF2361F09B0129
:10CE1000AC01B701C8010E946DAC87FD09C09A2D15
:10CE20008B2D860107C09BE087ED03E21BE302C068
:10CE30009E2D8F2D492F582FB801D10115964D9356
:10CE40005D936D937C9318971C919501A601639651
:10CE50006CAD7DAD8EAD9FAD63970E946DAC181625
:10CE600014F481E001C083E0182BF101108380E10C
:10CE7000FE013196A1ECB5E001900D928A95E1F7A3
:10CE8000F10181819281A381B4818093BD0590934A
:10CE9000BE05A093BF05B093C00580E16F96EEADCF
:10CEA000FFAD6F97A5EDB5E001900D928A95E1F782
:10CEB00080E16996EEADFFAD6997A8EAB5E0019013
:10CEC0000D928A95E1F781E00BC02896EFAC289788
:10CED000FFAC60960FAD609764961FAD649723C852
:10CEE000C959DF4F0FB6F894DEBF0FBECDBFDF913B
:10CEF000CF911F910F91FF90EF90DF90CF90BF9057
:10CF0000AF909F908F907F906F905F904F903F90E9
:10CF10002F9008956F927F928F929F92AF92BF92BF
:10CF2000CF92DF92EF92FF920F931F93CF93DF93F5
:10CF300000D01F92CDB7DEB74C013B0180918F0628
:10CF400090919006892BD9F5909194068091910645
:10CF5000981B9F709F3059F429833A834B835C83DD
:10CF60000E94FBAA5C814B813A812981EDCFD09050
:10CF700094068091940666E5869FC00111245701AE
:10CF8000C02E79018A019301A40160E08B56994F6C
:10CF90000E94385C8823A9F0209194069091910614
:10CFA000291303C094E690938E0691E09D0D9F7027
:10CFB0009093940689830E94D258898103C080E0AF
:10CFC00001C081E00F900F900F900F90DF91CF91F3
:10CFD0001F910F91FF90EF90DF90CF90BF90AF9097
:10CFE0009F908F907F906F9008958091940690917C
:10CFF0009106891B8F708F3019F40E94FBAAF5CF20
:10D00000809194068F5F8F70E091940696E59E9FC5
:10D01000F0011124EB56F94FDF011D929A95E9F7C3
:10D0200098E090834091D5055091D6056091D70541
:10D030007091D805458B568B678B708F4091D905C1
:10D040005091DA056091DB057091DC05418F528FBC
:10D05000638F748F4091DD055091DE056091DF058F
:10D060007091E005458F568F678F70A34091E10561
:10D070005091E2056091E3057091E40541A352A34C
:10D0800063A374A32091940690919106291303C081
:10D0900094E690938E06809394060C9416322F9209
:10D0A0003F924F925F926F927F928F929F92AF9238
:10D0B000BF92CF92DF92EF92FF920F931F93CF9385
:10D0C000DF93CDB7DEB7A9970FB6F894DEBF0FBEDA
:10D0D000CDBFF801A0918F06B0919006AB2B09F05F
:10D0E000A7C016010E2DF8A7EFA33EA32DA36A013A
:10D0F0007B01FC01408051806280738020915A0640
:10D1000030915B0640915C0650915D06C301B2010F
:10D110000E94ABAE0E947BAE698B7A8B8B8B9C8B13
:10D12000D7018D909D90AD90BC9020915E0630917E
:10D130005F064091600650916106C501B4010E94EE
:10D14000ABAE0E947BAE6D8B7E8B8F8B988FD601A2
:10D150002D913D914D915C9129A33AA34BA35CA3E2
:10D1600020916206309163064091640650916506F5
:10D1700069A17AA18BA19CA10E94ABAE0E947BAE5B
:10D18000698F7A8F8B8F9C8FEDA1FEA1C080D1809B
:10D19000E280F38020916606309167064091680630
:10D1A00050916906C701B6010E94ABAE0E947BAEEA
:10D1B0006D8F7E8F8F8F98A349825A826B827C827B
:10D1C0008D829E82AF82B88629A13AA14BA15CA133
:10D1D00029873A874B875C87CD86DE86EF86F88A7B
:10D1E0002091A90323FF10C06093E1057093E2052D
:10D1F0008093E3059093E405C092B405D092B50501
:10D20000E092B605F092B705AFA1B8A52D913D917A
:10D210004D915C917101BE016F5F7F4FCE014196D0
:10D2200079DE882331F089A70E94163289A501C0D2
:10D2300080E0A9960FB6F894DEBF0FBECDBFDF9198
:10D24000CF911F910F91FF90EF90DF90CF90BF9003
:10D25000AF909F908F907F906F905F904F903F9096
:10D260002F900895AF92BF92CF92DF92EF920F93DB
:10D270001F93CF93DF93CDB7DEB764970FB6F894C3
:10D28000DEBF0FBECDBFA98ABA8ACB8ADC8AFC0179
:10D2900080819181A281B38189839A83AB83BC838E
:10D2A000FB0180819181A281B3818D839E83AF83B5
:10D2B000B887FA0180819181A281B38189879A8799
:10D2C000AB87BC87F90180819181A281B3818D8771
:10D2D0009E87AF87B88BAE01475F5F4FBE016B5F24
:10D2E0007F4FCE0101960E945F59CE0141966C019D
:10D2F0009E01235F3F4FAE01475F5F4FBE016B5FF3
:10D300007F4F4097CCDE64960FB6F894DEBF0FBE19
:10D31000CDBFDF91CF911F910F91EF90DF90CF9014
:10D32000BF90AF9008958F929F92AF92BF92EF926D
:10D33000FF920F931F93CF93DF937B018A01E90143
:10D34000FC0180809180A280B38020915A063091A8
:10D350005B0640915C0650915D06C501B4010E94D8
:10D36000ABAE0E947BAE6093D5057093D6058093DB
:10D37000D7059093D80520915E0630915F064091C5
:10D38000600650916106F70160817181828193810D
:10D390000E94ABAE0E947BAE6093D9057093DA0514
:10D3A0008093DB059093DC05209162063091630643
:10D3B0004091640650916506F80160817181828117
:10D3C00093810E94ABAE0E947BAE6093DD057093AB
:10D3D000DE058093DF059093E0052091660630918D
:10D3E00067064091680650916906688179818A8153
:10D3F0009B810E94ABAE0E947BAE6093E10570936F
:10D40000E2058093E3059093E4058092A80590924D
:10D41000A905A092AA05B092AB05F7018081918180
:10D42000A281B3818093AC059093AD05A093AE0526
:10D43000B093AF05F80180819181A281B38180937F
:10D44000B0059093B105A093B205B093B305888160
:10D450009981AA81BB818093B4059093B505A0936F
:10D46000B605B093B70590919406809191069817F0
:10D4700059F0DF91CF911F910F91FF90EF90BF90E6
:10D48000AF909F908F90B1CD0E949C5A80916F0079
:10D4900081FBCC27C0F981FF05C080916F008D7F93
:10D4A00080936F0021EE35E04DED55E069ED75E0BC
:10D4B00085ED95E00E944635CC2329F080916F00E0
:10D4C000826080936F00DF91CF911F910F91FF9049
:10D4D000EF90BF90AF909F908F900895CF93DF9380
:10D4E000CDB7DEB760970FB6F894DEBF0FBECDBFE5
:10D4F000FC0180819181A281B38189839A83AB836E
:10D50000BC83FB0180819181A281B3818D839E8345
:10D51000AF83B887FA0180819181A281B381898725
:10D520009A87AB87BC87F90180819181A281B38101
:10D530008D879E87AF87B88BAE01475F5F4FBE0177
:10D540006B5F7F4FCE0101960E945F599E01235F62
:10D550003F4FAE01475F5F4FBE016B5F7F4FCE0114
:10D560000196E1DE60960FB6F894DEBF0FBECDBF28
:10D57000DF91CF910895CF92DF92EF92FF92FC015D
:10D58000C080D180E280F3802091660630916706EA
:10D590004091680650916906C701B6010E94ABAE82
:10D5A0000E947BAE6093E1057093E2058093E305F2
:10D5B0009093E405C092B405D092B505E092B6050B
:10D5C000F092B7059091940680919106981729F0F2
:10D5D000FF90EF90DF90CF9008CD0E949C5A8091F1
:10D5E0006F0081FB992790F981FF05C080916F0042
:10D5F0008D7F80936F004091E1055091E20560912D
:10D60000E3057091E4054093F9045093FA046093A4
:10D61000FB047093FC04992329F080916F008260D1
:10D6200080936F00FF90EF90DF90CF900895CF929E
:10D63000DF92EF92FF920F931F93CF93DF93C6E495
:10D64000D6E006E316E0C12CD12C7601C394699193
:10D650007991899199910E940DAD288939894A89DA
:10D660005B890E94ABAE0E94E1ACF80161937193BB
:10D67000819391938F01C616D706E806F90610F438
:10D680006B017C01F6E0C635DF0709F76FEF7FEF2E
:10D69000CB01A70196010E9498AF2093D10530934A
:10D6A000D2054093D3055093D405DF91CF911F91BC
:10D6B0000F91FF90EF90DF90CF9008950F931F93FD
:10D6C000CF93DF930AE516E0C6E2D6E0F801219198
:10D6D0003191419151918F0160E070E080E89FE3CA
:10D6E0000E9474AC6993799389939993F6E0C63359
:10D6F000DF0761F72CE532E048E552E064E572E0CF
:10D7000080E592E0EBDEDF91CF911F910F918FCFFB
:10D7100085EF9BE00C94D65381548A3108F041C0C8
:10D72000A82FB0E040911E0C50911F0C6091200C6E
:10D730007091210C04C076956795579547958A9509
:10D74000D2F740FF2EC0E091290CF0912A0CAC5F7B
:10D75000B34F8C918823E9F0E80FF11D808190EDA3
:10D76000980F9A3098F08E3211F481810CC08D326E
:10D7700011F08B3271F4818190ED980F9A3030F076
:10D780008E3239F4828180538A3018F49E2F8F2F85
:10D7900002C090E080E09093250C8093260C81E0FD
:10D7A000089580E00895B8DF882341F081E020915A
:10D7B000250C3091260C232B09F480E008950F935B
:10D7C0001F93CF938091250C9091260C009711F117
:10D7D000FC018F01C1912C2F2F7DA9F0C53411F0D0
:10D7E000C536B9F7F801108260E070E08091250C31
:10D7F0009091260C0E94FDAFF801C083562F472F51
:10D80000382F292F0BC060E070E0CF911F910F914E
:10D810000C94FDAF50E040E030E020E0652F742F25
:10D82000832F922FCF911F910F9108958091250CF6
:10D830009091260C009731F04AE050E060E070E0F3
:10D840000C9463B160E070E0CB010895CF9384E560
:10D85000AADF882359F1EADF97FD24C0E7DF6F3F95
:10D8600071058105910509F0FCF4E0DFC62F16165D
:10D87000FCF40E94F0158DE40E9472186AE070E0DA
:10D880008091220C9091230C0E9465196C2FCC0F73
:10D89000770B87E095E10E9413168AE00E947218C8
:10D8A0008FEF07C0C0E004C0CFEF02C080E001C02E
:10D8B0008C2FCF910895BF92CF92DF92EF92FF927B
:10D8C0000F931F93CF93DF9380E8E82E85E0F82E27
:10D8D00000E512E09BEFC92E9BE0D92ECDE4D3E00A
:10D8E000BC2E84E0B80E89915EDF8823B1F067DF3B
:10D8F000F6012081211104C020919005222339F0E6
:10D90000F80120813181428153810E9494ABF7015B
:10D9100060837183828393830AC0F801808191813F
:10D92000A281B381F70180839183A283B383F4E062
:10D93000EF0EF11C0C5F1F4F8FEFC81AD80ABC12F4
:10D94000D2CF86E430DF8823B9F039DF20E030E041
:10D95000A9010E9470AE18167CF431DF20E030E09F
:10D9600040E752E40E9474AC60934C0270934D0205
:10D9700080934E0290934F02DF91CF911F910F91B0
:10D98000FF90EF90DF90CF90BF900895CF92DF92FD
:10D99000EF92FF926B017C010E946511C60ED71EAB
:10D9A000E81EF91E0E946511DC01CB018C199D094E
:10D9B000AE09BF09B7FF03C00E94FBAAF3CFFF90D7
:10D9C000EF90DF90CF9008956F927F928F929F9209
:10D9D000AF92BF92CF92DF92EF92FF920F931F937D
:10D9E000CF93DF93CDB7DEB73C01A090290CB09068
:10D9F0002A0CCDB6DEB66AE070E0C3010E94D0B357
:10DA00007C01009721F08C010619170904C0C3019D
:10DA10000E94DBB38C01C80101962DB73EB7281BCD
:10DA2000390B0FB6F8943EBF0FBE2DBF8DB79EB712
:10DA300001964C01A801B3010E94FCB3F401E00F70
:10DA4000F11F1082C40148D581E034D0E114F10403
:10DA500051F037019FEF691A790A0FB6F894DEBECC
:10DA60000FBECDBEC6CF0FB6F894DEBE0FBECDBE84
:10DA7000C501DF91CF911F910F91FF90EF90DF9043
:10DA8000CF90BF90AF909F908F907F906F9024C564
:10DA9000CF93C3E00E949687882341F0C15019F0CC
:10DAA0000E94E5A9F7CFCF910C9412AA80EF94E1E0
:10DAB000CF918ACFCF93C82F41E04093FA0B90913A
:10DAC000240C9D3409F45EC0943509F4F7C19734F1
:10DAD00009F0F8C12091220C3091230C2B31310533
:10DAE00009F43EC0CCF42430310544F42230310531
:10DAF00064F537FDE7C10E944197E7C12C3031053D
:10DB000061F12531310509F4E0C12430310509F016
:10DB1000D9C10E944A97D9C12A35310551F154F42F
:10DB20002D31310521F1FCF02E31310509F0CAC14A
:10DB300051D2CBC12C35310511F1F4F0293A3140E5
:10DB400009F0C0C10E944C85C0C181E0223031057E
:10DB500009F080E00E94729BB8C10E945592B5C145
:10DB60000E945992B2C180E00E944A7BAEC190DF10
:10DB7000ACC110929005A9C140939005A6C10E9426
:10DB80007679A3C12091220C3091230C29373105DD
:10DB900009F45DC10CF083C02836310509F42AC1AF
:10DBA0000CF044C02C34310509F421C104F52231B4
:10DBB000310509F43EC164F437FD84C122303105DA
:10DBC0000CF40DC12131310509F07CC19ED77DC116
:10DBD0002A32310509F405C12B34310509F404C199
:10DBE0002F31310509F06EC10E9453786EC1233583
:10DBF000310509F41BC16CF42135310509F411C15B
:10DC00000CF011C12D34310509F05CC10E949177EF
:10DC10005CC12535310509F40EC10CF40AC12C355F
:10DC2000310509F04FC10E94E8934FC120373105FB
:10DC300009F44BC1CCF42C36310509F446C15CF42F
:10DC40002A36310509F4E7C00CF0E8C00E94B2A101
:10DC50001092FA0B41C12E36310509F4CEC00CF0FA
:10DC6000CFC00E943FA131C12537310509F4E8C07A
:10DC70006CF42237310509F4E0C00CF4C3C023373B
:10DC8000310509F01FC10E940C791FC127373105EA
:10DC900009F4D8C00CF0D9C00E94C07816C12E3546
:10DCA00081E0380709F408C10CF04BC0233D310571
:10DCB00009F4D8C01CF5293C310509F4CAC07CF42C
:10DCC0002B39310509F4A4C02E3B310509F49DC060
:10DCD0002C38310509F0F6C00E9496A0F6C02C3C05
:10DCE000310509F4B9C02D3C310509F4B8C02B3C0D
:10DCF000310509F0E7C00E948295E7C02D3281E02E
:10DD0000380709F4B6C07CF42D3D310509F4ACC0E8
:10DD1000223E310509F4ABC02C3D310509F0D2C0DB
:10DD20000E949793D2C02F3281E0380709F4A7C030
:10DD30000CF4A2C02033314009F0C4C00E942593E6
:10DD4000C4C0243F81E0380709F4A8C014F5223983
:10DD500081E0380709F49AC06CF4203981E0380773
:10DD600009F490C00CF090C02F35314009F0AAC0E2
:10DD7000ABD5ABC0243A81E0380709F489C0293A11
:10DD800081E0380709F487C02A39314009F09AC088
:10DD90009CC0283F81E0380709F486C04CF4263F38
:10DDA00081E0380709F47CC00CF07CC010D58DC030
:10DDB000243883E0380709F479C034F4233533403C
:10DDC00009F080C040D281C02B3883E0380709F4C5
:10DDD00070C0273E334009F075C093D776C0ACD2EF
:10DDE00074C00E942E7771C00E948D776EC00E9411
:10DDF0008F776BC00E941CA168C00E945C7965C0CF
:10DE00000AD763C00E947E7860C00E94AFA05DC048
:10DE10000E94D5A05AC00E9495A157C00E94ABA1F4
:10DE200054C05ED752C00E943A974FC00E943D979F
:10DE30004CC06DD64AC018D648C00E94BC7845C0B8
:10DE40007AD243C00E94B47840C081D73EC082D706
:10DE50003CC00E94539539C00E94A79536C00E94CD
:10DE60001D9633C07CD731C00E94CA922EC0C0D547
:10DE70002CC00E94A39629C00E94BC9426C00E9478
:10DE8000E19F23C06AD721C09BD01FC09ED01DC078
:10DE90000E947C861AC00E94057A17C096D415C0CD
:10DEA00098D413C098D411C0BBD40FC00E94D49191
:10DEB0000CC00E94A59209C0D2D407C08091220C48
:10DEC0001ED603C083E09CE072D41092FA0BC111FD
:10DED00003C0CF910C94FC9DCF910895CF93DF9315
:10DEE000C091C50E80E6C89FE0011124CC51D34FEC
:10DEF0008091A90380FF05C00E94F015CE010E9409
:10DF0000C918CE01E9D280E0DF91CF91D3CDCF9275
:10DF1000DF92EF92FF920F931F930E9465116B01A6
:10DF20007C018091E50E81112FC0809166028823CB
:10DF300059F18091FA0B882339F14091F60B5091F9
:10DF4000F70B6091F80B7091F90B97018601041B98
:10DF5000150B260B370B37FD2CC0833079F03CF4C2
:10DF6000813094F00E94F0158EED94E10BC0843066
:10DF700059F40E94F0158FEA94E104C00E94F01554
:10DF800087EC94E10E94E2152091660230E0A8EE51
:10DF9000B3E00E94DEAFDC01CB018C0D9D1DAE1DF8
:10DFA000BF1D8093F60B9093F70BA093F80BB093E3
:10DFB000F90B1F910F91FF90EF90DF90CF90089594
:10DFC00081E00E94524B0C94964E80E00E94524B8E
:10DFD0000C94964E8F929F92AF92BF92CF92DF9207
:10DFE000EF92FF920F931F93CF93DF93CDB7DEB7DE
:10DFF00028970FB6F894DEBF0FBECDBFC090500279
:10E00000D0905102E0905202F090530288E5CBDBB1
:10E01000811108C020E030E0A901C701B6010E94CB
:10E0200094AB01C0CCDB6D837E838F839887C090D7
:10E030005402D0905502E0905602F090570289E5C4
:10E04000B2DB811108C020E030E0A901C701B601B0
:10E050000E9494AB01C0B3DB6B017C0169837A83BE
:10E060008B839C838D809E80AF80B88422ED30E0CE
:10E0700040EE50EC0E9470AE87FDD2C027E030E049
:10E080004EE353E4C701B6010E946DAC18160CF4C0
:10E09000C7C023EA31E040E450ECC501B4010E945E
:10E0A00070AE87FDBDC027E030E042E253E4C50119
:10E0B000B4010E946DAC18160CF4B2C027E030E039
:10E0C00041E253E4C501B4010E946DAC18160CF492
:10E0D000A7C027E030E041E253E4C701B6010E9447
:10E0E0006DAC18160CF49CC080E00E94661A0E9469
:10E0F000965085E458DB182F8823B1F08091250CC9
:10E100009091260C892B09F489C090DB97FD0FC0F4
:10E110008DDB6F3F71058105910509F04CF486DBBD
:10E1200061117CC040E005C085E4F6DA77C010E0FC
:10E13000412F01E021E0BE016F5F7F4FCE010596C8
:10E140000E94F34B6B017C019B01AC010E9459AF13
:10E1500081115FC08D809E80AF80B88420E030E068
:10E16000A901C501B4010E946DAC87FD05C027E17E
:10E1700037EB41E558E304C027E137EB41E558EBC5
:10E18000C501B4010E9494ABAB01BC0184E295E1EE
:10E190000E942D1689809A80AB80BC8020E030E000
:10E1A000A901C501B4010E946DAC87FD05C027E13E
:10E1B00037EB41E558E304C027E137EB41E558EB85
:10E1C000C501B4010E9494ABAB01BC018FE195E1A4
:10E1D0000E942D1620E030E0A901C701B6010E947F
:10E1E0006DAC87FD05C027E137EB41E558E304C07E
:10E1F00027E137EB41E558EBC701B6010E9494AB2C
:10E20000AB01BC018AE195E10E942D168AE00E94D3
:10E2100072180E94B5500E94964E02C041E089CF0C
:10E2200028960FB6F894DEBF0FBECDBFDF91CF9119
:10E230001F910F91FF90EF90DF90CF90BF90AF9024
:10E240009F908F900895EF92FF920F931F93CF931B
:10E25000DF938AE561DA882309F456C08091250CA2
:10E260009091260C009709F44FC0FC017F01C191E9
:10E270002C2F2F7D89F0C53411F0C536B9F7F70181
:10E28000108260E070E08091250C9091260C0E9435
:10E29000FDAFF701C08304C060E070E00E94FDAFF5
:10E2A0008B01D82FC92F20E030E040E050EC0E94D5
:10E2B00070AE87FD1DC020E030E040EA50E4B801B8
:10E2C0008D2F9C2F0E946DAC181694F0C801AD2FB5
:10E2D000BC2F80936A0590936B05A0936C05B09357
:10E2E0006D05DF91CF911F910F91FF90EF900895F1
:10E2F0000E94F3158DE395E1DF91CF911F910F916E
:10E30000FF90EF900C94E2150E94F01540916A0581
:10E3100050916B0560916C0570916D058CE295E1F3
:10E320000E942D168AE0DF91CF911F910F91FF90EF
:10E33000EF900C9472180895CF92DF92EF92FF92B3
:10E340000F931F93CF93DF93C091270CD091280C8C
:10E3500080E529DA8823D1F08091250C9091260C54
:10E36000009749F04AE050E060E070E00E948BB214
:10E370006B017C0103C0C12CD12C760111E0C114CA
:10E38000D104E104F10431F410E004C010E0C12C28
:10E39000D12C760183E507DA882309F486C08091C1
:10E3A000250C9091260C009701F1FC017F01019151
:10E3B000202F2F7D89F0053411F00536B9F7F701CC
:10E3C000108260E070E08091250C9091260C0E94F4
:10E3D000FDAFF701008304C060E070E00E94FDAF74
:10E3E000B62FA72FF82FE92F04C0B0E0A0E0F0E08F
:10E3F000E0E020E030E04AE754E46B2F7A2F8F2FE3
:10E400009E2F0E94ABAE0E94E1AC6B017C0111110A
:10E4100009C0672B682B692B29F4209719F0888194
:10E42000811102C010E001C011E00E949C5A11232A
:10E4300029F00E94F015CE010E94C91883E0809354
:10E44000FA0B81E08093E60EC114D104E104F104DB
:10E4500029F10E946511C60ED71EE81EF91E0E9402
:10E460006511DC01CB018C199D09AE09BF09B7FD0F
:10E470000EC01092E60E81E08093FA0BDF91CF91EF
:10E480001F910F91FF90EF90DF90CF9008958091B2
:10E49000E60E882371F30E94FBAAE1CF8091E60E7D
:10E4A000882339F30E94FBAAF9CF1111BBCFB5CF56
:10E4B0001092280C1092270C8FE38093240C10925A
:10E4C000230C1092220C10921E0C10921F0C109212
:10E4D000200C1092210C08953F924F925F926F9200
:10E4E0007F928F929F92AF92BF92CF92DF92EF92E4
:10E4F000FF920F931F93CF93DF931F921F92CDB77D
:10E50000DEB789839A83D4DF8981282F9A81392FB6
:10E51000F90180812F5F3F4F8032D1F38E34B1F407
:10E52000818190ED980F9A3020F08D3211F08B326E
:10E5300069F43296DF0131962C9120532A30D0F3C2
:10E54000CD01FC01019620812032D9F3F0932A0CF1
:10E55000E093290C8F010F5F1F4F30806AE270E05B
:10E56000C8010E9432B4009731F0FC0131978081DC
:10E570008032E1F311828DE4381631F0E4E53E1685
:10E5800019F0F7E43F12FFC0F80180810F5F1F4FC1
:10E590008032D1F380538A3008F0F5C03092240CD9
:10E5A0001092230C1092220C4AE02091220C309100
:10E5B000230C429FC001439F900D11249093230C84
:10E5C0008093220C3196DF0111972C91022E000CC2
:10E5D000330B20533109280F391F3093230C20931C
:10E5E000220C808180538A3000F3DF0131968C91B8
:10E5F0008032D9F38DE438121AC02E31310591F0F2
:10E600003CF42731310571F02C31310581F40AC019
:10E610002537310564F02737310524F0203AE3E04F
:10E620003E0729F4B093280CA093270CACC010929D
:10E63000280C1092270C5091290CC12CD12C76015A
:10E64000C394FD0131964C91442309F49CC041329E
:10E65000A9F48DE4381212C02032310579F4F09318
:10E66000280CE093270C63E270E0CF010E9432B4E3
:10E67000009709F488C0FC01108285C041544A31DA
:10E6800008F055C0BF01FB0180816F5F7F4F803272
:10E69000D1F390ED980F9A3008F18E3211F4818108
:10E6A0000CC08D3211F08B3259F4818190ED980FAE
:10E6B0009A30A0F08E3221F4828180538A3070F03B
:10E6C0008091270C9091280C892B09F059C0CF011B
:10E6D00001979093280C8093270C52C0CF01A42F50
:10E6E000B0E04601570104C0880C991CAA1CBB1C51
:10E6F0004A95D2F740901E0C50901F0C6090200C51
:10E700007090210C84289528A628B72880921E0C8A
:10E7100090921F0CA092200CB092210C009711F047
:10E72000851B01C080E0AC5FB34F8C930AC0809121
:10E73000270C9091280C892B21F4B093280CA093DE
:10E74000270C808181548A3130F4DF017ACF80ED4B
:10E75000890F8A3040F44E2F6F2F91919111F7CF8E
:10E76000842F962F07C083ED890F8230A0F39B3250
:10E7700091F3F6CFFC01019640814032D9F3E5CF09
:10E7800080E090E0ACCF0F900F90DF91CF911F9180
:10E790000F91FF90EF90DF90CF90BF90AF909F9040
:10E7A0008F907F906F905F904F903F9008950E9460
:10E7B000F0156091290C70912A0C8BE595E10E946F
:10E7C000F61588E595E10C94E2150C945C3E0C94EA
:10E7D0004B4B0C94E941CF9383E50E948C6BC82F7F
:10E7E000882331F08091250C9091260C892B41F4DF
:10E7F00083E50E948C6BC1E08C2FCF910C942C434D
:10E8000015D897FD0BC012D86F3F71058105910592
:10E8100009F094F70BD8C1E06111EECFC0E0ECCF66
:10E820000E94444B882331F00E94F0158EE695E15A
:10E830000C94E21508950E94166C97FD0CC00E947E
:10E84000166C6F3F71058105910509F034F40E9443
:10E85000166C862F089580E008958FEF08950F932A
:10E860001F93CF9383E50E948C6B811104C001E557
:10E8700013E0C0E00DC0C0E0DEDF682F8C2F0E94E7
:10E88000D43CCF5FC530C1F7F2CFCF5FC43069F061
:10E89000F80181918F010E948C6B8823B1F3CBDF4B
:10E8A000682F8C2F0E94D43CF0CF82E40E948C6BA6
:10E8B000882329F0C0DF682F84E00E94D43CCF91E8
:10E8C0001F910F910C94813D0F931F93CF9383E57C
:10E8D0000E94D36B882309F465C0ADDF823029F133
:10E8E000833009F43FC0813009F05CC001E513E0DA
:10E8F000C0E0F80181918F010E94D36B882339F029
:10E900009ADF2FEF4FEF682F8C2F0E947D3CCF5F57
:10E91000C43079F782E40E94D36B882309F442C0A3
:10E920008ADF2FEF4FEF682F3AC001E513E0C0E018
:10E93000F80181918F010E94D36B882339F07BDF2E
:10E940002FEF482F6FEF8C2F0E947D3CCF5FC4309C
:10E9500079F782E40E94D36B882321F16CDF2FEFDB
:10E96000482F1CC001E513E0C0E0F80181918F0140
:10E970000E94D36B882339F05EDF282F4FEF6FEFB3
:10E980008C2F0E947D3CCF5FC43079F782E40E94D7
:10E99000D36B882339F04FDF282F4FEF6FEF84E0E0
:10E9A0000E947D3CCF911F910F910C94813DCF939C
:10E9B000DF931F921F92CDB7DEB769837A830E94DF
:10E9C0008C6B69817A81882361F08091250C90910C
:10E9D000260C009731F04AE050E060E070E00E94C1
:10E9E00063B1972F862F0F900F90DF91CF910895ED
:10E9F0001F93CF93DF9380E50E948C6B882381F176
:10EA000060E070E080E5D3DF182F6FEF7FEF83E5E4
:10EA1000CEDFEC010196039718F517FD21C00E9487
:10EA20009C5ACF3F8FEFD80729F0219771F4C1E0AE
:10EA3000D0E00DC0812F0E94B91331E020E0892B76
:10EA400009F030E0C32FD22F02C0C0E0D0E0812F08
:10EA50000E94B9138C179D0719F00E94FBAAF7CFEB
:10EA6000DF91CF911F9108950F931F93CF9383E56B
:10EA70000E948C6B882309F43EC08091250C9091F4
:10EA8000260C009701F1FC018F01C1912C2F2F7DE5
:10EA900089F0C53411F0C536B9F7F801108260E08D
:10EAA00070E08091250C9091260C0E94FDAFF8013A
:10EAB000C08304C060E070E00E94FDAFB62FA72FB6
:10EAC000F82FE92F04C0B0E0A0E0F0E0E0E020E0A3
:10EAD00030E04AE754E46B2F7A2F8F2F9E2F0E944D
:10EAE000ABAE0E94E1AC6093E10E7093E20E8093B6
:10EAF000E30E9093E40ECF911F910F91089520E0C3
:10EB000040E050E0BA010C94C5310C94CBA90F93AE
:10EB10001F93CF9383E50E948C6B882391F18091A2
:10EB2000250C9091260C009761F1FC018F01C19199
:10EB30002C2F2F7D89F0C53411F0C536B9F7F801B7
:10EB4000108260E070E08091250C9091260C0E946C
:10EB5000FDAFF801C08304C060E070E00E94FDAF2B
:10EB600020E030E04AE754E40E94ABAE0E94E1AC02
:10EB700060936B0270936C0280936D0290936E02AF
:10EB800046C088E50E948C6B811114C089E50E9403
:10EB90008C6B81110FC08AE50E948C6B81110AC0B9
:10EBA00085E40E948C6B811105C0CF911F910F915C
:10EBB0000C94775A0E949C5A88E50E948C6B88239B
:10EBC00031F0179A809191058E7F8093910589E5A8
:10EBD0000E948C6B882331F0169A809191058D7F6D
:10EBE000809391058AE50E948C6B882331F0159AF9
:10EBF000809191058B7F8093910585E40E948C6BB9
:10EC0000882329F0CF911F910F910C94D0A9CF9117
:10EC10001F910F910895FF920F931F93CF93DF934E
:10EC200083E50E948C6B8823F1F083E50E948C6B56
:10EC3000811102C060E015C08091250C9091260CD6
:10EC4000892BC1F30E94166C97FDF4CF0E94166CBD
:10EC50006F3F71058105910511F00CF03FC00E94D6
:10EC6000166C6093A9030E94F0158DEA95E10E944D
:10EC7000E2158091A903882329F103EA15E1C0E098
:10EC8000D0E020E08091A90390E00C2E02C0959581
:10EC900087950A94E2F780FF0EC0FF24F394F20EEA
:10ECA000222319F08CE20E947218F8018591949148
:10ECB0000E94E2152F2D21960E5F1F4FC530D10502
:10ECC00009F704C08FE995E10E94E2158AE0DF911F
:10ECD000CF911F910F91FF900C9472186FEFC1CFDD
:10ECE0000E9471230E941BA70E94775A60E070E087
:10ECF00080E00E94071B68EE73E080E090E00C94D7
:10ED0000A01581E08093700283E50E948C6B8823BC
:10ED100031F08091250C9091260C892B39F483E5F4
:10ED20000E948C6B811112C00C945B9E0E94166C29
:10ED300097FDFACF0E94166C6F3F71058105910512
:10ED400009F024F40E94166C662371F3089581E0A3
:10ED50000C94633080E00C9463300C949C5ACF93F5
:10ED60000E94F01584ED95E10E94E21583E50E9472
:10ED70008C6BC82F8823D1F08091250C9091260CA4
:10ED8000892B91F00E94166C97FD0DC00E94166CA5
:10ED90006F3F71058105910509F034F40E94166CEE
:10EDA000C1E0611101C0C0E0C093450280914502FD
:10EDB0000E9467168CEC95E10E94E21540913902A1
:10EDC00050913A0260913B0270913C028AEC95E1CD
:10EDD0000E942D1640913D0250913E0260913F02EB
:10EDE0007091400287EC95E10E942D1640914102FE
:10EDF00050914202609143027091440284EC95E18B
:10EE00000E942D168CEB95E10E94E21540912D0297
:10EE100050912E0260912F02709130028AEB95E1A1
:10EE20000E942D16409131025091320260913302BE
:10EE30007091340287EB95E10E942D1640913502C6
:10EE400050913602609137027091380284EB95E15F
:10EE50000E942D168AE0CF910C9472180F931F9385
:10EE6000CF93DF9383E50E94D36B882309F450C0CE
:10EE7000E2DC182F80E50E94D36B81110AC081E08B
:10EE8000111101C080E0DF91CF911F910F910C947F
:10EE90008A1580E50E94D36B882331F00E94166C9E
:10EEA000EB0177FD35C002C0CDE0D0E00C2F89E446
:10EEB0000E94D36B882351F08091250C9091260CF1
:10EEC000892B49F0B8DC811106C017C089E40E9483
:10EED0008C6B882391F061E08C2F0E944E13612F80
:10EEE0008C2F0E948A13612F70E08C2F0E943112A8
:10EEF000083071F41093C7040BC0802F0E9494A9AE
:10EF0000882349F3DF91CF911F910F910C94BCA9F5
:10EF1000DF91CF911F910F9108950C9494A70C94B9
:10EF200030A70C941BA74F925F926F927F92AF9283
:10EF3000BF92CF92DF92EF92FF92CF93DF93EB01DC
:10EF4000FC0160817181828193812CE3C22ED12CDE
:10EF5000E12CF12CA70196010E9498AFB62EA72EA6
:10EF6000CA01B901A70196010E9498AF6B017C010B
:10EF7000CA01B90128E130E040E050E00E9498AFBA
:10EF80002B013C01C9016DE671E00E9484AF61155F
:10EF90007105D9F0AF92BF92DF92CF925F924F92FC
:10EFA0009F938F937F936F938CE096E19F938F93C2
:10EFB000DF93CF930E945DB48DB79EB70E960FB6C8
:10EFC000F8949EBF0FBE8DBF61C00097C9F0AF928D
:10EFD000BF92DF92CF925F924F929F938F938CEF6D
:10EFE00095E19F938F93DF93CF930E945DB4EDB72C
:10EFF000FEB73C960FB6F894FEBF0FBEEDBF46C0FD
:10F000004114510461047104B9F0AF92BF92DF92D0
:10F01000CF925F924F9280EF95E19F938F93DF9312
:10F02000CF930E945DB48DB79EB70A960FB6F89441
:10F030009EBF0FBE8DBF2AC0C114D104E104F104EC
:10F04000A9F0AF92BF92DF92CF9288EE95E19F93A5
:10F050008F93DF93CF930E945DB4EDB7FEB73896E0
:10F060000FB6F894FEBF0FBEEDBF10C0AF92BF92B7
:10F0700084EE95E19F938F93DF93CF930E945DB4CD
:10F080000F900F900F900F900F900F90DF91CF91F6
:10F09000FF90EF90DF90CF90BF90AF907F906F90F8
:10F0A0005F904F900895CF93DF93CDB7DEB7699708
:10F0B0000FB6F894DEBF0FBECDBF0E9460A76E8B67
:10F0C0007F8B888F998FBE016F5F7F4FCE014696F1
:10F0D0002ADF0E94F015BE016F5F7F4F80E296E14C
:10F0E0000E94F6158AE00E94721869960FB6F8948D
:10F0F000DEBF0FBECDBFDF91CF91089583E50E94A3
:10F100008C6B882331F08091250C9091260C892BF3
:10F1100071F40E94F0154091660250E060E070E0EA
:10F120008DE296E10E9457168AE00C9472180E94B4
:10F13000166C97FD17C00E94166C6F3F7105810514
:10F14000910509F01CF40E94166C01C06FEF862F28
:10F1500090E0CD971CF46093660208958CE3809351
:10F160006602089560E0F3CF81E00E948A150E9454
:10F17000CA3080E00C948A150E949C5A0C94964EDA
:10F180001F93CF93DF93C091270CD091280C83E07D
:10F1900010E040E08150C9F09881292F2B7F213465
:10F1A000C9F729812133B1F7913421F0953419F44D
:10F1B00041E001C011E09E012E5F3F4FE9012F5F4A
:10F1C0003F4F98819032D1F3E5CF41110E94F01565
:10F1D000112321F084E396E10E94E215CE01DF9134
:10F1E000CF911F910C94C9180F931F93CF938C014B
:10F1F000C62F88E396E10E94E215C8010E94E2153D
:10F200008AE30E9472186AE070E08C2F90E0CF9140
:10F210001F910F910C946B198DE497E10E94E215F8
:10F2200060E08DE397E1E0DF60E088E297E1DCDF1A
:10F2300061E081E297E1D8DF60E086E197E1D4DF29
:10F2400061E086E097E1D0DF60E08DEF96E1CCDF12
:10F2500061E083EF96E1C8DF61E089EE96E1C4DF0B
:10F2600061E081EE96E1C0DF61E083ED96E1BCDF15
:10F2700060E085EC96E1B8DF60E086EB96E1B4DF14
:10F2800060E088EA96E1B0DF60E082E996E1ACDF19
:10F2900061E081E896E1A8DF60E082E796E1A4DF23
:10F2A00060E08DE596E1A0DF61E08AE496E19CDF15
:10F2B00060E08DE396E198CF8EE40E948C6B88230A
:10F2C000A1F08091250C9091260C009771F04AE0F6
:10F2D00050E060E070E00E9463B16093C70E7093ED
:10F2E000C80E8093C90E9093CA0E08954F925F92F4
:10F2F0006F927F929F92AF92BF92CF92DF92EF92E6
:10F30000FF920F931F93CF93DF9385E5E82E83E061
:10F31000F82E00E512E0B12C912CA12CF70181917F
:10F320007F010E948C6B882309F450C08091250CCA
:10F330009091260C009709F449C0FC013F01C1914E
:10F340002C2F2F7D89F0C53411F0C536B9F7F301A4
:10F35000108260E070E08091250C9091260C0E9454
:10F36000FDAFF301C08304C060E070E00E94FDAF18
:10F370006B01D82FC92FF80120813181428153813F
:10F380000E9493AB2B013C012DEB37E346E855EB94
:10F390000E9470AE87FD0AC02DEB37E346E855E3C7
:10F3A000C301B2010E946DAC181684F4F3E0BF16DD
:10F3B00019F09924939402C0AA24A394A6016D2F56
:10F3C0007C2FF8014083518362837383B3940C5F75
:10F3D0001F4FF4E0BF12A2CF992019F00E94BE4E39
:10F3E00003C0A1100E94C84EDF91CF911F910F91D1
:10F3F000FF90EF90DF90CF90BF90AF909F907F9065
:10F400006F905F904F900C94964EBF92CF92DF9288
:10F41000EF92FF920F931F93CF93DF9329E5E22E94
:10F4200023E0F22E0BE21CE06701C0E0D0E0BB2439
:10F43000B394F60181916F010E948C6B882351F186
:10F440000E949C5AF8016081662389F070E080E098
:10F4500090E00E940FAD9B01AC01FE01E25DF34F15
:10F4600060817181828193810E9474AC03C060E0ED
:10F4700070E0CB012091250C3091260C232B11F04C
:10F480000E94DF6BFE01E25CF34F60837183828335
:10F490009383B12C24960F5F1F4FCC30D10549F6D2
:10F4A00086E40E948C6B882371F10E949C5A0E9412
:10F4B000DF6B8B01D82FC92F20E030E040E85FE3FD
:10F4C0000E9470AE18167CF020E030E0A901B8016F
:10F4D0008D2F9C2F0E946DAC87FF09C000E010E0CB
:10F4E000D0E0C0E004C000E010E0D0E8CFE3C80105
:10F4F000AD2FBC2F80933A0C90933B0CA0933C0C07
:10F50000B0933D0CB12C83E50E948C6B882369F08D
:10F510000E949C5A0E94DF6B60936702709368029E
:10F520008093690290936A02ABC0BB2009F4A8C023
:10F530008EE099E10E94E21520E030E0A90160919F
:10F540003A0C70913B0C80913C0C90913D0C0E94C8
:10F550006DAC811104C08BE099E10E94E21582E05C
:10F5600099E10E94E21540913A0C50913B0C609158
:10F570003C0C70913D0C8EED98E10E942D168DEBA8
:10F5800098E10E94E2158BE998E10E94E2150EE3F2
:10F590001CE0C9E5D3E093E0D92EDE0C80E20E94A6
:10F5A000721889910E947218F8016191719181918C
:10F5B00091918F0142E050E00E94F0198AE00E9490
:10F5C0007218DC12EBCF4091670250916802609193
:10F5D000690270916A0287E798E10E942D168AE01D
:10F5E0000E94721885E598E10E94E2158EE2C82E0D
:10F5F0008CE0D82ECBE2DCE013E01C0F888188235E
:10F60000D1F080E20E947218F70180810E94721886
:10F61000688170E080E090E00E940FAD9B01AC013A
:10F62000F60160817181828193810E9474AC42E015
:10F6300050E00E94F0192196FFEFEF1AFF0A84E0D4
:10F64000C80ED11C1C13DACF80912B0C81110CC079
:10F6500080912C0C811108C080912D0C811104C067
:10F6600081E498E10E94E2158AE0DF91CF911F9139
:10F670000F91FF90EF90DF90CF90BF900C94721895
:10F68000DF91CF911F910F91FF90EF90DF90CF907E
:10F69000BF9008952F923F924F925F926F927F9208
:10F6A0008F929F92AF92BF92CF92DF92EF92FF9292
:10F6B0000F931F93CF93DF93CDB7DEB76A970FB643
:10F6C000F894DEBF0FBECDBF182F81E00E948A15CF
:10F6D0008FE40E94D36B8823B9F08091250C909120
:10F6E000260C892BB1F00E94166C97FD18C00E9461
:10F6F000166C6F3F71058105910509F054F40E9465
:10F70000166C611106C00BC08FE40E948C6B8823BD
:10F7100031F0909192059770973009F40FC20E94D2
:10F720009C5A20911506288F80E00E94661A0E943C
:10F73000965081E00E947630111119C088E50E9430
:10F740008C6B382E89E50E948C6B182F8AE50E94FD
:10F750008C6B282E311006C0111110C081110EC003
:10F76000312E0AC0112351F0312E082F08C011E0AC
:10F77000332433942224239401E001C000E080E18B
:10F78000E0E5F2E0A0E8B5E001900D928A95E1F79E
:10F79000011102C0222019F082E00E944E5382E53E
:10F7A0000E94D36B882371F18091250C9091260CD7
:10F7B000009709F457C0FC015F012191322F3F7D72
:10F7C00099F0253411F02536B9F7D5011C9260E087
:10F7D00070E08091250C9091260C2A8F0E94FDAF3D
:10F7E0002A8DF501208304C060E070E00E94FDAF27
:10F7F0006B017C0120E030E0A9010E946DAC882300
:10F8000089F106C0C12CD12C20E8E22E30E4F32E81
:10F81000011105C0311003C0112309F410C1C60144
:10F82000D7018093880590938905A0938A05B093AA
:10F830008B05209158023091590240915A02509103
:10F840005B02B601C7010E9470AE18165CF4198203
:10F850001A821B821C82BE016F5F7F4F88E895E091
:10F860000E94575001110CC0332009F4FCC0111143
:10F8700007C080E00E944E53002309F47EC1DCC023
:10F880001092540210925502109256021092570292
:10F890001092500210925102109252021092530292
:10F8A0000E94BE4EE6E3F4E12491298FE5E4F4E101
:10F8B00085909590A590B490E9E4F4E14590559039
:10F8C00065907490A3019201C501B4010E9470AECD
:10F8D00018162CF4A5019401C301B20104C0A301C0
:10F8E0009201C501B4010E9474AC6B017C01EEE28F
:10F8F000F4E185919591A591B4918D879E87AF870D
:10F90000B88BEAE2F4E185919591A591B491898B48
:10F910009A8BAB8BBC8B2D853E854F855889BC015E
:10F92000CD010E946DAC87FD09C09D859D8BAE8584
:10F93000AE8BBF85BF8BE889ED8708C0F989FD8B49
:10F940002A892E8B8B898F8B9C899D87A701960195
:10F95000C701B6010E94ABAE20E030E040E85FE3B3
:10F960000E9494AB0E9418AF9B01AC016D897E8907
:10F970008F899D850E94ABAE69877A878B879C872C
:10F98000E7E3F4E1F49020E030E040EC5FE3C30112
:10F99000B2010E94ABAE2B013C016F2DFF0C770B27
:10F9A000880B990B0E940FAD9B01AC01C301B20102
:10F9B0000E94ABAE69837A838B839C8320E030E026
:10F9C00040EC5FE3C501B4010E94ABAE6B017C016A
:10F9D000A98D6A2FAA0F770B880B990B0E940FAD88
:10F9E0009B01AC01C701B6010E94ABAE6D837E8363
:10F9F0008F839887AE01475F5F4FBE016F5F7F4F78
:10FA0000CE0105960E9475500E943D30109254021E
:10FA10001092550210925602109257021092500204
:10FA2000109251021092520210925302011121CFF2
:10FA30003110A0C0112319F081E00E944E530E94A2
:10FA4000BE4EF090E70480E00E946330812C912C40
:10FA500090EAA92E90E4B92E89829A82AB82BC8268
:10FA6000011115C0A8C01111E7CF0E94BE4EF09041
:10FA7000E70480E00E94633080E090E0A0EAB0E418
:10FA800089839A83AB83BC83222009F48BC080E0F6
:10FA900090E0ADE1B3E48D839E83AF83B887BE0170
:10FAA0006F5F7F4FCE0105960E94575080E090E037
:10FAB000A0EAB0E489839A83AB83BC8301110BC0B5
:10FAC000111109C08091540290915502A0915602E3
:10FAD000B091570204C080E090E0A9E3B3E48D83C5
:10FAE0009E83AF83B88701110BC0311009C080918C
:10FAF000500290915102A0915202B091530204C061
:10FB000080E090E0A0EAB0E489879A87AB87BC8761
:10FB1000AE014F5F5F4FBE016B5F7F4FCE01099615
:10FB20000E9475508F2D0E9463300E943830888D5E
:10FB30000E94661A0E94B5500E94964E80E00E9474
:10FB40008A156A960FB6F894DEBF0FBECDBFDF915F
:10FB5000CF911F910F91FF90EF90DF90CF90BF90CA
:10FB6000AF909F908F907F906F905F904F903F905D
:10FB70002F90089580E00E944E5311115DCF0E9496
:10FB8000BE4EF090E70480E00E946330812C912CFF
:10FB900080EAA82E80E4B82E89829A82AB82BC8249
:10FBA00021101FC08091580290915902A0915A02D1
:10FBB000B0915B0270CF2220A9F380E090E0ADE12C
:10FBC000B3E48D839E83AF83B887BE016F5F7F4FA1
:10FBD000CE0105960E94575089829A82AB82BC82E0
:10FBE0006FCF80E090E0ADE1B3E48D839E83AF837F
:10FBF000B887BE016F5F7F4FCE0105960E945750B8
:10FC000089829A82AB82BC825DCF80E1E0E5F2E03E
:10FC1000A0E8B5E001900D928A95E1F708954F9222
:10FC20005F926F927F928F929F92AF92BF92CF928C
:10FC3000DF92EF92FF920F931F93CF93DF93CDB795
:10FC4000DEB72E970FB6F894DEBF0FBECDBF2701EB
:10FC500038012E874A875B876C877D878987D5DF48
:10FC600089852E854A855B856C857D858F3F51F022
:10FC700094E0899FF0011124E058FA4F40835183AA
:10FC8000628373832F3F51F0A4E02A9FF001112477
:10FC9000E058FA4F4082518262827382BFEFCB16E6
:10FCA00051F084E0C89EF0011124E058FA4F8082A0
:10FCB0009182A282B3828090800590908105A0906D
:10FCC0008205B090830520E030E042E253E4C501B4
:10FCD000B4010E946DAC87FF11C020E030E040E429
:10FCE00050ECC501B4010E9470AE18166CF0812C66
:10FCF000912C30E4A32E30ECB32E06C0812C912C35
:10FD000022E2A22E23E4B22E8092800590928105F9
:10FD1000A0928205B092830540908405509085059D
:10FD2000609086057090870520E030E04EE353E454
:10FD3000C301B2010E946DAC87FF11C020E030E02A
:10FD400040EE50ECC301B2010E9470AE18166CF088
:10FD5000412C512C90EE692E90EC792E06C0412C4E
:10FD6000512C8EE3682E83E4782E409284055092C5
:10FD7000850560928605709287058091880590912F
:10FD80008905A0918A05B0918B058D839E83AF83F1
:10FD9000B88720E030E04FE153E4BC01CD010E9480
:10FDA0006DAC87FF11C020E030E040E050EC6D8189
:10FDB0007E818F8198850E9470AE18166CF080E06D
:10FDC00090E0A0E0B0EC04C080E090E0AFE1B3E4EC
:10FDD0008D839E83AF83B8878D819E81AF81B885E7
:10FDE0008093880590938905A0938A05B0938B052D
:10FDF00080E090E0A8E4B2E489839A83AB83BC837B
:10FE0000DE0111966D01ED80FE800F811885A30142
:10FE10009201C501B4010E94A34F2E960FB6F8942B
:10FE2000DEBF0FBECDBFDF91CF911F910F91FF902D
:10FE3000EF90DF90CF90BF90AF909F908F907F908A
:10FE40006F905F904F9008958F929F92AF92BF9264
:10FE5000CF92DF92EF92FF920F931F93CF93DF9396
:10FE6000EC016A017B0120E030E040E45FE368855B
:10FE700079858A859B850E9494ABA70196010E9493
:10FE800094ABAB01BC01812C912C5401CC24CA94BD
:10FE9000850174012FEF82E0C2DEEC80FD800E81CF
:10FEA0001F81488159816A817B8121E080E0B7DE32
:10FEB000DF91CF911F910F91FF90EF90DF90CF9046
:10FEC000BF90AF909F908F9008952F923F924F9246
:10FED0005F926F927F928F929F92AF92BF92CF92DA
:10FEE000DF92EF92FF920F931F93CF93DF93CDB7E3
:10FEF000DEB72E970FB6F894DEBF0FBECDBF898751
:10FF00008B014A87222359F0812C912C90E8A92E4D
:10FF10009EE3B92E80E090E0A0EAB1E40CC08AE054
:10FF2000882E87ED982E83E2A82E8CE3B82E80E0F1
:10FF300090E0A0E8BFE389839A83AB83BC8321115F
:10FF400005C080E090E0A0EAB0E404C080E090E06A
:10FF5000A8E4B2E48D839E83AF83B88756DE412C3C
:10FF6000512C3201B985A4E0BA9FC0011124FC01D3
:10FF7000E058FA4F1F01C801110FAA0BBB0B8B876A
:10FF80009C87AD87BE872D813E814F815885C301F7
:10FF9000B2010E946DAC87FF3FC06B857C858D856B
:10FFA0009E850E940FADA50194010E94ABAE9B01FE
:10FFB000AC01D1016D917D918D919C910E9494AB8A
:10FFC000F1016083718382839383E0908805F090D0
:10FFD000890500918A0510918B0520918405309147
:10FFE0008505409186055091870560918005709147
:10FFF00081058091820590918305DE0111966D0146
:020000021000EC
:100000000E94A34F0E949C5A83B182958170B1E0F7
:100010008B27EA858E1324C0398524E0329FF001B6
:100020001124E058FA4F60817181828193812E966C
:100030000FB6F894DEBF0FBECDBFDF91CF911F91F9
:100040000F91FF90EF90DF90CF90BF90AF909F9077
:100050008F907F906F905F904F903F902F9008957A
:10006000A5019401C301B2010E9494AB2B013C0194
:100070008ACF4F925F926F927F928F929F92AF92B0
:10008000BF92CF92DF92EF92FF920F931F93CF9385
:10009000DF93CDB7DEB728970FB6F894DEBF0FBE5B
:1000A000CDBFB82E6B01A42E4901C801B701FF24B2
:1000B000F39420E030E040EA50E40E946DAC8111FE
:1000C000F12CA3DD84E0B89E80011124F801E058F2
:1000D000FA4F80819181A281B3818D839E83AF830A
:1000E000B8872F2D4A2DB6018B2DEFDE2B013C0159
:1000F0008114910411F1F11020C041E04A256627D6
:1001000077276C197D0920E08B2DDFDEA30192019A
:100110000E9493AB6B017C0120E030E0A9010E94BA
:1001200070AE87FF04C0F7FAF094F7F8F094D401AA
:10013000CD92DD92ED92FC921397F801E058FA4FC0
:100140008D819E81AF81B88580839183A283B383A3
:1001500080E090E0A8E4B2E489839A83AB83BC8317
:10016000E0908805F090890500918A0510918B0533
:100170002091840530918505409186055091870531
:100180006091800570918105809182059091830531
:10019000DE0111966D010E94A34FC301B2012896A2
:1001A0000FB6F894DEBF0FBECDBFDF91CF911F9188
:1001B0000F91FF90EF90DF90CF90BF90AF909F9006
:1001C0008F907F906F905F904F9008952F923F9205
:1001D0004F925F926F927F928F929F92AF92BF9257
:1001E000CF92DF92EF92FF920F931F93CF93DF9303
:1001F000CDB7DEB769970FB6F894DEBF0FBECDBF9F
:100200003C014C8B5D8B6E8B7F8B2D878CE0E1E10D
:10021000F3E0DE01119601900D928A95E1F74C8989
:100220005D896E897F89C3010FDE2D852230D1F073
:1002300060F42223F1F0213009F073C1212C312C1C
:1002400060E8462E6FEB562E46C03D853330C9F12F
:10025000343009F066C1212C312C70E8472E7FEB39
:10026000572E36C0212C312CF0E84F2EFFE35F2EA5
:100270002FC09301205E3F4FEC88FD880E891F89B7
:1002800041E06FEF7FEF82E0F4DE6B017C0120E064
:1002900030E040E05FE369857A858B859C850E942C
:1002A000ABAE9B01AC01C701B6010E9493ABF30159
:1002B0006087718782879387C486D586E686F786AE
:1002C00030C1212C312CE0E84E2EEFE35E2E03C02E
:1002D000DD24D39401C0D12C2D2D30E03F872E8713
:1002E000002309F463C0C901880F991F880F991F63
:1002F0007301E80EF91EE1E0F0E0EC0FFD1FE80FDE
:10030000F91F20E030E040E05FE36081718182818D
:1003100093810E94ABAEF701E05CFF4F20813181F9
:10032000428153810E9493AB9B01AC01C201B10198
:1003300090580E94ABAEF7012081318142815381F8
:100340000E9494ABAB01BC01812C912C5401CC24B4
:10035000CA94850174012FEF8D2D61DCEC88FD8836
:100360000E891F899301205E3F4F41E06FEF7FEFC1
:1003700082E07FDE4B015C01F3016487758786872D
:10038000978720E030E040E05FE369857A858B85E0
:100390009C850E94ABAE9B01AC01C501B4010E94DB
:1003A00093ABF30160877187828793878E859F85E2
:1003B000880F991F880F991F9301280F391F3F87B6
:1003C0002E87E1E0F0E0EC0FFD1FE80FF91F20E0C1
:1003D00030E040E05FE360817181828193810E941F
:1003E000ABAE688B798B8A8B9B8B52014101B7FA3C
:1003F000B094B7F8B0948E859F85805C9F4F998F9D
:10040000888F20E030E040E05FE3FC016081718193
:10041000828193810E94ABAE9B01AC01688979898E
:100420008A899B890E9494AB2C893D894E895F897A
:100430000E9494AB9B01AC01C501B4010E94ABAE1C
:10044000EE85FF8520813181428153810E9494ABEA
:10045000AB01BC01812C912C5401CC24CA948501A0
:1004600074012FEF8D2DDBDB23E333E343E35FE305
:10047000F30164857585868597850E9493ABAB01F2
:10048000BC012FEF82E0CBDBFD85AF2EB12C450107
:1004900028E0820E911C880C991C880C991C860CF3
:1004A000971CC201B1010E94DCACEC88FD880E896A
:1004B0001F89940141E08D2DDCDD6B017C0120E082
:1004C00030E040E05FE3E88DF98D608171818281E9
:1004D00093810E94ABAE9B01AC01688979898A89BE
:1004E0009B890E9494AB9B01AC01C201B1010E94A7
:1004F000ABAE9B01AC01C701B6010E9494ABEE8587
:10050000FF856083718382839383F5013396EE0FB9
:10051000FF1FEE0FFF1FE60DF71DC082D182E282A2
:10052000F38269960FB6F894DEBF0FBECDBFDF91A0
:10053000CF911F910F91FF90EF90DF90CF90BF90E0
:10054000AF909F908F907F906F905F904F903F9073
:100550002F900895CF92DF92EF92FF920F93CF9357
:10056000DF93EC016A017B0100E020E02FDE22E056
:10057000B701A601CE012ADE23E0B701A601CE0114
:1005800025DEB701A601CE015FDC1CAA1DAA1EAAAA
:100590001FAA18AE19AE1AAE1BAE288539854A853A
:1005A0005B8560E070E0CB010E9493AB6CAF7DAFE8
:1005B0008EAF9FAFDF91CF910F91FF90EF90DF90C3
:1005C000CF9008958F929F92AF92BF92CF92DF9279
:1005D000EF92FF920F931F93CF93DF93EC01C090A4
:1005E0003A0CD0903B0CE0903C0CF0903D0C80E03D
:1005F00090E0A0E8BFE380933A0C90933B0CA0936B
:100600003C0CB0933D0C8090670290906802A090E3
:100610006902B0906A02109267021092680210920A
:10062000690210926A02CE0195DF0E949C5A00E591
:1006300012E02CAD3DAD4EAD5FADF801608571852A
:10064000828593850E9494ABF801608771878287C9
:100650009387188619861A861B861CAE1DAE1EAEA1
:100660001FAE0E94BE4E8092670290926802A092D6
:100670006902B0926A02C0923A0CD0923B0CE092AE
:100680003C0CF0923D0CDF91CF911F910F91FF90A8
:10069000EF90DF90CF90BF90AF909F908F90089594
:1006A0002F923F924F925F926F927F928F929F9282
:1006B000AF92BF92CF92EF92FF920F931F93CF937F
:1006C000DF93CDB7DEB728970FB6F894DEBF0FBE25
:1006D000CDBF5C0180913A0C90913B0CA0913C0CF9
:1006E000B0913D0C8D839E83AF83B88710923A0CF6
:1006F00010923B0C10923C0C10923D0C80916702C2
:1007000090916802A0916902B0916A0289839A83EC
:10071000AB83BC8310926702109268021092690248
:1007200010926A02C50116DFEEE3FCE0D5019C964B
:100730004D915D916D917C919F9740835183628330
:10074000738398964D915D916D917C919B974483B5
:1007500055836683778390964D915D916D917C91E1
:100760009397408751876287738780E090E0A0E885
:10077000BFE380933A0C90933B0CA0933C0CB09356
:100780003D0C10926702109268021092690210925A
:100790006A0280E5282E82E0382E20E030E040E436
:1007A00050E4F10160857185828593850E9494AB48
:1007B0004B015C0120E030E040E450E4D1011496AC
:1007C0006D917D918D919C9117970E9494AB2B0117
:1007D0003C0120E030E040E450E4F10160817181AF
:1007E000828193810E9494ABAB01BC0192E0C92E3F
:1007F0008301720121E080E012DA20E030E040E481
:1008000050E4D10118966D917D918D919C911B972B
:100810000E9493AB4B015C0120E030E040E450E4E7
:10082000F10164817581868197810E9493AB2B01D0
:100830003C0120E030E040E450E4D1016D917D9135
:100840008D919C910E9493ABAB01BC01830172011D
:1008500021E080E0E4D989819A81AB81BC818093D9
:10086000670290936802A0936902B0936A028D8137
:100870009E81AF81B88580933A0C90933B0CA093F6
:100880003C0CB0933D0C28960FB6F894DEBF0FBE1B
:10089000CDBFDF91CF911F910F91FF90EF90CF903F
:1008A000BF90AF909F908F907F906F905F904F9090
:1008B0003F902F9008958F929F92AF92BF92CF92C8
:1008C000DF92EF92FF92C0903A0CD0903B0CE090F8
:1008D0003C0CF0903D0C812C912C20E8A22E2FE3B3
:1008E000B22E80923A0C90923B0CA0923C0CB092AB
:1008F0003D0C8090670290906802A0906902B090D1
:100900006A021092670210926802109269021092B5
:100910006A0258DE8092670290926802A092690291
:10092000B0926A02C0923A0CD0923B0CE0923C0C1E
:10093000F0923D0CFF90EF90DF90CF90BF90AF9082
:100940009F908F9008959C018CE0EDE1F3E0D90138
:1009500001900D928A95E1F798E0E9E2F3E0D90180
:10096000A05CBF4F01900D929A95E1F708954F92C8
:100970005F926F927F928F929F92AF92BF92CF922F
:10098000EF92FF920F931F93CF93DF93CDB7DEB714
:10099000CC54D1090FB6F894DEBF0FBECDBFCE0147
:1009A0000196D1DF40903A0C50903B0C60903C0C8B
:1009B00070903D0C80E090E0A0E8BFE380933A0C9B
:1009C00090933B0CA0933C0CB0933D0C809167023C
:1009D00090916802A0916902B0916A022D968CAF45
:1009E0009DAFAEAFBFAF2D97109267021092680215
:1009F0001092690210926A0240E050E060EA70E4EE
:100A0000CE01019658DF40E050E060E87FE3CE0180
:100A1000019646DE40E050E060E87FE3CE010196BB
:100A20004ADF812C912C5401CC24CA948501740195
:100A30002FEF40E050E066E173E480E0F0D82D96BF
:100A40008CAD9DADAEADBFAD2D97809367029093F9
:100A50006802A0936902B0936A0240923A0C5092E5
:100A60003B0C60923C0C70923D0CC45BDF4F0FB6A8
:100A7000F894DEBF0FBECDBFDF91CF911F910F91D4
:100A8000FF90EF90CF90BF90AF909F908F907F900E
:100A90006F905F904F9008959F92AF92BF92CF92C8
:100AA000DF92EF92FF920F931F93CF93DF93CDB717
:100AB000DEB7C854D1090FB6F894DEBF0FBECDBF64
:100AC00081E00E948A1500914502109245029090A3
:100AD000150680E00E94661A41E061E081E00E9414
:100AE000FD518111EEC0CE0101962DDF85E50E94FA
:100AF0008C6B882341F12091250C3091260C211517
:100B0000310509F1F9015F011191812F8F7D99F074
:100B1000153411F01536B9F7F501108260E070E078
:100B20008091250C9091260C0E94FDAF6B017C01F9
:100B3000F50110830EC060E070E0C9010E94FDAFB6
:100B40006B017C0106C0C12CD12C80E8E82E8FE31C
:100B5000F82E82E40E948C6B882331F0B701A60145
:100B6000CE0101969DDDADC084E50E948C6B88238B
:100B700091F08091250C9091260C009731F04AE07D
:100B800050E060E070E00E9463B1B701A601CE01C1
:100B9000019618DD96C086E50E948C6B882309F4C7
:100BA0008FC0B701A601CE010196D4DC8AE00E9475
:100BB000721888EA99E10E94E2154D855E856F857D
:100BC000788980EA99E10E942D168AE00E947218C5
:100BD000498D5A8D6B8D7C8D87E999E10E942D1688
:100BE0008AE00E9472184D895E896F89788D8DE840
:100BF00099E10E942D168AE00E9472188AE00E94F4
:100C0000721884E899E10E94E21549855A856B853E
:100C10007C8581E899E10E942D168AE00E94721875
:100C20008AE00E94721886E799E10E94E2154DA5BC
:100C30005EA56FA578A98DE699E10E942D168AE040
:100C40000E94721849A55AA56BA57CA583E699E177
:100C50000E942D168AE00E94721849A15AA16BA128
:100C60007CA18BE599E10E942D168AE00E94721802
:100C70008AE00E9472188DE399E10E94E2158AE0F1
:100C80000E94721884E50E9472186AE070E080E0A9
:100C900090E00E94651989E299E10E94E21521968F
:100CA0004CAD5DAD6EAD7FAD219786E299E10E94BE
:100CB0002D168AE00E9472188AE00E94721801C004
:100CC00056DE892D0E94661A0093450280E00E943C
:100CD0008A15C85BDF4F0FB6F894DEBF0FBECDBFDD
:100CE000DF91CF911F910F91FF90EF90DF90CF9008
:100CF000BF90AF909F9008951F93CF93DF93CDB790
:100D0000DEB72C970FB6F894DEBF0FBECDBF83E5DC
:100D10000E948C6B8823B9F08091250C9091260C51
:100D2000892BC9F00E94166C97FD10C00E94166CAA
:100D30006F3F71058105910509F06CF40E94166CF6
:100D4000611109C003C01091150606C080E00E9421
:100D5000661A10E001C011E080915002909151029A
:100D6000A0915202B091530289839A83AB83BC83D2
:100D70008091540290915502A0915602B091570271
:100D80008D839E83AF83B8878091580290915902DA
:100D9000A0915A02B0915B0289879A87AB87BC8782
:100DA00086E50E948C6B882331F06DED79E181EF4F
:100DB00095E00E9445A6812F0E94661A112351F0EA
:100DC00080911506811106C00E94F3158EEB99E102
:100DD0000E94E2150E94F01580EB99E10E94E21555
:100DE000809115060E946F164CE050E060E572E0BD
:100DF000CE0101960E9425B4892B59F02C960FB68E
:100E0000F894DEBF0FBECDBFDF91CF911F910C9440
:100E1000964E2C960FB6F894DEBF0FBECDBFDF9175
:100E2000CF911F9108958F929F92AF92BF92CF92D0
:100E3000DF92EF92FF92CF934B015C0169017A013F
:100E400022ED30E040EE50ECC701B6010E9470AEDA
:100E500087FD33C027E030E04EE353E4C701B6011D
:100E60000E946DAC18164CF123EA31E040E450ECDE
:100E7000C501B4010E9470AE87FD1FC027E030E0BD
:100E800042E253E4C501B4010E946DAC1816ACF007
:100E900027E030E041E253E4C501B4010E946DACAB
:100EA00018165CF0C1E027E030E041E253E4C701EE
:100EB000B6010E946DAC18160CF4C0E08C2FCF91D7
:100EC000FF90EF90DF90CF90BF90AF909F908F906A
:100ED0000895CF93DF93D82FC62F0E94D36B88231A
:100EE000D1F08091250C9091260C892B11F481E092
:100EF0001AC00E94166C97FD15C00E94166C6F3FB9
:100F000071058105910509F094F70E94166C81E046
:100F1000611109C007C08D2F0E948C6B8111E7CF32
:100F20008C2F01C080E0DF91CF9108952F923F92E6
:100F30004F925F926F927F928F929F92AF92BF92E9
:100F4000CF92DF92EF92FF920F931F93CF93DF9395
:100F5000CDB7DEB7CB51D1400FB6F894DEBF0FBE90
:100F6000CDBF81E00E948A1541E061E081E00E94EE
:100F7000FD5181111AC080911506882329F060E087
:100F80008FE4A7DF811111C0FE0131968CE3DF01F0
:100F90001D928A95E9F7309015068AE40E948C6BC1
:100FA000982E882329F00E94851A912C0C94A791E1
:100FB00060E070E086E50E94D774C351DF4F9983EB
:100FC0008883CD5ED040059718F080EC9BE136C158
:100FD00060E084E47EDFC950DF4F8883C75FD04084
:100FE000C351DF4F28813981CD5ED0402330310598
:100FF0004CF460E084E56DDFC450DF4F8883CC5F44
:10100000D04006C031E0C450DF4F3883CC5FD040C1
:1010100062E070E088E50E94D774182F62E070E00B
:1010200089E50E94D774082F80E50E94D36B811157
:1010300003C0612F802F03C00E94166C862F623080
:1010400019F087E99BE1FAC0823019F08EE69BE146
:10105000F5C083E50E94D36B882319F00E94DF6BF3
:1010600004C060E070E88BEB95E420E030E040E7FE
:1010700052E40E9474AC60934602709347028093DE
:1010800048029093490288E40E948C6B882391F176
:101090000E94DF6B0E94DCAC8B0177FF02C00F5F08
:1010A0001F4F15950795119501951109035B1F4F6A
:1010B0000E3F4FEF14072CF44DEFA42EBB24BA942F
:1010C00001C058016501C60ED71E51EAC516D104EC
:1010D0001CF031EAC32ED12C0A3FAFEF1A0714F4EB
:1010E00009EF1FEF7801E60EF71EB1EAEB16F104E7
:1010F000CCF135C08CE40E94D36B882331F00E9480
:10110000DF6B0E94DCAC5B0104C02DEFA22EBB2480
:10111000BA9482E50E94D36B882331F00E94DF6B82
:101120000E94DCAC6B0103C091EAC92ED12C86E48D
:101130000E94D36B882331F00E94DF6B0E94DCACED
:101140008B0102C009EF1FEF82E40E94D36B88235A
:1011500031F00E94DF6B0E94DCAC7B0103C081EAAE
:10116000E82EF12CB801012E000C880B990B0E947F
:101170000FADC250DF4F688379838A839B83CE5F34
:10118000D040B5010B2C000C880B990B0E940FADC1
:10119000CE5FDE4F688379838A839B83C250D140C0
:1011A000C250DF4F288139814A815B81CE5FD040B8
:1011B0003ADE882309F440C0B7010F2C000C880BDD
:1011C000990B0E940FAD9B01AC01B6010D2C000CD8
:1011D000880B990BC85EDE4F2883C851D140C75E8B
:1011E000DE4F3883C951D140C65EDE4F4883CA51B5
:1011F000D140C55EDE4F5883CB51D1400E940FAD28
:10120000C85EDE4F2881C851D140C75EDE4F3881AD
:10121000C951D140C65EDE4F4881CA51D140C55E3A
:10122000DE4F5881CB51D140FEDDCA50DF4F88835D
:10123000C65FD040811106C082E59BE10E94E215A5
:101240000C94A791B6016A197B09072E000C880B34
:10125000990B0E940FADC65FDE4F688379838A8346
:101260009B83CA50D140B701601B710B072E000C45
:10127000880B990B0E940FADC25FDE4F68837983A4
:101280008A839B83CE50D140C351DF4FE881F981DF
:10129000CD5ED040EF2B91F08CE39BE10E94E215F4
:1012A000C950DF4FE881C75FD040EE2321F082E3D1
:1012B0009BE10E94E2158AE00E9472180E949C5AEB
:1012C00080E00E94661A81E00E94524B882329F038
:1012D000832D0E94661A0C94A7910E94965060E09C
:1012E00085E4F7DD811107C0F2E0C350DF4FF883DA
:1012F000CD5FD04006C021E0C350DF4F2883CD5FD3
:10130000D040C151DF4F19821882CF5ED040C75202
:10131000DF4F188219821A821B82C95DD040C850E3
:10132000DF4F188219821A821B82C85FD040C751D2
:10133000DF4F1882C95ED0404FEF5FEFC352DF4FDF
:1013400059834883CD5DD0405FEFCB50DF4F58834A
:10135000C55FD0408FEFCD50DF4F8883C35FD04053
:1013600091E0CB52DF4F9883C55DD040C352DF4F31
:1013700088819981CD5DD0400196880F991F880F93
:10138000991F4DE350E04C0F5D1F480F591FCB5183
:10139000DF4F59834883C55ED040DC011497C85F96
:1013A000DE4FB983A883C850D1408CE0C352DF4FD1
:1013B00028813981CD5DD040829FF001839FF00D5F
:1013C0001124CA5FDE4FF983E883C650D140CF5164
:1013D000DF4F19821882C15ED040C151DF4F888132
:1013E0009981CF5ED040092E000CAA0BBB0BCE5EBC
:1013F000DE4F88839983AA83BB83C251D140C151F8
:10140000DF4FA881B981CF5ED040AA0FBB1FCA5E53
:10141000DE4FB983A883C651D140CB52DF4F5881EC
:10142000C55DD040CD50DF4F8881C35FD040581795
:1014300009F497C2CE5EDE4F688179818A819B81F3
:10144000C251D1400E940FAD9B01AC01C65FDE4F7F
:10145000688179818A819B81CA50D1400E94ABAE5C
:101460009B01AC01CE5FDE4F688179818A819B81CF
:10147000C250D1400E9494AB4B015C01CB52DF4F74
:10148000B881C55DD0406B2FBB0F770B880B990BD4
:101490000E940FAD9B01AC01C25FDE4F6881798174
:1014A0008A819B81CE50D1400E94ABAE9B01AC01A2
:1014B000C250DF4F688179818A819B81CE5FD040A5
:1014C0000E9494AB6B017C0120E030E0A901C501D2
:1014D000B4010E946DAC87FD05C020E030E040E023
:1014E0005FE303C020E030E0A901C501B4010E9420
:1014F00094AB0E944AADC355DF4F688379838A83DA
:101500009B83CD5AD04020E030E0A901C701B6014D
:101510000E946DAC87FD05C020E030E040E05FE355
:1015200003C020E030E0A901C701B6010E9494ABDE
:101530000E944AADC755DF4F688379838A839B83B6
:10154000C95AD040C352DF4FE881F981CD5DD04008
:101550003196C352DF4FF983E883CD5DD040CA5E38
:10156000DE4FE881F981C651D140CB52DF4F28814F
:10157000C55DD040E20FF11D27FDFA95EE0FFF1F6C
:1015800041EA50E04C0F5D1FE40FF51FC352DF4FDF
:1015900088819981CD5DD0409183808301E0C351E2
:1015A000DF4F2881CD5ED040C350DF4F4881CD5FF3
:1015B000D040BE0167557F4FCE0183559F4F0E949B
:1015C000F34BC752DF4F688379838A839B83C95D5E
:1015D000D0409B01AC010E9459AF882321F0832D9C
:1015E0000E94661AD5C1C752DF4F288139814A81CE
:1015F0005B81C95DD040C850DF4F688179818A81A5
:101600009B81C85FD0400E9494ABC850DF4F688375
:1016100079838A839B83C85FD040CF51DF4FE881B5
:10162000F981C15ED040C85FDE4FA881B981C85042
:10163000D140EA0FFB1F2DE630E02C0F3D1FE20FDB
:10164000F31FC752DF4F88819981AA81BB81C95D91
:10165000D04084839583A683B783C355DF4F4880EA
:1016600059806A807B80CD5AD040CB51DF4FA88112
:10167000B981C55ED0404D925D926D927D92CB5105
:10168000DF4FB983A883C55ED040CF51DF4FE881DB
:10169000F981C15ED0403496CF51DF4FF983E883A2
:1016A000C15ED040C755DF4F88809980AA80BB803B
:1016B000C95AD0401C968D929D92AD92BC921F97B4
:1016C00020E030E040E85FE35C962D933D934D933E
:1016D0005C935F97A301920169817A818B819C81E0
:1016E0000E9494AB69837A838B839C83A5019401C8
:1016F0006D817E818F8198850E9494AB6D837E83FE
:101700008F839887C752DF4F288139814A815B8157
:10171000C95DD04069857A858B859C850E9494AB94
:1017200069877A878B879C87A3019201C301B201E5
:101730000E94ABAE9B01AC016D857E858F8598893B
:101740000E9494AB6D877E878F87988BA50194014B
:10175000C501B4010E94ABAE9B01AC0169897A89D5
:101760008B899C890E9494AB698B7A8B8B8B9C8B29
:10177000C752DF4F288139814A815B81C95DD040E2
:10178000CA01B9010E94ABAE9B01AC016D897E8993
:101790008F89988D0E9494AB6D8B7E8B8F8B988FE9
:1017A000A5019401C301B2010E94ABAE9B01AC0143
:1017B000698D7A8D8B8D9C8D0E9494AB698F7A8F09
:1017C0008B8F9C8FC752DF4F288139814A815B8183
:1017D000C95DD040C301B2010E94ABAE9B01AC0118
:1017E0006D8D7E8D8F8D98A10E9494AB6D8F7E8FB5
:1017F0008F8F98A3C752DF4F288139814A815B813F
:10180000C95DD040C501B4010E94ABAE9B01AC01E3
:1018100069A17AA18BA19CA10E9494AB69A37AA330
:101820008BA39CA31DA10EA13FA028A420E030E023
:10183000A901C301B2010E9470AE7301620187FF6A
:1018400004C0F7FAF094F7F8F094212F302F432DCD
:10185000522DC701B6010E9470AE181624F0C12E99
:10186000D02EE32CF22CCDA2DEA2EFA2F8A619A571
:101870000AA53BA42CA420E030E0A901C501B401D5
:101880000E9470AE7501640187FF04C0F7FAF094FE
:10189000F7F8F094212F302F432D522DC701B601B8
:1018A0000E9470AE181624F0C12ED02EE32CF22C1C
:1018B000C9A6DAA6EBA6FCA620E030E040E85FE38C
:1018C00069AD7AAD8BAD9CAD0E9494AB69AF7AAF38
:1018D0008BAF9CAFC752DF4FC880D980EA80FB80B6
:1018E000C95DD04095018401B301A201CE018358A6
:1018F0009F4F0E94D3A1CF51DF4FA881B981C15E14
:10190000D040AA0FBB1FCF51DF4FE881F981C15EE4
:10191000D040AE0FBF1FCA5FDE4F28813981C6504D
:10192000D140A20FB31FA65BB34FFE01E358FF4F98
:101930008CE001900D928A95E1F70E94FBAACB52B0
:10194000DF4F3881C55DD040CB50DF4F4881C55F48
:10195000D040340FCB52DF4F3883C55DD040312C9F
:101960005CCDC151DF4FA881B981CF5ED0401197C6
:1019700079F0C752DF4F288139814A815B81C95D87
:10198000D040CA01B9010E9459AF882309F4A4C408
:1019900080E00E94524B882381F0832D0E94661ABA
:1019A00020E030E040EC5FE7C752DF4F2883398307
:1019B0004A835B83C95DD04071C4C752DF4F288121
:1019C00039814A815B81C95DD040CA01B9010E9459
:1019D00059AF811163C4CE0101960E94B6A78DA5AF
:1019E0009EA5AFA5B8A9C352DF4F88839983AA8368
:1019F000BB83CD5DD04029A93AA94BA95CA9CF51A1
:101A0000DF4F288339834A835B83C15ED0408DA931
:101A10009EA9AFA9B8ADCB51DF4F88839983AA8324
:101A2000BB83C55ED04020E030E040E85EE3C850B4
:101A3000DF4F688179818A819B81C85FD0400E9495
:101A4000ABAEC151DF4F688379838A839B83CF5EBE
:101A5000D040C351DF4FA881B981CD5ED040AB2BC0
:101A600009F480C142E65CE066E57CE0CE01835883
:101A70009F4F0E94A5A246E55CE06AE47CE0CE01AF
:101A800087579F4F0E94A5A2AE0143585F4FBE01EA
:101A900067577F4FCE018B569F4F0E94EDA1CB56CB
:101AA000DF4F488059806A807B80C559D040C75637
:101AB000DF4F88809980AA80BB80C959D040C35627
:101AC000DF4F288139814A815B81CD59D040CB528B
:101AD000DF4F288339834A835B83C55DD0402091E3
:101AE0006E0C30916F0C4091700C5091710CC301D1
:101AF000B2010E94ABAE6B017C012091720C30915F
:101B0000730C4091740C5091750CC501B4010E9486
:101B1000ABAE9B01AC01C701B6010E9494AB6B0157
:101B20007C012091760C3091770C4091780C50918B
:101B3000790CCB52DF4F688179818A819B81C55DA9
:101B4000D0400E94ABAE9B01AC01C701B6010E9420
:101B500094AB6B017C0180914A0C90914B0CA0914D
:101B60004C0CB0914D0CBC01CD019058A3019201D9
:101B70000E94ABAEC751DF4F688379838A839B8312
:101B8000C95ED04020914E0C30914F0C4091500CCA
:101B90005091510CC501B4010E94ABAE9B01AC0148
:101BA000C751DF4F688179818A819B81C95ED040AE
:101BB0000E9493ABC751DF4F688379838A839B83ED
:101BC000C95ED0402091520C3091530C4091540C7E
:101BD0005091550CCB52DF4F688179818A819B816E
:101BE000C55DD0400E94ABAE9B01AC01C751DF4F39
:101BF000688179818A819B81C95ED0400E9493ABC4
:101C00009B01AC01C701B6010E9494AB6B017C0142
